S0030000FC
S113000098080020DD000000E5000000E700000083
S113001000000000000000000000000000000000DC
S1130020000000000000000000000000EF000000DD
S11300300000000000000000F3000000F5000000D4
S1130040F7000000F9000000FB000000FD000000C4
S1130050FF00000001010000030100000501000091
S113006007010000090100000B0100000D01000060
S11300700F01000011010000130100001501000030
S113008017010000190100001B0100001D01000000
S11300901F010000210100002301000025010000D0
S11300A027010000290100002B0100002D010000A0
S11300B02F01000031010000330100003501000070
S11300C0EF3FE8FF0448854600F070F80048004719
S11300D0C9080000C046C04698080020164880475A
S11300E016480047FEE7FEE7FEE7FEE7FEE7FEE709
S11300F0FEE7FEE7FEE7FEE7FEE7FEE7FEE7FEE7D4
S1130100FEE7FEE7FEE7FEE7FEE7FEE7FEE7FEE7C3
S1130110FEE7FEE7FEE7FEE7FEE7FEE7FEE7FEE7B3
S1130120FEE7FEE7FEE7FEE7FEE7FEE7FEE7FEE7A3
S1130130FEE7FEE7FEE7000019070000C500000027
S113014030B50B46014600202022012409E00D466B
S1130150D5409D4205D31D469540491B25469540F3
S113016040191546521E002DF1DC30BDD2B201E01B
S11301700270401C491EFBD270470022F6E710B5FE
S113018013460A4604461946FFF7F0FF204610BD01
S113019030B504460020034600E05B1C934203D2C2
S11301A0E05CCD5C401BF8D030BD0000064C01255E
S11301B0064E05E0E36807CC2B430C3C984710340B
S11301C0B442F7D3FFF782FF3C0C00005C0C000044
S11301D0F8B504460D460020002C00D100BF002ACB
S11301E000D100BF012C01D141263043012A01D1A5
S11301F012263043022C01D1C0263043022A01D1F9
S113020030263043134E307076788027BE43114F2A
S11302107E70012C08D1FF2100BF0E4EB3781E461C
S11302200E4033468B42F8D10A4E76784027BE43BF
S1130230084F7E70012A0BD10026009603E000BF10
S1130240009E761C0096FF276937009EBE42F6D9B1
S1130250F8BD00000004024001200649087000BFF8
S113026004480078802108400028F9D00120024980
S113027008707047000C02408400002070B50346EB
S113028014460020002B01D1C0B202E0054680359F
S1130290E8B2012902D1051DE8B206E0022903D122
S11302A005460835E8B200E0C0B2012C02D1851C35
S11302B0E8B200E0C0B2084DA870AD78012635431D
S11302C0054EB570002201E000BF521C7D252D01B2
S11302D0AA42F9D970BD0000000C024070B5002498
S11302E02448007920210840002801D0224D3FE015
S11302F000F046F80546214800788021084000288F
S113030036D01E4880780840002801D01A4D02E0FB
S113031000F036F80546194880780007840F022C4F
S113032001DBAD0804E0012C01D16D0800E000BF41
S1130330124880788007C00F002801D02D0101E009
S11303400C2045430D4800784007840F002C02D14F
S1130350601CC4B207E0032C03D1601C4006040EE9
S113036001E06006040E21462846FFF7E9FE054633
S1130370284670BD0004024000127A00000C0240BE
S113038000B5C0229178F82211401C4A127811431A
S1130390EA2923D00ADC0A46E03A130000F01BFAEB
S11303A00A181C20242A2A2A2A161A2AED291FD0C0
S11303B004DCEB2916D0EC291CD117E0F02903D07A
S11303C0F82917D10E4817E00E4815E00E4813E03F
S11303D00E4811E00E480FE00E480DE00E480BE009
S11303E00E4809E00E4807E00E4805E00E4803E019
S11303F00E4801E00D4800BF00BF00BD201C0240B4
S11304000090D003006CDC020048E80100366E0165
S11304100024F400001BB70000127A00808D5B00FA
S113042000093D00C0C62D0080841E0040420F001C
S113043070B500250F24E402102221462031104813
S1130440FFF7A6FE002819D14022214630310C487E
S11304501030FFF79DFE002810D11022A118084883
S11304601038FFF795FE002808D1102221460448D1
S11304702038FFF78DFE002800D10125284670BDE5
S113048024000020F0B591B05548006800790006BA
S1130490534909684968FF221202114009020843BE
S11304A04F490968496812021140090A08434C4936
S11304B009684968090E08434A49086048480068C1
S11304C0007A0006464A12689268FF231B021A400B
S11304D012021043424A126892681B021A40120A1E
S11304E010433F4A12689268120E1043052292028A
S11304F08118104600F098F80526B60238480068BE
S1130500007A000636490968097AFF22120211406E
S11305100902084332490968098912021140090A8B
S113052008432F4909688968090E08438006800E2C
S1130530002818D12A480068007A0006284909686A
S1130540896812121140090208432549096889681B
S113055012021140090A0843214909688968090EF1
S11305600843800919E01E480068007A00061C4907
S113057009688968FF2212021140090208431849D8
S11305800968896812021140090A08431449096874
S11305908968090E08438009401C074600251AE0B3
S11305A0FF22402101A8FFF7E1FD002407E0A80194
S11305B000190C490968085C01A90855641C402C01
S11305C0F5D3402201A9304600F004FA00F0EEF819
S11305D040366D1C7F1E002FE2D111B0F0BD00002B
S11305E0740000208000002010B50020002113E0DA
S11305F0084608220AE0C307DB0F002B04D0430897
S1130600074C6340184600E04008521E002AF2D10D
S11306108B00044CE050491CFF29E9D910BD0000AF
S11306202083B8ED9400002070B505460E462C4694
S113063005E0204600F008F8FF34FF340234B442E9
S1130640F7D3002070BD0000014610200D4AD06091
S1130650F120106255205060AA2090600020C04311
S1130660086000BF07480068C007C00F0028F9D021
S11306700448006801221043024A10600020D06040
S113068010627047000002400246F1200B4B1862D2
S1130690AA20586055209860116000BF0748006880
S11306A0C007C00F0028F9D004480068012318438C
S11306B0024B1860002018627047000000000240DE
S11306C010B501231A4600211846FFF781FD0122C7
S11306D011461046FFF7D2FDFFF7BEFD014800F0BA
S11306E0E5F810BD0090D0031A20084908722B20A9
S11306F048723C2088724D20C8727F2004490968E2
S11307000860AC20034948707047000000040240B0
S1130710000000200010024010B580201B494871E1
S11307201A201A49203908722B2048723C208872FA
S11307304D20C872002016494860FFF7CFFD1549C7
S113074008600020C0431449086014490860144834
S113075014490860114903221202891848600F499C
S1130760891888600D498918C8600C49891808617E
S11307700A4989184861094989188861074989180B
S1130780C861AC200849487010BD00002004024034
S113079000B001409000002080E200E000E100E0B1
S11307A0C0C0C0C000E400E000100240AC20014919
S11307B04870704700100240F0B506460F461446D4
S11307C0354605E028462168FFF75EFF241D2D1DF0
S11307D0BD42F7D3F0BD30B47446641E2578641C62
S11307E0AB4204D3635D5B00E31830BC18471D467D
S11307F0F8E702E008C8121F08C1002AFAD17047BE
S11308007047002001E001C1121F002AFBD170478C
S1130810F0B501460022D24308780006FF273F02C4
S11308200E683E40360230433F020E683E40360AB0
S113083030430E68360E30430446087900063F12F2
S11308404E683E40360230433F024E683E40360A10
S113085030434E68360E30430346087A00063F1292
S11308608E683E40360230433F028E683E40360A70
S113087030438E68360E3043054609E018785B1C19
S113088050400006800D084E3058160A704002464B
S113089028466D1E0028F1D1D243A24201D1012085
S11308A0F0BD0020FCE700009400002010B50446D1
S11308B003492046FFF744FC0249087010BD0000BC
S11308C040420F008C00002010B501246407394811
S11308D03949086039483A4908603A483A49086051
S11308E0354800680068401C002852D0324800682F
S11308F0006833490968096888424AD03248006868
S11309004068002845D12C480068007A00062A492E
S113091009688968FF221202114009020843264926
S11309200968896812021140090A084322490968C2
S11309308968090E08430521890240180721090323
S1130940884226D2FFF750FEFFF772FD012820D11E
S113095019480068FFF75CFF00281AD0FFF7B0FEC3
S1130960FFF7C2FEFFF78EFD144800F05EF80C227C
S113097011480168114800F02DF800BFBFF34F8FF4
S113098012481349C860BFF34F8F00BF00BF00BFB8
S1130990FDE772B6032109032046FFF7EEFB0521AC
S11309A08902086880F3088800BF486880470020EF
S11309B010BD000010700000740000200002500000
S11309C078000020000450007C0000200400FA0598
S11309D000ED00E0F8B504460D4616460027A119BF
S11309E02A462046FFF7E8FE3846F8BD014672B6AF
S11309F008208F4AD060F120106255205060AA2050
S1130A0090600020C043086000BF89480068C007A8
S1130A10C00F0028F9D00120854A10600020D06062
S1130A20F020106262B600207047014672B61020B2
S1130A307F4AD060F120106255205060AA20906057
S1130A400020C043086000BF79480068C007C00F99
S1130A500028F9D00120764A10600020D060F020F0
S1130A6010621046006804221040002805D00420BB
S1130A706F4A106062B60120704762B60020FBE73F
S1130A8070B503461D46F120694E3062002415E01E
S1130A9072B6AA20664E70605520B0601078287037
S1130AA0521C6D1C62B600BF61480068C007C00FCD
S1130AB00028F9D001205E4E3060641C8C42E7D3DC
S1130AC0F0205B4E3062002070BDF7B5FFB0FFB080
S1130AD089B006460F460021FFA8C1610121049197
S1130AE04802874206D9FFA8C161C0697FB07FB0C0
S1130AF00CB0F0BD029600240DE002980078FFA926
S1130B0088610298401C02908869FF2801D0002067
S1130B100490601C84B2BC42EFD30498002809D02E
S1130B20444845490860FFA83946826A3046FFF7C1
S1130B30A7FF6DE0750AF119681C4002814202D9D1
S1130B400120039001E000200390710A4902019101
S1130B50F105C90D0091039800280FD0002408E086
S1130B600198007805A908550198411C0191601C61
S1130B7084B2012080028442F2DB0EE0002408E00B
S1130B800198007805A908550198411C0191601C41
S1130B9084B2012040028442F2DB00240DE0FFA86D
S1130BA0806A01780098001905AA1154FFA8806A88
S1130BB0411CFFA88162601C84B2BC42EFD303983D
S1130BC0002816D01B481C4908606802FFF72DFF57
S1130BD0184819490860691C4802FFF726FF1548A0
S1130BE015490860680205AA01218902FFF748FF38
S1130BF00EE01048104908606802FFF716FF0D4820
S1130C000D490860680205AA01214902FFF738FF6F
S1130C10FFA8C0696AE730B50446002304E02578DC
S1130C201570641C521C5B1C8B42F8D330BD000051
S1130C3000000240CDAB3412880000205C0C0000A0
S1130C400000002094000000F2070000F00C0000F7
S1130C50940000200408000002080000C000000006
S1130C605469616E59696E673130300000000000CC
S1130C7054593230302E3038303030306200000079
S1130C80424154333247313339474B3634464200BC
S1130C9043414E5F53544400000000000000000034
S1130CA043414E5F43485F300000000000000000F5
S1130CB043414E5F3530304B6270730000000000DA
S1130CC0E8070000E0070000DF0700000000000064
S1130CD00000000000000000000000000000000010
S1130CE00000000000000000000000000000000000
S1130CF0FFFFFFFFFFFFFFFFFFFFFFFFFFFFFFFF00
S1130D00FFFFFFFFFFFFFFFFFFFFFFFFFFFFFFFFEF
S113140090210020DD140000E5140000E714000022
S113141000000000000000000000000000000000C8
S1131420000000000000000000000000EF140000B5
S11314300000000000000000F314000099440000C4
S11314404D39000091390000C1390000F139000024
S1131450213A0000513A0000813A0000B13A0000FC
S1131460E13A0000113B0000453B0000593B0000FD
S1131470693B00009D3B0000AD3B0000BD3B00000C
S1131480F13B0000353C00007D3C0000C53C000001
S11314900D3D0000553D0000653D0000993D0000F4
S11314A0CD3D0000FD3D0000313E0000653E0000E2
S11314B0753E0000853E0000B93E0000ED3E000090
S11314C0EF3FE8FF0448854600F084F800480047F1
S11314D0E9630000C046C0469021002016488047BA
S11314E016480047FEE7FEE7FEE7FEE7FEE7FEE7F5
S11314F0FEE7FEE7FEE7FEE7FEE7FEE7FEE7FEE7C0
S1131500FEE7FEE7FEE7FEE7FEE7FEE7FEE7FEE7AF
S1131510FEE7FEE7FEE7FEE7FEE7FEE7FEE7FEE79F
S1131520FEE7FEE7FEE7FEE7FEE7FEE7FEE7FEE78F
S1131530FEE7FEE7FEE7000061470000C514000077
S113154030B50B46014600202022012409E00D4657
S1131550D5409D4205D31D469540491B25469540DF
S113156040191546521E002DF1DC30BD70B5002423
S11315702546002801DA01244042002901DA012528
S11315804942FFF7DDFFAC4200D04042002C00D0BE
S1131590494270BDD2B201E00270401C491EFBD228
S11315A070470022F6E710B513460A46044619466A
S11315B0FFF7F0FF204610BD30B504460020034677
S11315C000E05B1C934203D2E05CCD5C401BF8D08E
S11315D030BD0000064C0125064E05E0E36807CC4B
S11315E02B430C3C98471034B442F7D3FFF76EFFFB
S11315F0E46D0000046E000070B58C180578401C82
S11316006B075B0F01D10378401C2A1106D10278C5
S1131610401C03E006780E70401C491C5B1EF9D187
S11316202B0705D40023521E0DD40B70491CFAE776
S11316300378401CCB1A921C03E01D780D70491CE2
S11316405B1C521EF9D5A142D8D3002070BD000006
S1131650F0B591B0072000031F49086001218904F7
S11316604720C00201F00AFF312002F027FE47267E
S1131670F602392464011094002726E0FF22402159
S11316806846FFF787FF002507E0B80140191249B3
S11316900968085C694648556D1C402DF5D30A203D
S11316A001F017F840226946304604F0B5FE04F014
S11316B08DFD40367F1C641E1098001B39210901E2
S11316C0884202D1312002F0F9FD002CD6D131201C
S11316D002F0F4FD11B0F0BDEC050020F0B591B0BE
S11316E04720C0021749086001460720000301F0A3
S11316F0C5FE07252D033926760100271DE0FF22AC
S1131700402101A8FFF746FF002407E0B8010019B3
S11317100C490968085C01A90855641C402CF5D3E0
S11317200A2000F0D6FF402201A9284604F074FEE6
S113173004F04CFD40357F1C761E002EDFD111B025
S1131740F0BD0000EC05002010B502F05DFC05487A
S11317500078012803D003480078032801D102F05F
S1131760CFFD10BDF00500200348044A0168116054
S1131770001D01685160704700045000FC05002002
S1131780072000030449086048600020088248825A
S1131790401E0249086070476C180020540600205F
S11317A0582211527047014600205322525C1023E4
S11317B01A40002A08D05322525C0C231A4092107B
S11317C0032A18D1032016E05422525A0123DB03C2
S11317D01A40002A0ED05322525C0C231A40921055
S11317E0032A05D05322525C9207920F032A01D197
S11317F0022000E0012070470246002058239B5A33
S11318000B40002B01D0012000E0002070470000B5
S1131810014600226020405AFF231B0218400005A5
S1131820020F1001014BC01870470000005504401E
S113183010B5002A0AD056231B5A0C0223435624FF
S1131840235256231B5A8B43235209E056231B5A17
S11318500C02A3435624235256231B5A0B432352F0
S113186010BD0000F8B504460D4601270026344893
S1131870844203D10121022000F0E4F92878401EBB
S1131880A0702088FF21013108432080208840086F
S113189040002080A878401EC1B25A2001556879C2
S11318A00007000CE97909020843A97908435C217F
S11318B00853288981B240200153A868C000C10C94
S11318C042200153A88981B244200153E868C00032
S11318D0C10C46200153288A81B24820015328694B
S11318E0C000C10C4A200153A88A81B24C20015384
S11318F06869C000C10C4E2001535020005B297957
S113190009020843502108535020005B2979884379
S11319105021085300E0761C5020005B4007400F24
S11319202979884202D007488642F4D15020005BCE
S11319304007400F2979884200D000273846F8BD77
S113194000540440FFFF00000146FF22C889C0077D
S1131950C00F00280AD00120C88100E0521EC889A7
S1131960C007C00F002801D0002AF7D1C889C007DA
S1131970C00F00280FD10220C8810420C881487AF2
S1131980400840004872487A38239843487200203F
S11319904872012070470020FCE700000246507A9C
S11319A0012318435072507A0B78DB0018435072AD
S11319B0087A012808D1888850814868000C0123DE
S11319C0DB031843908108E0087A002805D1508190
S11319D0486880001A4B18409081487A012804D145
S11319E0507A40231843507206E0487A002803D105
S11319F0507A4023984350720878002811D1C87A4D
S1131A001072087B1070487B5070887B9070CB7B81
S1131A10D370087C10714B7C5371887C9071CB7CA3
S1131A20D371887A002803D00120C002D08101E05C
S1131A300820D081FF200130D081012070470000B0
S1131A40FC1F0000002904D0427A80231A4342720A
S1131A5003E0427A80239A434272704730B50246CB
S1131A6000200F4B5024A45A0D022C435025AC5295
S1131A705024A45A8C43AC5200E05B1E5024A45A58
S1131A806407640F8C4201D0002BF6D15024A45A71
S1131A906407640F002C01D0002000E0012030BD59
S1131AA0FFFF0000827A80231A40802A00D08172CE
S1131AB07047000070B5044600250023002D02D0B5
S1131AC00126602006530420C88188890126F60374
S1131AD03040002808D0012010728889C004C00852
S1131AE04E893043506006E00020107288890F4E02
S1131AF0304080105060087AD072002304E0CE5C3D
S1131B0010460C30C6545B1CD07A9842F7DCC88966
S1131B1004263040002804D1C889F6023040002849
S1131B2001D0002070BDD07AFCE70000FC1F00004B
S1131B30027C80231A40802A00D00174704710B5BB
S1131B400246FF23D089C007C00F00280AD0012015
S1131B50D08100E05B1ED089C007C00F002801D0EF
S1131B60002BF7D1D089C007C00F002801D0002076
S1131B7010BD507A012420435072507A3824A04377
S1131B805072C87A1072487A00280FD1087B1070FE
S1131B90487B5070887B9070CC7BD470087C10712B
S1131BA04C7C5471887C9071CC7CD471FF200130C2
S1131BB0D0814000D081107ADAE70000F8B50446FD
S1131BC00D460020002C00D100BF002A00D100BF28
S1131BD0012C01D141263043012A01D11226304380
S1131BE0022C01D1C0263043022A01D130263043D1
S1131BF0134E307076788027BE43114F7E70012CCF
S1131C0008D1FF2100BF0E4EB3781E460E40334666
S1131C108B42F8D10A4E76784027BE43084F7E7037
S1131C20012A0BD10026009603E000BF009E761C1B
S1131C300096FF276937009EBE42F6D9F8BD000022
S1131C4000040240002905D0054A12780243044BDF
S1131C501A7004E0024A12788243014B1A707047EA
S1131C602004024001200649087000BF044800789F
S1131C70802108400028F9D00120024908707047EB
S1131C80000C02402400002070B5034614460020D6
S1131C90002B01D1C0B202E005468035E8B201292B
S1131CA002D1051DE8B206E0022903D10546083534
S1131CB0E8B200E0C0B2012C02D1851CE8B200E019
S1131CC0C0B2084DA870AD7801263543054EB570F5
S1131CD0002201E000BF521C7D252D01AA42F9D942
S1131CE070BD0000000C024070B500242448007947
S1131CF020210840002801D0224D3FE000F046F8A2
S1131D0005462148007880210840002836D01E4826
S1131D1080780840002801D01A4D02E000F036F81F
S1131D200546194880780007840F022C01DBAD08B2
S1131D3004E0012C01D16D0800E000BF1248807856
S1131D408007C00F002801D02D0101E00C2045437D
S1131D500D4800784007840F002C02D1601CC4B2E7
S1131D6007E0032C03D1601C4006040E01E060066A
S1131D70040E21462846FFF7E3FB0546284670BDBE
S1131D800004024000127A00000C024000B5C02298
S1131D909178F82211401C4A12781143EA2923D081
S1131DA00ADC0A46E03A130004F03CFA0A181C2044
S1131DB0242A2A2A2A161A2AED291FD004DCEB2900
S1131DC016D0EC291CD117E0F02903D0F82917D13B
S1131DD00E4817E00E4815E00E4813E00E4811E0D7
S1131DE00E480FE00E480DE00E480BE00E4809E0E7
S1131DF00E4807E00E4805E00E4803E00E4801E0F7
S1131E000D4800BF00BF00BD201C02400090D0035D
S1131E10006CDC020048E80100366E010024F40086
S1131E20001BB70000127A00808D5B0000093D00A2
S1131E30C0C62D0080841E0040420F0010B5044629
S1131E40204600F077FA002010BD000010B51821DC
S1131E501348FFF7A6FB124812490860124848606D
S1131E60012008810020887201220F490D4800F0EA
S1131E7021F900210B48FFF715FE20210B48FFF73D
S1131E8090FB0A480A4948600A4B01220A4908485B
S1131E9000F076F955210648FFF74AFE10BD000010
S1131EA05C06002094060020B4690000740600203B
S1131EB0A00600203D1E00009869000010B50A46E7
S1131EC01DE0016807231B03994207D30F23DB029C
S1131ED0994203D203685B1C036010E00B780A4C40
S1131EE0247863401B069B0D084CE358064C246879
S1131EF0240A6340044C236003685B1C036013469C
S1131F00521E002BDDD110BD54060020E4690000F0
S1131F1010B5014600200022087803024C782343C0
S1131F20184603028C78234318460302CC782343D3
S1131F30184643084340DB00840863401A46044BB8
S1131F405A40044B1A600123034C237010BD000057
S1131F50010200002C0600202806002010B50446CB
S1131F60002004F02DFA022841D1214800780028ED
S1131F7002D101201E4908701D48007801281FD194
S1131F801B484078401C1A49487021465A20FFF7E4
S1131F90D7FA17494978884229D80020144948704B
S1131FA008468078401C8870084680780A2803D345
S1131FB00020887002200870002004F041FA16E026
S1131FC00B480078022812D109484078401C08497F
S1131FD0487021467D20C000FFF7B2FA04494978D1
S1131FE0884204D800200249487004F029FA10BD40
S1131FF00000002000B587B000216846017104216B
S113200041710C480290411003910B4904910591D0
S11320100A480690FFF71AFF01A804F03DFA00F001
S113202065F900F00FF80021054802F083F807B0C5
S113203000BD0000FFFF1F00FFFFFF1F3D21000048
S11320400205000010B53F204001174948600020F8
S11320500872012008700020487201208872134819
S1132060FFF772FC10491148FFF798FC01210F4853
S1132070FFF7E8FC0E480C49486000200872012074
S11320800870002048720120887208481030FFF759
S11320905BFC054905481030FFF780FC012103482B
S11320A01030FFF7CFFC10BDB406002010550440DB
S11320B0DF070000F0B50B4614464360048100219D
S11320C036E0002216E02C254D4346687519AD5CB8
S11320D018274F430668F619B5542C254D43466816
S11320E07519AD5C18274F430668F6190836B554C0
S11320F0551CEAB2082AE6D3002518274F43066880
S1132100F619357418274F430668F619757418279D
S11321104F430668F619B57418274F430668F61935
S1132120F57418274F430668F61975614D1CA9B25A
S113213005898D42C5DC00258572F0BD70B5044665
S1132140606800F0C3FA0546E27A23460C33294658
S1132150094800F083FA09496068884203D0491CA1
S11321606068884206D1E17AA28890B222460C3295
S113217000F00EFD70BD000094060020DF07000093
S1132180FFB581B004460F460025002600200090CC
S11321902760039820810498E0600020207400BF29
S11321A09DE01C206843216808586A0161688850D2
S11321B01C2068432168081880686A0161688918CE
S11321C048601C2068432168081840686A016168F7
S11321D0891888601C20684321680818C0686A014F
S11321E061688918C8601C20684321680818007C4D
S11321F06A016168891808741C20684321680818FA
S1132200407C6A016168891848741C20684321680D
S11322100818807C6A016168891888831C206843D7
S113222021680818C07C6A016168891888740020D4
S11322306A0161688918C8741C20684321680818F9
S11322404068002813D01C20684321680818C07C0B
S1132250002805D1401E6A0161688918C8831AE004
S11322600020C0436A0161688918C88313E01C20F8
S1132270684321680818C07C002805D000206A0142
S113228061688918C88306E000206A0161688918BA
S1132290C88301200090002607E000216A016068DD
S11322A0801814308155701CC6B2690160684018EA
S11322B0808BB042F1DC1C20684321680818406917
S11322C000280AD06B016268D218104614301C230F
S11322D06B432268D21851698847681CC5B22089AB
S11322E0A84200DD5DE7009805B0F0BD00B585B0FB
S11322F0FD20C00001900021684601720170417206
S113230081720821C172002004E0002203A90A544A
S1132310411CC8B26946C97A8142F6DC0448FFF719
S113232013FB69460248FFF739FB05B000BD000006
S11323308055044030B585B00446002520680190DE
S1132340A1796846C17261794172002101720170FC
S113235000BF05E020460830415D03A841556D1CCF
S11323606846C07AA842F5D8FD21C9000198401AF0
S113237004D169460348FFF7E2FB00E000BF00BF59
S113238005B030BD8055044010B501246407FFF743
S1132390EBF90A4800680A4988420BD107484068AB
S11323A0002809D1032109032046FFF7FAF801F0B8
S11323B03DFE01E001F0FCFD10BD0000FC05002025
S11323C0A55A7AA710B500202D490870FFF7CCF95B
S11323D02C4844682C48844202D02C48844214D1AE
S11323E02948844203D101202549087002E00220D3
S11323F02349087001F026FE00F092F9002003F052
S1132400FBFE0A2000F065F935E02148844228D11A
S113241000F0BAF91F4880680121890488421DD25E
S11324201C4800680F21C902884217D11948416825
S11324300920800300F044F800280FD0FFF74EF97C
S113244000F076F9144A5168106800F039F8002851
S113245004D0002003F0D0FE03F03AFF01F0F2FDB7
S113246009E001F0EFFD00F05BF90A2000F031F91A
S113247001200A490870034840680949086010BDF2
S1132480F0050020FC050020A33A7AA7A88A7AA7C1
S1132490A55AA55A60180020541800204E060020A2
S11324A02006002070B504462546002D07D10020E3
S11324B003F0A2FE0A2000F00CF903F009FF70BD3E
S11324C0FEB504460F460F20C002844203D0092003
S11324D08003844237D1009707208003009F8742FE
S11324E02FD20020C043194908600120C002201ADD
S11324F0019026460EE03078761C1449097848404D
S11325000006800D1249085810490968090A484014
S11325100E4908600098411E00910028EBD10B4839
S11325200068C04309490860019800F059F9029015
S1132530064801680298814201D1012504E0002582
S113254002E0002500E000252846FEBD54060020D8
S1132550E469000070B5C0B000261D48008A1C491B
S1132560498A884205DB1A48008A1949498A401A6F
S113257084B2002C28D0FF2240216846FFF70AF8D5
S1132580002513E01248418A408A401C104A5082B8
S113259010461430405C694648551046408AFF286E
S11325A002DD002011464882681C85B2A542E9DBA1
S11325B0074922460868694603F02EFF064621466D
S11325C00348001DFFF77AFC304640B070BD0000A0
S11325D06C18002070B50125FFF7BCFF094800689E
S11325E0C043084908600720000300F0F9F80446D6
S11325F004480068A04201D1002501E0FFF7C0F8BB
S1132600284670BD5406002070B500250F24E4024E
S11326101022214620311048FEF7CEFF002819D1A0
S11326204022214630310C481030FEF7C5FF002807
S113263010D11022A11808481038FEF7BDFF002859
S113264008D11022214604482038FEF7B5FF00289F
S113265000D10125284670BD9C050020FFB581B03E
S113266004460F463D462089A8422DDD18206843C4
S113267021680818007C002826D1002609E0049867
S1132680815D182068432268101808308155701C39
S1132690C6B2082EF3D3012118206843226810180B
S11326A041742C20684361680818006A00280BD024
S11326B018236B432268D218104608302C236B432E
S11326C06268D218116A884705B0F0BD014601203E
S11326D07047002101E000BF491C8142FBD37047D1
S11326E010B500240C4A51681068FFF7E9FE002871
S11326F00FD0FEF7ADFF00F047F808484168092005
S11327008003FFF7DDFE002801D0012402E000244D
S113271000E00124204610BD541800206018002059
S1132720014802490860704700025000F805002083
S113273000B5134800F054F8124908601048001D11
S113274000F04EF80F494860084600680F21C9029E
S1132750884210D10B4840687121C902884202D9CD
S11327600020C04304E0074840680F21C902401814
S11327700449886003E00020C0430249886000BD2A
S1132780047000005418002000B5134800F028F825
S1132790124908601048001D00F022F80F494860F3
S11327A0084600680F21C902884210D10B484068CE
S11327B007218903884202D90020C04304E0074866
S11327C040680921890340180449886003E0002017
S11327D0C0430249886000BD04380200601800202C
S11327E010B504460023204600F059FE034618069F
S11327F0FF210902194009020843FF210904194075
S1132800090A0843190E08430346184610BD10B5BB
S113281000F0E8FD00F0D6F800F00EFB00F002F83E
S113282010BD000070B541480078912800D070BDFB
S113283000F0BEF8012876D13D4800883D49088063
S113284008468078F021884320303A498870084649
S11328508078000900013549097A0907090F0843FE
S1132860344988703148807A401E3049887208465D
S11328700089401C088108460089C988884216DA04
S113288008202C49887200240EE0284841882848F2
S1132890001D415C2748C01C015524484088401C49
S11328A022494880601CC4B2072CEEDB2DE01F488F
S11328B000891E49C98888421CD11C4800791B49DB
S11328C08978401AC5B2681C1A49887200240EE03F
S11328D0164841881648001D415C1648C01C015525
S11328E012484088401C11494880601CC4B2AC4264
S11328F0EEDB0AE000F002FD00200C4908700C49F0
S11329000888092100F0B8F991E7012000F0B8FC2B
S1132910084A917A1088921C00F070F905490888D9
S1132920002100F0C1F800BF81E70000860C002000
S1132930220C0020300700201B49097E002932D0D8
S11329401949897E0C225143174A515A174A11805A
S113295000200CE01449897E0C225143124A891844
S1132960891C0A5C1149891C0A54411CC8B20828F4
S1132970F0DB0D49897E0C2251430B4A8918897A70
S11329800A4A91720121D1720749097E491E064AF9
S113299011761146897E491C91761146897E022959
S11329A001DB002191767047FC06002024070020FB
S11329B00349487B012802D10021014A5173704721
S11329C0940C002010B533484068002861D1314888
S11329D0007B030003F026FC07590512212E3D4A13
S11329E059002D480078002807D000202A49087093
S11329F02A490888012100F03FF947E02648007879
S1132A00002809D000202449087025494A880888EC
S1132A100123091D00F040F938E01F480078002820
S1132A2007D000201C4908701C490888022100F0C6
S1132A3023F92BE018480078002809D00020164913
S1132A40087017494A8808880923091D00F024F9E9
S1132A501CE011480078002807D000200E490870B7
S1132A600E490888092100F007F90FE00A480078A8
S1132A70002809D000200849087009494A880888B4
S1132A800323091D00F008F900E000BF00BF00F0B7
S1132A9035FC10BD940C0020860C0020220C002074
S1132AA03C0700207047000070B504460D463448CA
S1132AB00088A04263D1002D61D1324800782228D9
S1132AC04ED004DC20283DD0212856D141E0902866
S1132AD002D0912851D115E02A48C08801280AD192
S1132AE000202849087000F009FC274908880021C3
S1132AF000F0C2F805E0032000F0C2FBA020214949
S1132B0008703BE01F4800891E49C98888420AD1E1
S1132B1000201C49087000F0F1FB1B4908880021C3
S1132B2000F0AAF80DE01748807A002806D000F0DB
S1132B30E5FB1449087B00F087FB02E0032000F06A
S1132B409FFB1BE0062000F09BFB11200D49087041
S1132B5014E0062000F094FB11200A4908700DE0EF
S1132B6000200849087000F0C9FB08494A88088811
S1132B700923091D00F090F800E000BF00BF70BDFC
S1132B8018070020860C0020220C00203C0700209F
S1132B9070B50346184C247E022C00DB70BD164C25
S1132BA0647E0C256C43144D2B5300200AE0155C05
S1132BB0114C647E0C2674430F4EA419A41C255496
S1132BC0441CE0B28842F2D30B4C647E0C2674435E
S1132BD0094EA419A1723446247E641C35462C7611
S1132BE02C46647E641C6C762C46647E022C01DBCD
S1132BF000246C7600BFD1E7FC060020F0B585B058
S1132C0007460D4616461A480780002406E0317828
S1132C101748801C0155761C601CC4B2AC42F6DB1C
S1132C202C4605E0AA211248801C0155601CC4B240
S1132C30082CF7DB0E480088019008216846C17211
S1132C400021417201720170002406E00848801CD2
S1132C50015D03A80155601CC4B2082CF6DB69466B
S1132C600448FEF76CFF01200149887205B0F0BDED
S1132C70180700209055044070B504460D462946B7
S1132C80204601F0B7FD70BD70B504460D462946D7
S1132C90204601F0BDFD70BDF8B504460D4616464C
S1132CA01F463B4632462946204601F0B2FDF8BD98
S1132CB0F8B507460E4615465C480078002804D04F
S1132CC009213846FFF7D8FFF8BD002D01D0602D4B
S1132CD004DD09213846FFF7CFFFF5E754480780A4
S1132CE04580002406E031785148001D0155761CCA
S1132CF0601CC4B2AC42F6DB00204C494870084664
S1132D008580FF2088727F20087308468088082801
S1132D102EDA0120C8800846808848800120088176
S1132D20434800884349088008468078F021884356
S1132D304049887008468078000900013B490979B8
S1132D400907090F08433B49887038480079401C3B
S1132D508872002407E03648001D015D3548C01C18
S1132D600155601CC4B231488088A042F3DC4AE0BB
S1132D700721681CFEF7FAFB002907D00721284623
S1132D800830FEF7F3FB2949C88005E00721681CD9
S1132D90FEF7ECFB2549C880062024494880012021
S1132DA00881234800882349088008468078F02158
S1132DB0884310301F498870084680780009000154
S1132DC01A4989880905090F08431A498870084671
S1132DD04088FF2109028843144989880902FF2297
S1132DE012021140084313494880082088720024C5
S1132DF007E00F48001D015D0E48001D0155601CD1
S1132E00C4B2062CF5DB012000F03AFA094A917AA3
S1132E101088921CFFF7F2FE9020044908700549BF
S1132E2008880021FFF740FE00BF4DE7860C002014
S1132E30220C00203007002010B5FFF77DFD144858
S1132E40C07A002822D0124880780009002806D0D1
S1132E50012807D002280AD0032810D10CE000F082
S1132E609BF90FE000F09EF800F056FA0AE000F03B
S1132E7011F800F051FA05E000F0FEF802E0FFF767
S1132E8011FE00BF00BF00200149C87210BD000040
S1132E902407002010B540480078112800D010BD48
S1132EA03E4800883F214901884200D0F7E73B486B
S1132EB080780007000F3849097A0907090F88420A
S1132EC00CD000203449087000F018FA34494A88BC
S1132ED008880423091DFFF7DFFEE0E72E48008978
S1132EE0401C2D4908810846807A401E8872084695
S1132EF00089C98888421BDA2848807A082800D0CB
S1132F00CDE700240EE02548C01C015D224842881C
S1132F102348001D815420484088401C1E49488095
S1132F20601CC4B2072CEEDB062000F0A9F930E0E7
S1132F301948808818494988401A1849897A88426A
S1132F4003DA1648807A082800D0A8E700240EE0A7
S1132F501248C01C015D104842881148001D81546C
S1132F60601CC4B20C484088401C0B4948800A4885
S1132F704088094989888842EADB002006490870AC
S1132F8000F0BCF906494A8808880023091DFFF7A8
S1132F9083FE00BF83E70000860C00202407002086
S1132FA03C07002070B53148007880210840802813
S1132FB000D170BD2E4800883F214901884200D0CD
S1132FC0F7E72B48807A082800D0F2E72848807871
S1132FD005072D0F2D0226484088000A0543082DB9
S1132FE000DAE6E7012021494870062048800846B7
S1132FF085800120088100208872C8728988481C55
S11330000721FEF7B3FA002909D018498988084630
S113301008300721FEF7AAFA1449C88007E01349CB
S11330208988481C0721FEF7A1FA1049C880104876
S113303000881049088008464580002407E00C48B1
S1133040001D015D0B48001D0155601CC4B2062C17
S1133050F5DB042000F014F9102004490870054A37
S113306051881088FFF710FE00BFA2E7860C0020ED
S1133070240700203C07002010B544480078A0280D
S113308008D042480078912804D040480078A1280C
S113309000D010BD3E4800883F21490188420AD033
S11330A03C4908880921FFF7E7FD00F027F90020D3
S11330B036490870EDE73648807A08280AD0354941
S11330C008880921FFF7D8FD00F018F900202F49DE
S11330D00870DEE72E4880780007000F002804D02F
S11330E0012825D0022843D12EE028484078002822
S11330F000D048E02648C078002803D101202349A5
S1133100487003E02248C078204988721F4800783C
S1133110912803D01E4800791C49087391201B494B
S1133120087000F0EBF81949087B00F08DF82AE0EC
S113313016484078002800D025E0A12013490870E3
S1133140032000F09DF81EE010484078002800D0CD
S113315019E00E480078A02809D10E4908880821F2
S1133160FFF78AFD00F0CAF80020084908700AE059
S1133170084908880521FFF77FFD00F0BFF800200B
S11331800249087000BF00BF00BF82E7860C002020
S113319024070020220C002010B528480078802144
S11331A00840802800D110BD24480078002806D0AB
S11331B0234800883F214901884200D0F3E7204892
S11331C0807A1F4989780907090F884203DD1C4862
S11331D0807A082800D0E6E7194880780007000FB5
S11331E0002805D0164880780007000F072800DD66
S11331F0D9E71348008813490880114880780007EC
S1133200000F4880002407E00D48C01C015D0D48F4
S1133210001D0155601CC4B20A484088A042F3DC7A
S113322000200649087000F069F806494A880888B1
S11332300023091DFFF730FD00BFB4E7860C002012
S1133240240700203C0700207F2805DC7D21C900DD
S11332504143094A91600BE0F12806DBF92804DCBC
S113326064214143044A916002E00449024A9160A6
S11332700221014A51737047940C002018F0010098
S113328000B5030002F0CEFF0729050B11171D231B
S113329029000121144A11731449516022E00221CA
S11332A0114A1173114951601CE003210E4A117334
S11332B00F49516016E004210B4A11730D49516006
S11332C010E00521084A1173002151600AE006212B
S11332D0054A11730849516004E00021024A117340
S11332E0516000BF00BF00BD940C0020A861000025
S11332F0F824010028230000F049020000200149BD
S113330008737047940C0020024909880918014A7F
S113331011807047940C002010B52E4800781028B6
S113332019D12D4840882D4988420ADD2C488078DF
S113333000090001801C2A49887022202549087050
S113334025E027488078000900012549887020205D
S1133350204908701BE01F480078112816D11D4829
S1133360807A002800D010BD1A484078002800D088
S1133370F9E700201749887219488078000900018C
S11333801749887020201349087000E0EBE7FD20FE
S1133390C0001349088008468078F0218843303003
S11333A00F49887000210E48C17002210171032069
S11333B00B4988720220FFF763FF094A917A10884B
S11333C0921CFFF71BFC064908880021FFF76CFBE1
S11333D000BFC8E7860C00203C070020E204000080
S11333E030070020244A118852888A4242D0224A57
S11333F052888A4204DA204A52888A1A90B207E034
S11334001D4A52880023DB439A1A521C521890B268
S1133410194A5180127B002A10D0174A5268002A98
S11334200CD0154A5268824205D9134A5268121ABE
S1133430114B5A6002E000220F4B5A600E4A527B35
S1133440022A17D10C4A9268002A0CD00A4A9268C0
S1133450824205D9084A9268121A074B9A6002E020
S11334600022054B9A60044A9268002A02D1012284
S1133470014B5A7370470000940C002070B5054648
S11334800E46FEF77DF92C4605E0204600F00AF8CA
S1133490FF34FF340234B442F7D3002070BD014638
S11334A008687047014610200D4AD060F120106270
S11334B055205060AA2090600020C043086000BFDF
S11334C007480068C007C00F0028F9D00448006806
S11334D001221043024A10600020D060106270473D
S11334E0000002400246F1200B4B1862AA205860EB
S11334F055209860116000BF07480068C007C00FDE
S11335000028F9D00448006801231843024B1860CE
S1133510002018627047000000000240F8B5002344
S1133520002500950024002200BF94E001259D4061
S1133530ACB20D8825400095009DA5426FD11A4676
S11335408D79012D0DD1464D03263602AD192D5C22
S1133550012696403543424E03273F02F61935545F
S11335600CE03F4D03263602AD192D5C0126964032
S1133570B5433B4E03273F02F6193554CD78002D51
S11335804ED1374D60352D5CCE78002E01D1012609
S113359000E000269640B543314E603635548D78B0
S11335A0002D2ED12E4D19267601AD192D5C8E7865
S11335B0002E01D1012600E000269640B543284E96
S11335C019277F01F61935540D79002D0ED1244D9C
S11335D050352D5C0E79002E01D1012600E0002625
S11335E09640B5431E4E5036355423E01C4D50359D
S11335F02D5C0E7996403543EEB2194D50352E545C
S113360018E0174D19267601AD192D5C8E78964079
S11336103543134E19277F01F61935540AE018E093
S11336200F4D60352D5CCE7896403543EEB20C4D8F
S113363060352E544D79012D0AD1094D30352D5C5C
S1133640012696403543EEB2054D30352E5400E048
S113365000BF5D1CABB2082B00DA67E7F8BD0000C1
S113366000000440FFB5074615461E4600243846B0
S1133670019900F01FF8002802D0012004B0F0BD29
S113368000240CE00A2060430949085CB04204D1DC
S11336902946204600F05EF807E0601C84B20A2048
S11336A060430349085C0028ECD100BF0020E5E733
S11336B0300000200246002A03D1402901DD012008
S11336C07047032A03D1022901DD0120F8E7042A07
S11336D003D1202901DD0120F2E7052A03D12029A5
S11336E001DD0120ECE70C2A03D1102901DD0120C2
S11336F0E6E70D2A05D1012903DD402901DA01207D
S1133700DEE70E2A03D1202901D10120D8E70020C9
S1133710D6E7000010B5064A03231B02D218125C38
S11337208A43034B032424021B191A5410BD0000BE
S11337300000044010B5064A03231B02D218125C91
S11337400A43034B032424021B191A5410BD00001E
S11337500000044070B502460020B1E00A23534340
S11337605A4C1B195B1C440004191B199B788B428F
S11337707DD10A235343554C1B195B1C4400041987
S11337801B195B78082B33D10A2353434F4C1B1965
S11337905B1C440004191B574D4C4E4D6419E35CEB
S11337A0012423430A245443484D6419641C4500EE
S11337B045196457464D474EAD192B550A235343BB
S11337C0424C1B195B1C440004191B57404C3546E2
S11337D06419E35C022423430A2454433B4D6419D3
S11337E0641C450045196457394DAD192B5564E0E7
S11337F00A235343354C1B195B1C440004191B1941
S11338005B78092B34D10A235343304C1B195B1CBE
S1133810440004191B572E4C2E4D6419E35C4024BC
S113382023430A245443294D6419641C4500451953
S11338306457274D274EAD192B550A235343234C68
S11338401B195B1C440004191B57214C3546641991
S1133850E35C8024A3430A2454431C4D6419641C70
S11338604500451964571A4DAD192B5525E025E03F
S11338700A235343154C1B195B1C440004191B57A2
S1133880134C144D6419E35C0A2454430F4D64191A
S1133890641C45004519641965780124AC40234330
S11338A0DCB20A235343094D5B195B1C45004519DF
S11338B05B57074D074EAD19EC5404E0431CD8B2D6
S11338C0032800DA4AE700BF70BD00003000002082
S11338D0000004407508000070B505460024032D5F
S11338E000D170BD002D01D0012D17D181210320FD
S11338F0800200F0CFFB8021114800F0CBFB0024B4
S113390009E0A2000F4BD2189178A200985A00F057
S1133910C1FB601CC4B23B2CF3DB0FE0022D0DD1C4
S1133920002409E0A200084BD2189178A200985A0A
S113393000F0B0FB601CC4B23B2CF3DB00BFD0E74B
S113394002060000C0670000AC68000010B50C4817
S11339500078002803D00B4A5068916888470848CB
S11339604078002803D0084A506891688847044882
S11339708078002803D0054A50689168884710BDB4
S1133980006000408001002000030020800400202B
S113399010B508480079002803D0074A1069516916
S11339A0884704484079002803D0044A5068916845
S11339B0884710BD00600040800100200C030020F7
S11339C010B50848007A002803D0074AD069116A64
S11339D088470448407A002803D0044A5068916814
S11339E0884710BD006000408001002018030020BB
S11339F010B50848007B002803D0074A906AD16AB2
S1133A0088470448407B002803D0044A50689168E2
S1133A10884710BD0060004080010020240300207E
S1133A2010B50848007C002803D0074A506B916BFE
S1133A3088470448407C002803D0044A50689168B1
S1133A40884710BD00600040800100203003002042
S1133A5010B50848007D002803D0074A106C516C4B
S1133A6088470448407D002803D0044A5068916880
S1133A70884710BD00600040800100203C03002006
S1133A8010B50848007E002803D0074AD06C116D99
S1133A9088470448407E002803D0044A506891684F
S1133AA0884710BD006000408001002048030020CA
S1133AB010B50848407F002803D0074A5068916831
S1133AC088470448007F002803D0044A906DD16DD4
S1133AD0884710BD0060004054030020800100208E
S1133AE010B508484078002803D0074A5068916808
S1133AF0884704480078002803D0044A506E916E29
S1133B00884710BD20600040600300208001002031
S1133B1010B509480079002803D0084A106F516F86
S1133B2088470548001D4078002803D0044A50689F
S1133B309168884710BD000020600040800100208B
S1133B406C03002010B5034AD06F7832916888471F
S1133B5010BD00008001002010B5024A5068916831
S1133B60884710BD0402002010B50948007C0028D5
S1133B7003D0084A50689168884705481030407857
S1133B80002803D0044A50689168884710BD00009B
S1133B9020600040100200209003002010B5024A6B
S1133BA050689168884710BD1C02002010B5024A75
S1133BB050689168884710BD2802002010B5094854
S1133BC0007F002803D0084A506891688847054858
S1133BD01C304078002803D0044A50689168884714
S1133BE010BD00002060004034020020B403002017
S1133BF010B50C480078002803D00B4A506891682F
S1133C00884708484078002803D0084A50689168DB
S1133C10884704488078002803D0054A5068916892
S1133C20884710BD4060004040020020C0030020CF
S1133C304005002010B50D480079002803D00C4A37
S1133C405068916888470948001D4078002803D0CF
S1133C50084A5068916888470448001D8078002805
S1133C6003D0054A50689168884710BD4060004001
S1133C704C020020CC0300204C05002010B50D4858
S1133C80007A002803D00C4A506891688847094894
S1133C9008304078002803D0084A50689168884763
S1133CA0044808308078002803D0054A5068916899
S1133CB0884710BD4060004058020020D80300200F
S1133CC05805002010B50D48007B002803D00C4A8D
S1133CD050689168884709480C304078002803D020
S1133CE0084A50689168884704480C308078002856
S1133CF003D0054A50689168884710BD4060004071
S1133D0064020020E40300206405002010B50D487F
S1133D10007C002803D00C4A506891688847094801
S1133D2010304078002803D0084A506891688847CA
S1133D30044810308078002803D0054A5068916800
S1133D40884710BD4060004070020020F00300204E
S1133D507005002010B5024A50689168884710BD6C
S1133D607C02002010B50948007E002803D0084AD0
S1133D70506891688847054818304078002803D077
S1133D80044A50689168884710BD000040600040B4
S1133D90880200200804002010B50948007F00288C
S1133DA003D0084A50689168884705481C30407819
S1133DB0002803D0044A50689168884710BD000069
S1133DC040600040940200201404002010B508480C
S1133DD00078002803D0074A50689168884704484F
S1133DE04078002803D0044A50689168884710BD81
S1133DF060600040A00200202004002010B50948A3
S1133E000079002803D0084A50689168884705481B
S1133E10001D4078002803D0044A50689168884700
S1133E2010BD000060600040AC0200202C040020A3
S1133E3010B50948007A002803D0084A50689168F0
S1133E408847054808304078002803D0044A506861
S1133E509168884710BD000060600040B8020020EF
S1133E603804002010B5024A50689168884710BD94
S1133E70C402002010B5024A50689168884710BDFA
S1133E80D002002010B50948007D002803D0084A5C
S1133E90506891688847054814304078002803D05A
S1133EA0044A50689168884710BD00006060004073
S1133EB0DC0200205C04002010B50948007E0028C4
S1133EC003D0084A506891688847054818304078FC
S1133ED0002803D0044A50689168884710BD000048
S1133EE060600040E80200206804002010B5094822
S1133EF0007F002803D0084A506891688847054825
S1133F001C304078002803D0044A506891688847E0
S1133F1010BD000060600040F40200207404002022
S1133F20F8B504460D4600260C2060431D49085C84
S1133F30002801D00120F8BD0C2060431949401825
S1133F4085600C20604340188068002801D101205E
S1133F50F1E701210C206043124A1154002220464B
S1133F60E317DB0E1B185B115B01E31A9B000E4F7A
S1133F70DB19E717FF0E3F197F11DA5502F060F9DC
S1133F8000222046E317DB0E1B185B115B01E31ACA
S1133F909F00064BFB18E717FF0E3F197F11DA55F8
S1133FA03046C8E780010020006000400061004006
S1133FB0FEF72AFB01281BD107200003FFF76FFA45
S1133FC0401C002803D10D4802F016F913E0FEF757
S1133FD0AFFB0B4A51681068FEF772FA012803D14F
S1133FE0002002F009F906E0044802F005F902E0B5
S1133FF0024802F001F902F06BF90000A55AA55A33
S11340005418002000BFFEE705480078022806D1B6
S113401004480068002802D1012003490870704751
S11340204E060020200600201C06002010B572B6A3
S11340300121C903086880F3088800BF48688047E5
S113404010BD0000022006490870002005490860E0
S11340508860C86004498873C87308747047000096
S11340604E0600206C1800206C1D002010B50123A2
S11340701A4600211846FDF7A1FD012211461046FB
S1134080FDF702FEFDF7EEFD014802F08BF910BDCD
S11340900090D003FEB505460C460020C0430290B4
S11340A0EFB22804060E0F2E42DA082F40DA012060
S11340B0B8406946088080202040002816D101209D
S11340C08870A007800F022801D1487109E0A00779
S11340D0800F012802D16946487102E00020694638
S11340E04871F0B26946FFF719FA1FE000206946EB
S11340F088700E202040002800D000BF10202040EF
S1134100002802D16946087102E00120694608715D
S1134110E007C00F002802D16946887102E001203F
S113412069468871F0B26946FFF7F8F900200290F9
S11341300298FEBDF8B504460F460020C043009027
S1134140E6B22004050E0F2D11DA082E0FDA012035
S1134150B04086B2002F04D1E8B23146FFF7DAFA54
S113416003E0E8B23146FFF7E5FA0020009000983A
S1134170F8BD000070B504460D46601E0D49884226
S113418000D90124002C00D1012440200A490870E0
S1134190084600786043094948610321081F02F07A
S11341A05BF8002005498861072008610448056020
S11341B070BD0000FFFFFF000800002000E000E0E9
S11341C0040000200020C043002809DBC206D20EF0
S11341D001219140054A1160BFF34F8FBFF36F8FE8
S11341E000BF0020024908618861704780E100E057
S11341F000E000E01A20084908722B2048723C2095
S113420088724D20C8727F20044909680860AC2078
S11342100349487070470000000402400C0000206D
S113422000100240F0B5054600262846FFF737F98E
S11342300346DCB2FF2000021840070A002323468D
S11342401802384303461E463046F0BD10B51548E3
S1134250007801280DD114480078401C12490870D8
S113426008460078642804DB0020087001200F4908
S113427008700F480078012813D10E4800780128EF
S113428004D100200B4908700B4908700A480078D3
S1134290401C0949087008460078322801DD02F004
S11342A017F810BD2606002025060020240600204D
S11342B01C0600201E0600201D06002010B586B036
S11342C00446FD20C000029008216846C173002105
S11342D0417301730171032101747F2101A84173AA
S11342E084737821C173AA21017441748174C174E7
S11342F001A90248FDF723FC06B010BD8055044017
S11343000EB500200190029002216846017100213F
S11343104171322181710121C171F421017201A81D
S11343200523FD22D20000210090102001F0FCFEA4
S11343300EBD000010B50146012904D0022921D088
S1134340032970D145E00022494B1A70494B1A7079
S1134350494B1A70494B1A70494B1A70494B1A60F1
S1134360494B1A609A60DA60484B9A730023474AB3
S1134370D3730022454B1A74521E454B1A60454BA9
S11343801A6073E000223B4B1A7001223A4B1A70F8
S113439000223A4B1A703A4B1A703A4B1A603A4B55
S11343A01A609A60DA600023384A9373D3731374E3
S11343B0002005E00022354B1A3B1A54421C90B2EF
S11343C02828F7D30022D243314B1A60314B1A60AC
S11343D04CE00022274B1A700122274B1A7000224E
S11343E0264B1A70264B1A70264B1A60264B1A60FD
S11343F09A60DA60254B9A730023244AD3735A1EB9
S1134400234B1A60234B1A600022204B1A7400209D
S113441005E000221D4B1A3B1A54421C90B2282876
S1134420F7D323E0FFE70022114B1A70114B1A70E7
S1134430114B1A70114B1A70114B1A70114B1A60F0
S1134440114B1A609A60DA600023104A93730022B9
S11344500E4BDA731A74002005E000220B4B1A3B52
S11344601A54421C90B22828F7D300BF00BF10BDD5
S11344701C0600201D0600201E0600202706002022
S1134480280600202C0600206C1800206C1D00203B
S1134490500600205406002010B505480068002886
S11344A002D003480068804700F011F810BD0000F6
S11344B00400002010B5FFF7C9FE10BD10B50A2096
S11344C0FDF74CFD10BD704770477047704710B53D
S11344D03220FEF719FF10BD0CB500BF0548006877
S11344E00090044800680190019900988842F5D131
S11344F000980CBD2000002010B5FEF788F900F0EC
S113450083FA10BD70B53148006831490968401814
S11345102E490860084600687D21C900884211D3ED
S11345202A480068FDF70CF806467D21C900274893
S11345300068FDF705F825480160264800688019E1
S113454024490860244840682149096840182249E0
S1134550486008460068002837D10025084684686A
S11345602EE02068002829D01B4960684968002291
S1134570D243511A884205D21749606849684018E5
S1134580606002E00020C0436060A1686068884207
S113459014D3206801280AD100202060002D03D103
S11345A00D492069886004E02069286101E0002049
S11345B06060E068002801D0E068804725462469EF
S11345C0002CCED100200449486070BD1C0000209E
S11345D01800002020000020E406002010B5FFF79A
S11345E0F1FD322000F008F802493220FFF7C2FD45
S11345F010BD00000545000010B504460D480460D8
S113460000200D4908600D4908600D4908604860A4
S11346108860FFF761FF0B490860002048608860EC
S11346200120C860032008610520486107208861D3
S113463010BD0000180000201C00002020000020F5
S1134640E4060020C806002070B5FFF755FFFFF709
S113465043FF05463A480068A84203D83848006832
S11346602C1A06E0364800680021C943081A40198C
S1134670441C3348056040680019314948600846C5
S11346804068022806D308460079C007C00F486076
S1134690FFF71AFF2A4880680019294988600846EC
S11346A08068052807D388680521FCF749FF24485A
S11346B08160FFF70BFF2248C06800192049C860D9
S11346C00846C0680A2807D3C8680A21FCF738FFDF
S11346D01B48C160FFF7F2FE194800690019184928
S11346E0086108460069142807D308691421FCF7F7
S11346F027FF13480161FFF7E6FE114840690019DE
S11347000F49486108464069322807D34869322175
S1134710FCF716FF0A484161FFF7D7FE0848806995
S113472000190749886108468069642807D38869A5
S11347306421FCF705FF02488161FFF7BBFE70BDF1
S1134740C806002010B5FFF791FCFFF753FD0020C9
S1134750FFF7C2F8FFF742FFFDF74CFC10BD000065
S113476010B580201B4948711A201A492039087253
S11347702B2048723C2088724D20C87200201649B4
S11347804860FDF7B1FA154908600020C043144998
S11347900860144908601448144908601149032248
S11347A01202891848600F49891888600D498918D0
S11347B0C8600C49891808610A498918486109497F
S11347C08918886107498918C861AC20084948706C
S11347D010BD00002004024000B001405806002033
S11347E080E200E000E100E0C0C0C0C000E400E0FE
S11347F00010024000B503460A46002A03D11846B9
S113480000F0DAF803E00121184600F0D5F800BD05
S11348107047F0B505460E4617461C46002C05D1D8
S11348203A463146284600F0C9F805E001233A46E5
S11348303146284600F0C2F8F0BD70B504460D4676
S11348401646324629462046FEF732FA70BD00006D
S113485008B554488079002872D000205249087065
S11348605248807831283ED00CDC222820D004DC49
S1134870102814D0112877D163E0272821D02828C4
S113488072D127E0372849D004DC342834D03628C4
S11348906AD13AE03E285DD0852865D147E0414A97
S11348A0203A918C414A1088D21C00F0B1F86FE094
S11348B03C4A203A918C3D4A1088D21C00F034FACC
S11348C066E0384A203A918C384A1088D21C00F0AD
S11348D041FB5DE0334A203A918C344A1088D21C63
S11348E000F0ACFC54E02F4A203A918C2F4A1088F7
S11348F0D21C00F09BFD4BE02A4A203A918C2B4AB3
S11349001088D21C01F044F842E0264A203A918CE7
S1134910264A1088D21C01F09BF939E0214A203A3A
S1134920918C224A1088D21C01F094FA30E01D4A7E
S1134930203A918C1D4A1088D21C01F053FB27E0C9
S11349402FE0184A203A918C184A1088D21C00F0A3
S11349505DF91DE0134A203A918C144A1088D21C48
S113496001F0DCFA14E0FFE7104800883F21490118
S113497088420CD111200E494870481C0B49009004
S113498088780123FD22D200194601F0CDFB00BF37
S113499000BF01200749087003490870002001493D
S11349A0887108BD841100201C060020A40C00207E
S11349B0F20500201E06002070470000F0B50446F2
S11349C0002B12D10125094EB571094D2C80551EBD
S11349D0203EB584002006E00E78054DAD1C2E5413
S11349E0491C451CA8B29042F6DBF0BD841100209E
S11349F0A40C002070B504460D46164632462946DE
S1134A002046FFF71AFF70BD10B5FFF721FF10BD58
S1134A10F7B582B00020764948700398C6B20120E9
S1134A2074490870029C002505E00498405D7249B1
S1134A304855681C85B2B542F7DB012E11DA6F4880
S1134A40844201D105B0F0BD132069494870481C67
S1134A500123FD22D20019460090102001F064FBCE
S1134A60F0E76548007847067F0E012F14D0022F27
S1134A7012D0032F10D06148844200D1E2E7122003
S1134A805B494870481C0123FD22D200194600905E
S1134A90102001F049FBD5E7012E10D0574884427D
S1134AA000D1CFE7132052494870481C0123FD224E
S1134AB0D20019460090102001F036FBC2E7012E07
S1134AC04DD14D480078012803D04B480078812807
S1134AD00AD100204A49087001204A490870084652
S1134AE00078FFF727FC4BE043480078022803D006
S1134AF04148007882280CD101203E490870404981
S1134B00087002203F49087008460078FFF712FC3D
S1134B1036E039480078032803D0374800788328E2
S1134B200CD10120334908703549087003203549F8
S1134B30087008460078FFF7FDFB21E02F48844207
S1134B4000D17FE712202A494870481C0123FD2226
S1134B50D20019460090102001F0E6FA72E72748C7
S1134B60844200D16EE7132021494870481C012378
S1134B70FD22D20019460090102001F0D5FA61E719
S1134B801D480078032803D01B480078012816D15B
S1134B90002019494870322088700120C870F42020
S1134BA0087108460523FD22D20000210090102040
S1134BB001F0BAFA14480068FDF774FC15E00E48D9
S1134BC00078022811D100200B49487032208870E7
S1134BD00120C870F420087108460523FD22D20084
S1134BE000210090102001F09FFA00BF2AE7000086
S1134BF0F20500201E06002054130020DF070000E9
S1134C001C0600204E06002020060020FEB50E469D
S1134C101746F5B200203F490870002404E0385DCF
S1134C203D490855601C84B2AC42F8DB012D0CDA16
S1134C3013203A494870481C0123FD22D20019462A
S1134C400090112001F070FAFEBD33480078400650
S1134C50400E0190019801280CD012202F49487071
S1134C60481C0123FD22D20019460090112001F0B6
S1134C705BFAE9E7012D0CD0132028494870481C41
S1134C800123FD22D20019460090112001F04CFAB4
S1134C90DAE72348007801280CD122201F49487004
S1134CA0481C0123FD22D20019460090112001F076
S1134CB03BFAC9E718480078012803D01648007861
S1134CC0812819D114480078812804D1012014497D
S1134CD0087001F0FDFA10480123FD22D2000021E2
S1134CE00090112001F020FA01200D4908700D48B0
S1134CF0FDF7EFFC01F0ECFA122008494870481C5B
S1134D000123FD22D20019460090112001F00CFA73
S1134D1000BF99E71D06002054130020F20500206F
S1134D204E06002070170000F7B584B005460F4604
S1134D30002002900295FEB27E4908707E494870B8
S1134D407E48029D854201D107B0F0BD002405E0F4
S1134D500698005D7A490855601C84B2B442F7DBBA
S1134D60022E0CDA132074494870481C0123FD22DA
S1134D70D20019460090222001F0D6F9E4E77048E9
S1134D80007800026E49497808430390022E0CD043
S1134D90132069494870481C0123FD22D20019469A
S1134DA00090222001F0C0F9CEE7664A0398811AE8
S1134DB0904254D00ADC64494018002866D0042884
S1134DC07ED06249401800287BD131E00C2918D0EC
S1134DD00E29F9D1002408E05D4800681D30015D0A
S1134DE0574AA01C1154601C84B2062CF4DB5448AE
S1134DF00823FD22D20000210090222001F094F922
S1134E0094E0002408E0524800681730015D4C4AE1
S1134E10A01C1154601C84B2062CF4DB48480823FF
S1134E20FD22D20000210090222001F07DF97DE0D6
S1134E30002408E046480068001D015D404AA01CAB
S1134E401154601C84B2062CF4DB3D480823FD2277
S1134E50D20000210090222001F066F966E00024CF
S1134E6008E03B4800680A30015D354AA01C115433
S1134E70601C84B20D2CF4DB31480F23FD22D200D8
S1134E8000210090222001F04FF94FE010202C491E
S1134E90087024204870422088705F20C870562013
S1134EA00871312048712E2088713020C871087231
S1134EB008460923FD22D20000210090222001E0AF
S1134EC003E021E001F030F930E010201C490870C3
S1134ED028204870322088703020C8703220087131
S1134EE034204871302088713520C871312008720F
S1134EF03320487208460A23FD22D2000021009084
S1134F00222001F011F911E00C490298884200D1E5
S1134F101AE7312008494870481C0123FD22D200B9
S1134F2019460090222001F0FFF800BF00BF00BF27
S1134F300AE700001D060020F2050020DF0700003C
S1134F405413002087F10000DCEFFFFFA41EFFFFD5
S1134F50F8050020F7B584B000270020A8490870A0
S1134F60A8490498884201D107B0F0BD0598C5B29C
S1134F70002405E00698005DA3490855601C84B22E
S1134F80AC42F7DBA148007801280CDC7F20A04963
S1134F904870481C0123FD22D200194600902720A6
S1134FA001F0C2F8E0E7012D0CDA132098494870AB
S1134FB0481C0123FD22D20019460090272001F04D
S1134FC0B3F8D1E79048007847067F0E092F0ED03A
S1134FD00A2F0CD012208E494870481C0123FD2250
S1134FE0D20019460090272001F09EF8BCE70A2F52
S1134FF010D18848007801280CD0242084494870B6
S1135000481C0123FD22D20019460090272001F0FC
S11350108BF8A9E780480078012816D17F480078EA
S1135020012805D100207D4908707B4908700CE0F7
S1135030372077494870481C0123FD22D2001946C5
S11350400090272001F070F88EE76F480078092857
S113505002D00A287ED15EE0012D0CD013206C49C9
S11350604870481C0123FD22D200194600902720D5
S113507001F05AF8C0E001206649087068480078D9
S113508000280BD16748008886B230126649088030
S1135090F0B26649088001206149087009205A4924
S11350A0087061480078C043313048705F48007828
S11350B0C043233088705C4800785630C8705A4822
S11350C00078713008715A480078022806D1092006
S11350D00870002048708870C87008714A48417888
S11350E06846017248488178684641724648C178EA
S11350F068468172444801796846C1724248052372
S1135100FD22D20000210090272001F00DF802A812
S1135110FCF7FEFE70E0052D0CD013203C494870CE
S1135120481C0123FD22D20019460090272000F0DC
S1135130FBFF19E7344840780006334989780904AD
S113514008433149C978090208432F4909790843BA
S1135150039000E043E0374903980968884217D177
S11351602F480078012813D102203149087001200A
S11351702B490870244800780A282FD1224801239B
S1135180FD22D20000210090272000F0CDFF25E071
S113519000202349087028480078401C26490870DC
S11351A00846807803280CDB362019494870481CCF
S11351B00123FD22D20019460090272000F0B4FFFD
S11351C0D2E6352012494870481C0123FD22D20042
S11351D019460090272000F0A7FFC5E60CE0122036
S11351E00B494870481C0123FD22D2001946009047
S11351F0272000F099FF00BF00BF00BFB4E6000005
S11352001D060020DF070000541300204E06002076
S1135210F205002034060020260600202406002083
S1135220280600203C06002030060020320600201C
S1135230270600202C06002036180020F7B582B07F
S11352400398C7B2029C002073490870002605E049
S11352500498805D71498855701C86B2BE42F7DBA4
S1135260022F11DA6E48844201D105B0F0BD13203B
S11352706C494870481C0123FD22D2001946009055
S1135280282000F051FFF0E76448007845066D0ED1
S1135290002D16D0012D14D0022D12D0032D10D0C4
S11352A05F48844200D1E0E712205E494870481C00
S11352B00123FD22D20019460090282000F034FF7B
S11352C0D3E759480078012810D15548844200D1C9
S11352D0CBE7222053494870481C0123FD22D20009
S11352E019460090282000F01FFFBEE7022F10D0BF
S11352F04B48844200D1B8E713204A494870481CFF
S11353000123FD22D20019460090282000F00CFF52
S1135310ABE742484078032810DD4148844200D17D
S1135320A3E731203F494870481C0123FD22D200E5
S113533019460090282000F0F7FE96E737480078D9
S1135340802810D008DC00280ED001281DD00228A7
S11353502CD003284BD13AE0812815D0822824D0C0
S1135360832844D132E000BF2C48007880210840D3
S1135370002808D129480123FD22D20000210090F1
S1135380282000F0D1FE44E000BF244800788021AA
S11353900840002808D121480123FD22D200002121
S11353A00090282000F0C0FE33E000BF1B480078C6
S11353B080210840002808D118480123FD22D2008A
S11353C000210090282000F0AFFE22E000BF134827
S11353D0007880210840002808D110480123FD22CC
S11353E0D20000210090282000F09EFE11E00C491C
S11353F00298884200D138E712200A494870481CB4
S11354000123FD22D20019460090282000F08CFED2
S113541000BF00BF00BF28E71D0600205413002072
S1135420DF070000F20500204E060020F7B588B023
S11354300020FA490870FA490898884201D10BB053
S1135440F0BD0998C6B2002405E00A98005DF5494C
S11354500855601C84B2B442F7DBF3480078012895
S11354600CD17F20F1494870481C0123FD22D20051
S113547019460090312000F057FEE0E7E9484078F3
S11354800002E849897808430390E6480078012837
S113549003D0E4480078812879D10398FF38FF3895
S11354A00438002806D0E2494018002870D00128AA
S11354B06FD1F1E1DC48007802280CD07F20DB4971
S11354C04870481C0123FD22D20019460090312067
S11354D000F02AFEB3E7D348C0780006D149097921
S11354E009040843CF49497909020843CD49897918
S11354F008430290CF48807B00285BD1CE480068E7
S1135500C043CD49086002980968884242D1CB481B
S113551000783E2813D10020C043C7490860012009
S1135520C44988730020BF49C87008460423FD227B
S1135530D20000210090312000F0F6FD77E0BF4852
S113554000783F2813D10020C043BB4908600220E3
S1135550B84988730020B349C87008460423FD2263
S1135560D20000210090312000F0DEFD5FE0002039
S1135570B04988730520AB49C87008460423FD224E
S1135580D20000210090312000F0CEFD4FE0EAE18E
S11355904EE0DAE10020A74988730520A149C870CC
S11355A008460423FD22D20000210090312000F09F
S11355B0BBFD3CE0A248008AA149498A884206DB37
S11355C09F48008A9E49498A401A80B204900498F0
S11355D0002806D09A494A8A14315018049900F0D8
S11355E095FE95480068C04393490860029809688D
S11355F088420CD100208B49C87008460423FD2240
S1135600D20000210090312000F08EFD0BE0052037
S11356108449C87008460423FD22D200002100906A
S1135620312000F081FD0020C0438349086099E1E6
S11356300B2E0CDA13207D494870481C0123FD22EF
S1135640D20019460090312000F06EFDF7E675484F
S11356500079000673494979090408437149897935
S1135660090208436F49C979084307906D48007AD5
S113567000066C49497A090408436A49897A09028F
S113568008436849C97A0843069006990798401860
S11356904721C902884203D302206A49087002E004
S11356A001206849087067480078012878D13120C2
S11356B0FEF704FE00200590FDF766F8FDF738F8C4
S11356C06148806801218904884205D25E480068E7
S11356D00F21C902884212D05C4880684721C90260
S11356E0884205D2594800680F21C902884202D075
S11356F0012005901FE0FCF7F3FF05901BE0524AE0
S113570051681068FCF7DCFE002811D00720000364
S1135710FEF788FD07464720C002FEF783FD874257
S113572002D10120059006E0FCF7DAFF059002E0C3
S1135730FCF7D6FF05900598012832D1444800F0C3
S11357405BFD0A20FCF7C5FF4721C90207200003BF
S1135750FDF794FE0546002D12D13D483D490860F1
S113576001203449C87300202E49C8700846042318
S1135770FD22D20000210090312000F0D5FC8AE007
S113578000202C49C87305202649C8700846042304
S1135790FD22D20000210090312000F0C5FC7AE007
S11357A00FE000212348C173722020494870481C2F
S11357B00123FD22D20019460090312000F0B4FCF0
S11357C069E020480078022856D13120FEF776FDA2
S11357D01F4800F011FD0A20FCF77BFF012189041A
S11357E007200003FDF74AFE05460A20FCF771FF77
S11357F0002D31D116481749086001210D48C173A5
S113580000200849C87008460423FD22D200002164
S11358100090312000F088FC3DE000001D060020CF
S1135820DF070000541300204E060020F20500207C
S11358300203FFFF6C1D002050060020F605002027
S11358406C180020F1050020601800205418002076
S1135850A55AA55A2006002000204A49C8730520ED
S11358604949C87008460423FD22D2000021009053
S1135870312000F059FC0EE000204249C873052095
S11358804149C87008460423FD22D200002100903B
S1135890312000F049FC65E0FCF7B6FE012844D154
S11358A0032E32D1FCF796FE00281ED1782037490A
S11358B04870481C0123FD22D20019460090312073
S11358C000F032FC002000F097FC0A20FCF701FFF6
S11358D000202D49C87008460423FD22D20000216F
S11358E00090312000F020FC2EE000212548817337
S11358F005202549C87008460423FD22D200002152
S11359000090312000F010FC1EE000201D49887337
S113591013201D49C87008460123FD22D2001946F0
S11359200090312000F000FC0EE000211548817346
S113593005201549C87008460423FD22D200002121
S11359400090312000F0F0FB0CE031200F4948704A
S1135950481C0123FD22D20019460090312000F09A
S1135960E3FB00BF0CE0122008494870481C0123E7
S1135970FD22D20019460090312000F0D5FB5EE5EF
S113598000BF5CE56C1D002054130020F2050020CC
S1135990FEB50E461746F0B201900120A3490870E7
S11359A0A348007800280CD13320A2494870481C31
S11359B00123FD22D20019460090342000F0B4FBEC
S11359C0FEBD9D48007802280CD07F20994948707C
S11359D0481C0123FD22D20019460090342000F017
S11359E0A3FBEDE7002095490870F0B201900198FF
S11359F00A280CD013208F494870481C0123FD222B
S1135A00D20019460090342000F08EFBD8E7002421
S1135A1004E0385D8A490855601C84B201988442C8
S1135A20F7DB87480078002803D18548407844286C
S1135A300CD013207F494870481C0123FD22D2005A
S1135A4019460090342000F06FFBB9E77D480078D8
S1135A50022872D17C48C07B00280CD17020754983
S1135A604870481C0123FD22D200194600903420BE
S1135A7000F05AFBA4E77248807800067049C978A0
S1135A80090408436E490979090208436C494979B4
S1135A9005460D436D4805606948807900066849EC
S1135AA0C979090408436649097A09020843644923
S1135AB0497A084365498860084600680721090354
S1135AC088422CD1614800686049896840180121E6
S1135AD0890488420CD3312056494870481C01235C
S1135AE0FD22D20019460090342000F01DFB67E728
S1135AF0202053490870012048700220887008460D
S1135B000323FD22D20000210090342000F00CFB7E
S1135B1001204D49087400204C49C86083E03120BD
S1135B2044494870481C0123FD22D20019460090C4
S1135B30342000F0F9FA43E7FFE7424800780128EF
S1135B4071D14148C07B00280CD17020394948707C
S1135B50481C0123FD22D20019460090342000F095
S1135B60E3FA2DE73648807800063549C9780904F8
S1135B7008433349097909020843314949790546FB
S1135B800D43324805602E48807900062C49C979B6
S1135B90090408432A49097A090208432849497A29
S1135BA008432A4988600846006807210903884297
S1135BB02CD1264800682549896840184721C90224
S1135BC088420CD331201B494870481C0123FD2214
S1135BD0D20019460090342000F0A6FAF0E6202006
S1135BE01749087001204870022088700846032372
S1135BF0FD22D20000210090342000F095FA01200B
S1135C001149087400201149C8600CE03120094989
S1135C104870481C0123FD22D2001946009034200C
S1135C2000F082FACCE600BFCAE600001E0600209F
S1135C3027060020F20500204E060020F60500206D
S1135C4054130020F10500206C1D00206C18002066
S1135C50F7B5C4B01646002042900120754908707B
S1135C607548007802280DD07F2074494870481C7C
S1135C700123FD22D20019460090362000F054FA88
S1135C8047B0F0BD6E48007800280CD133206B4932
S1135C904870481C0123FD22D2001946009036208A
S1135CA000F042FAECE7459D002404E0305D6549CC
S1135CB00855601C84B2AC42F8DB62480078624943
S1135CC0097C88420CD073205C494870481C01232D
S1135CD0FD22D20019460090362000F025FACFE7C5
S1135CE05948007C43905848007C401C564908742D
S1135CF0681E5649C8600846C068FF2101318842C1
S1135D000CD973204D494870481C0123FD22D20050
S1135D1019460090362000F007FAB1E7681E80B2F9
S1135D2041904A48006807210903884251D34748F3
S1135D3000680121890488424BD2002445E03019CF
S1135D4041784248028A008A401C404B1882184617
S1135D5014308154143800683D49884233D21846BF
S1135D60008A40282FDBFF22402101A8FBF712FC08
S1135D7000270CE03548418A408A401C334A50824F
S1135D8010461430405C01A9C855781C87B2402FD6
S1135D90F0DB40212D48143000F0B8FA2B494022A2
S1135DA0086801A900F038FB42904298002809D104
S1135DB040212648001DFCF781F800202349088271
S1135DC0488200E004E0601C84B241988442B6DB5F
S1135DD00CE0722019494870481C0123FD22D200AE
S1135DE019460090362000F09FF949E77D20C00055
S1135DF0FCF76FFC429800280CD1124943980870B4
S1135E0008460123FD22D20000210090362000F034
S1135E108BF90CE0722009494870481C0123FD22CB
S1135E20D20019460090362000F07EF928E700BF22
S1135E3026E700001E0600204E060020F205002082
S1135E4027060020541300206C1D00206C1800202D
S1135E50C0FF0300F8B504460D461646FCF7D4FB14
S1135E60012823D1FCF7B6FB002812D1782026495B
S1135E704870481C0123FD22D200194600903720A7
S1135E8000F052F9002000F0B7F90A20FCF721FCD9
S1135E9018E072201C494870481C0123FD22D200DE
S1135EA019460090372000F03FF90BE072201649A4
S1135EB04870481C0123FD22D20019460090372067
S1135EC000F032F9012011490870002010490874CB
S1135ED01048007802280CD07F200B494870481CD9
S1135EE00123FD22D20019460090372000F01CF94E
S1135EF0F8BD09480023FD22D2001946009037203E
S1135F0000F012F900BFF3E7F20500201E0600209E
S1135F106C1D00204E06002054130020F7B582B0FB
S1135F2005460E460195F7B2012F0DD013202849DE
S1135F304870481C0123FD22D200194600903E20DF
S1135F4000F0F2F805B0F0BD002405E00498005D0F
S1135F5020490855601C84B2BC42F7DB1D48007818
S1135F60002815D01B480078802811D01A490198C0
S1135F70884200D1E6E7122015494870481C0123E5
S1135F80FD22D200194600903E2000F0CDF8D9E75A
S1135F9010480078802806D101201049087000209C
S1135FA00F490870CEE700200A49087001200B4908
S1135FB0087000200A49087006480123FD22D20017
S1135FC0002100903E2000F0AFF800BFBAE70000C7
S1135FD0F205002054130020DF0700001E060020F5
S1135FE01D060020F7B582B0074600204949087015
S1135FF00398C5B2002405E00498005D464908559D
S1136000601C84B2AC42F7DB012D0DDA1320434946
S11360104870481C0123FD22D200194600908520B7
S113602000F082F805B0F0BD3B4800784606760ED5
S1136030012E0ED0022E0CD0122038494870481C74
S11360400123FD22D20019460090852000F06CF84F
S1136050E8E73348007801280CD17F202F494870A5
S1136060481C0123FD22D20019460090852000F02F
S11360705BF8D7E7012D0CD0132028494870481C41
S11360800123FD22D20019460090852000F04CF82F
S1136090C8E721480078012807D0022816D08128B3
S11360A002D0822822D110E000BF1B480078802152
S11360B00840002808D118480123FD22D2000021FD
S11360C00090852000F030F821E000BF12480078ED
S11360D080210840002808D10F480123FD22D20066
S11360E000210090852000F01FF810E00D48874241
S11360F000D197E7122009494870481C0123FD226A
S1136100D20019460090852000F00EF800BF00BFB1
S113611000BF87E71D06002054130020F20500206D
S11361204E060020DF070000FFB581B00646174683
S11361300A9D0298002822D0224807807F20214906
S113614088700846C670403104984884002406E0EC
S113615029781C48001D01556D1C601C84B2194827
S11361604030408CA042F3DC16494031498C891CF4
S11361708AB214490888891CFEF73CFC20E01248C6
S11361800780402030431049887040310498488487
S1136190002406E029780C48C01C01556D1C601CC5
S11361A084B209484030408CA042F3DC06494031B7
S11361B0498C491C8AB204490888891CFEF71AFCD8
S11361C005B0F0BDF01100208C110020AC20014975
S11361D04870704700100240F0B506460F4614465A
S11361E0354605E028462168FDF77CF9241D2D1D60
S11361F0BD42F7D3F0BD000010B504460648074978
S1136200086008464460064800F0D1F9034A0821B2
S1136210034800F0F7F910BDA55A7AA7FC05002041
S11362200004500030B47446641E2578641CAB42EC
S113623004D3635D5B00E31830BC18471D46F8E7E0
S1136240002805DBC206D20E01219140014A1160EB
S11362507047000080E200E010B5002819DB1A4AFC
S113626003231B02D21883089B00D2588307DC0E39
S1136270FF23A3409A438B071B0E8407E40EA3401D
S11362801A43114B032424021B198408A4001A5135
S113629018E00E4A03071B0F083B9B089B00D258CB
S11362A08307DC0EFF23A3409A438B071B0E84074E
S11362B0E40EA3401A43054B0407240F083CA4082A
S11362C0A4001A5110BD000000E100E01CED00E044
S11362D0BFF34F8F03480449C860BFF34F8F00BF1B
S11362E000BFFDE70400FA0500ED00E002E008C885
S11362F0121F08C1002AFAD170477047002001E03C
S113630001C1121F002AFBD17047000010B50246DC
S11363100B4611460EE00878491C094C247860406D
S11363200006800D074C2058054C2468240A604060
S1136330034C206018465B1E0028ECD110BD000001
S113634050060020E469000010B5044600211048FE
S1136350417002210F48FBF74FFA002816D00221A2
S11363600C48FBF71DFA0B48FBF752FA0A49086080
S11363700A4A084601680748FBF79CFB084800687E
S1136380002803D0054806490968884710BD000065
S11363905C6000400054044010000020B40600205B
S11363A01400002010B5044603492046FBF7C8F842
S11363B00249087010BD000040420F002800002070
S11363C070B50446002C01D1064D01E0012070BDDA
S11363D02846FBF7E8F9032801D10220F7E700205B
S11363E0F5E700000054044072B605208002094914
S11363F08860BFF35F8F62B6FBF7C6FFFBF7E2FF6F
S1136400FEF7A0F9FBF7A0F903E0FEF71DF9FFF78B
S1136410DDFEFAE700ED00E0F8B505460E46144649
S11364200027291932462846FFF7D6FE034800689C
S11364300019024908603846F8BD00006C180020B5
S11364400346002B01D1104A01E00120704750207F
S1136450815A0E48014007200143502081520C48C4
S11364600068C1890B4801400220014308480068C4
S1136470C1815020815A05480140FF200130014369
S1136480502081520020E1E700540440F8F8000055
S113649010000020FCFC000010B588B00446212345
S11364A01F2202210520FDF7DDF820231E220121F1
S11364B00520FDF7D7F80221684601830021817683
S11364C0012181770021C176017706A90520FDF716
S11364D025F801216846018381760021C17606A949
S11364E00520FDF71BF8042168460183002181760D
S11364F0C176022141770021817706A90520FDF7A5
S11365000DF86178684601700221418000214171D3
S11365100B2181710221C171002101716068029017
S1136520A0680390E06804902069059069460C48CF
S1136530FBF798F90B496069086001210848FBF7EB
S11365408DFA012202210648FBF772F90649372029
S1136550FDF7E6FC002105484170002008B010BD9D
S11365600054044014000020496300005C610040B2
S1136570014672B608208F4AD060F120106255207F
S11365805060AA2090600020C043086000BF894882
S11365900068C007C00F0028F9D00120854A1060A8
S11365A00020D060F020106262B6002070470146DF
S11365B072B610207F4AD060F120106255205060DE
S11365C0AA2090600020C043086000BF794800689A
S11365D0C007C00F0028F9D00120764A10600020BF
S11365E0D060F02010621046006804221040002899
S11365F005D004206F4A106062B60120704762B66D
S11366000020FBE770B503461D46F120694E306259
S1136610002415E072B6AA20664E70605520B06062
S113662010782870521C6D1C62B600BF6148006867
S1136630C007C00F0028F9D001205E4E3060641CF2
S11366408C42E7D3F0205B4E3062002070BDF7B57A
S1136650FFB0FFB089B006460F460021FFA8C16114
S1136660012104914802874206D9FFA8C161C0698B
S11366707FB07FB00CB0F0BD029600240DE002980C
S11366800078FFA988610298401C02908869FF285D
S113669001D000200490601C84B2BC42EFD3049863
S11366A0002809D0444845490860FFA83946826A51
S11366B03046FFF7A7FF6DE0750AF119681C400228
S11366C0814202D90120039001E000200390710A65
S11366D049020191F105C90D0091039800280FD0DA
S11366E0002408E00198007805A908550198411C88
S11366F00191601C84B2012080028442F2DB0EE02E
S1136700002408E00198007805A908550198411C67
S11367100191601C84B2012040028442F2DB002417
S11367200DE0FFA8806A01780098001905AA1154A9
S1136730FFA8806A411CFFA88162601C84B2BC422D
S1136740EFD30398002816D01B481C490860680240
S1136750FFF72DFF184819490860691C4802FFF724
S113676026FF154815490860680205AA0121890217
S1136770FFF748FF0EE01048104908606802FFF771
S113678016FF0D480D490860680205AA0121490257
S1136790FFF738FFFFA8C0696AE730B50446002355
S11367A004E025781570641C521C5B1C8B42F8D3E2
S11367B030BD000000000240CDAB34122C0000209C
S11367C001000000020000000300000004000000BB
S11367D00500000006000000000100000101800027
S11367E0020180000501800006018000070180008D
S11367F00002000001020000020200000302000087
S1136800050200000702000001038000000480006C
S1136810030400000005000001058000020581005A
S11368200305000004050000050580000006800043
S113683001068000020680000306800000070000B5
S1136840010700000207000003070000040700001E
S1136850050700000607000007070000000C810080
S1136860010C8000020C8000030C8000040C8000EA
S1136870070D8000000E8100010E8100060E8000CD
S11368800000000000000000000000000000000004
S113689000000000000000000000000000000000F4
S11368A000000000000000000000000001000000E3
S11368B00200800003008000040080000500000046
S11368C00600000000018000010180000201800038
S11368D0050180000601800007018000000281009C
S11368E00102800002020000030200000502000011
S11368F0070200000103800000048000030400007C
S11369000005000001058100020581000305000067
S113691004050000050580000006810001068100D1
S11369200206810003068100000780000107800041
S113693002078000030700000407000005070000A9
S11369400607000007070000000C0000010C80008F
S1136950020C8000030C8000040C8000070D8000F2
S1136960000E0000010E0000060E80000000000072
S11369700000000000000000000000000000000013
S11369800000000000000000000000000000000003
S11369900000000000000000EE060000401F0000A0
S11369A0581B000000000000000108000000000067
S11369B000000000000000000000000000000000D3
S11369C00000000000000000000000008813000028
S11369D002040000000000000000000000000000AD
S11369E03123567100000000963007772C610EEEBB
S11369F0BA51099919C46D078FF46A7035A563E912
S1136A00A395649E3288DB0EA4B8DC791EE9D5E038
S1136A1088D9D2972B4CB609BD7CB17E072DB8E737
S1136A20911DBF906410B71DF220B06A4871B9F38C
S1136A30DE41BE847DD4DA1AEBE4DD6D51B5D4F4C5
S1136A40C785D38356986C13C0A86B647AF962FD2A
S1136A50ECC9658A4F5C0114D96C0663633D0FFA77
S1136A60F50D088DC8206E3B5E10694CE44160D57D
S1136A70727167A2D1E4033C47D4044BFD850DD267
S1136A806BB50AA5FAA8B5356C98B242D6C9BBDB7A
S1136A9040F9BCACE36CD832755CDF45CF0DD6DC75
S1136AA0593DD1ABAC30D9263A00DE518051D7C81C
S1136AB01661D0BFB5F4B42123C4B3569995BACFA7
S1136AC00FA5BDB89EB802280888055FB2D90CC6C8
S1136AD024E90BB1877C6F2F114C6858AB1D61C141
S1136AE03D2D66B69041DC760671DB01BC20D29860
S1136AF02A10D5EF8985B1711FB5B606A5E4BF9FED
S1136B0033D4B8E8A2C9077834F9000F8EA80996DF
S1136B1018980EE1BB0D6A7F2D3D6D08976C64914A
S1136B20015C63E6F4516B6B62616C1CD830658563
S1136B304E0062F2ED95066C7BA5011BC1F4088240
S1136B4057C40FF5C6D9B06550E9B712EAB8BE8B81
S1136B507C88B9FCDF1DDD62492DDA15F37CD38C0A
S1136B60654CD4FB5861B24DCE51B53A7400BCA308
S1136B70E230BBD441A5DF4AD795D83D6DC4D1A43A
S1136B80FBF4D6D36AE96943FCD96E34468867AD11
S1136B90D0B860DA732D0444E51D03335F4C0AAAB0
S1136BA0C97C0DDD3C710550AA41022710100BBEB3
S1136BB086200CC925B56857B3856F2009D466B9FA
S1136BC09FE461CE0EF9DE5E98C9D9292298D0B02F
S1136BD0B4A8D7C7173DB359810DB42E3B5CBDB7DC
S1136BE0AD6CBAC02083B8EDB6B3BF9A0CE2B6035D
S1136BF09AD2B1743947D5EAAF77D29D1526DB0412
S1136C008316DC73120B63E3843B64943E6A6D0D5C
S1136C10A85A6A7A0BCF0EE49DFF099327AE000AA7
S1136C20B19E077D44930FF0D2A3088768F2011E3A
S1136C30FEC206695D5762F7CB67658071366C19D1
S1136C40E7066B6E761BD4FEE02BD3895A7ADA10F2
S1136C50CC4ADD676FDFB9F9F9EFBE8E43BEB717D3
S1136C60D58EB060E8A3D6D67E93D1A1C4C2D8385D
S1136C7052F2DF4FF167BBD16757BCA6DD06B53FC3
S1136C804B36B248DA2B0DD84C1B0AAFF64A033602
S1136C90607A0441C3EF60DF55DF67A8EF8E6E3181
S1136CA079BE69468CB361CB1A8366BCA0D26F25CA
S1136CB036E2685295770CCC03470BBBB916022217
S1136CC02F260555BE3BBAC5280BBDB2925AB42B2C
S1136CD0046AB35CA7FFD7C231CFD0B58B9ED92C41
S1136CE01DAEDE5BB0C2649B26F263EC9CA36A75A6
S1136CF00A936D02A906099C3F360EEB856707725D
S1136D0013570005824ABF95147AB8E2AE2BB17BC3
S1136D10381BB60C9B8ED2920DBED5E5B7EFDC7C4A
S1136D2021DFDB0BD4D2D38642E2D4F1F8B3DD68A1
S1136D306E83DA1FCD16BE815B26B9F6E177B06F9C
S1136D407747B718E65A0888706A0FFFCA3B066689
S1136D505C0B0111FF9E658F69AE62F8D3FF6B6116
S1136D6045CF6C1678E20AA0EED20DD75483044EB8
S1136D70C2B30339612667A7F71660D04D47694946
S1136D80DB776E3E4A6AD1AEDC5AD6D9660BDF4059
S1136D90F03BD83753AEBCA9C59EBBDE7FCFB2470C
S1136DA0E9FFB5301CF2BDBD8AC2BACA3093B353F1
S1136DB0A6A3B4240536D0BA9306D7CD2957DE54FA
S1136DC0BF67D9232E7A66B3B84A61C4021B685DD3
S1136DD0942B6F2A37BE0BB4A18E0CC31BDF055A4C
S1136DE08DEF022D046E0000000000205C06000000
S1136DF0F8150000746F00005C060020341B0000CE
S1136E00FC620000C10223C01301022320FF190306
S1136E101302024A210A1303024A220A1304024AF1
S1136E20230A4D0502040A0A1306021D1C02070167
S1136E300A1307024A1D1418080802010602070271
S1136E400A1808090201070207100A4D0A02010F75
S1136E501E4D0B02010E0A5C0C0201505C0D020473
S1136E600A4D0E02012E0A4D0F02012F0A1A103C80
S1136E70180807041A07050A113C480B07043707CA
S1136E8005091202020C1E4D1302020D0A4D1402D2
S1136E9003190A131504280E1904011B0408071604
S1136EA004021E0403A022174A291E12184B0128AB
S1136EB00A12191E020E0709090A121A4B031814A2
S1136EC0121B2D041E07095D121C1E051F07090B4A
S1136ED00A121E5A06BE191159FA4D2007031E0A3A
S1136EE04D2107031F0A2904590A111AFF0181A31E
S1136EF0054009420C13F0060A12200C095E24090D
S1136F0052CC09620CC10976780916840922240935
S1136F1082FC0946A801B4092EE4290C500C5469DA
S1136F20616E59696E67313030180A545932303005
S1136F302E3038300132621010424154333247311E
S1136F403339474B36344642900843414E5F5354DD
S1136F504429104C43485F3D591050083530304B9C
S1136F6062707323E8071AE0041ADF0401685AFF09
S1136F70014100005566010000000000000000000F
S1136F800000000BFFFFFFFFFFFFFFFFFFFFFFFFFE
S1137000BC672F2800007800000188D0FFFFFFFF35
S1137010FFFFFFFFFFFFFFFFFFFFFFFFFFFFFFFF7C
S1137020FFFFFFFFFFFFFFFFFFFFFFFFFFFFFFFF6C
S1137030FFFFFFFFFFFFFFFFFFFFFFFFFFFFFFFF5C
S1137040FFFFFFFFFFFFFFFFFFFFFFFFFFFFFFFF4C
S11378005469616E59696E673130300000000000C0
S113781054593230302E303830303030620000006D
S1137820424154333247313339474B3634464200B0
S113783043414E5F53544400000000000000000028
S113784043414E5F43485F300000000000000000E9
S113785043414E5F3530304B6270730000000000CE
S1137860E8070000E0070000DF0700000000000058
S1137870FFFFFFFFFFFFFFFFFFFFFFFFFFFFFFFF14
S1137880FFFFFFFFFFFFFFFFFFFFFFFFFFFFFFFF04
S1137890FFFFFFFFFFFFFFFFFFFFFFFFFFFFFFFFF4
S11378A0FFFFFFFFFFFFFFFFFFFFFFFFFFFFFFFFE4
S1138000802F0020DD800000E5800000E780000074
S1138010000000000000000000000000000000005C
S1138020000000000000000000000000EF800000DD
S11380300000000000000000F380000001A901001E
S11380405D0B0100A10B0100D10B0100010C01002B
S1138050310C0100610C0100910C0100C10C010004
S1138060F10C0100210D0100550D0100690D010005
S1138070790D0100AD0D0100BD0D0100CD0D010014
S1138080010E0100450E01008D0E0100D50E010008
S11380901D0F0100650F0100750F0100A90F0100FC
S11380A0DD0F01000D1001004110010075100100E9
S11380B08510010095100100C9100100FD10010098
S11380C0EF3FE8FF0448854600F02CFA00480047DB
S11380D03DEB0100C046C046802F00201648804773
S11380E016480047FEE7FEE7FEE7FEE7FEE7FEE789
S11380F0FEE7FEE7FEE7FEE7FEE7FEE7FEE7FEE754
S1138100FEE7FEE7FEE7FEE7FEE7FEE7FEE7FEE743
S1138110FEE7FEE7FEE7FEE7FEE7FEE7FEE7FEE733
S1138120FEE7FEE7FEE7FEE7FEE7FEE7FEE7FEE723
S1138130FEE7FEE7FEE700000DAF0100C58000008A
S113814030B50B46014600202022012409E00D46EB
S1138150D5409D4205D31D469540491B2546954073
S113816040191546521E002DF1DC30BD70B50024B7
S11381702546002801DA01244042002901DA0125BC
S11381804942FFF7DDFFAC4200D04042002C00D052
S1138190494270BDF0B51FB40646002082B00546C2
S11381A04024019100901BE0019922460F4630467D
S11381B000F066F9049A059B801A994110D3104681
S11381C01946224600F04CF9361A8F41019722468F
S11381D001200021009F00F043F938184D41009020
S11381E02046641E0028DFDC019B009829463246A5
S11381F007B0F0BDF0B51FB486B000200090019028
S113820002900698069980B204900798090C02041B
S11382100014114307900027089D099806913E46D3
S11382203C4603900398A9B20204000C03900498FE
S11382302D0C154348430021224600F011F9C719BB
S1138240714110340E46402CECDB3846029A00F0A3
S113825007F9009A019B80180090594102980191F6
S1138260103002904028CCDB00980BB0F0BD0346E0
S11382700B439B0703D009E008C9121F08C0042A56
S1138280FAD203E00B780370401C491C521EF9D249
S11382907047D2B201E00270401C491EFBD2704705
S11382A00022F6E710B513460A4604461946FFF7BE
S11382B0F0FF204610BD30B504460020034600E020
S11382C05B1C934203D2E05CCD5C401BF8D030BD14
S11382D00321001D401E037812021A43491EF9D5DA
S11382E010467047034603220870000A491C521EB8
S11382F0FAD518467047024670B54A40D30FDB07DB
S113830040002DD04A002AD0010E140E00021202A1
S11383100919400A520A8418E50104465443000A24
S1138320120A2E045043A4194219200CC543AA185A
S1138330120C0125AD03521C521912047F39240476
S113834000D0521C104301D44000491EC2B20C0696
S1138350C0092018401C4008802A02D003E00020F5
S113836070BD40084000002900DA0020184370BDA9
S113837070B502464A40D50F40004A00ED07400858
S11383805208002814D0002A12D0C40DD30D410283
S11383900120C0055202490A520AE41A09181218A7
S11383A07D34914201D3641C00E04900002C01DAC1
S11383B0002070BD0023914201D3891A0343400871
S11383C049000028F7D100290AD0914202D10121A5
S11383D0C90705E0914201D2012101E00121C9430D
S11383E0E005C018401900F05CF870BD10B500221B
S11383F09623114600F05DF810BDC20FD20740006D
S113840040080BD0C10D0723DB01C9184002090540
S1138410400A1143C2084007114370470020014637
S11384207047000010B5002904DB0124E407404232
S11384308C412146002B04DB1C460123DB075242FE
S1138440A341994200D1904210BD00000122D207FD
S1138450002800DB101A002900DB511A88427047FB
S113846010B5202A04DB0146203A9140002010BDBB
S1138470914020239C1A0346E3401943904010BDC9
S113848010B5202A04DB0846203AD040002110BD54
S11384900B46D340D0402024A21A914008431946E9
S11384A010BD002904DA401C490001D140084000F5
S11384B0704770B40024050C05D11024000402D1C7
S11384C0002921D01124050E01D100020834050F22
S11384D001D10001241D850F01D18000A41C0028B6
S11384E001DB4000641C002908D020252E1B0D460A
S11384F0F540A14000D001212943084301061B1B7C
S1138500000ADB1D02D5002070BC7047DB0518187B
S113851080180029F8DA401C4900F5D170BC4008E5
S113852040007047064C0125064E05E0E36807CC81
S11385302B430C3C98471034B442F7D3FFF7C6FDE5
S11385401CFF01003CFF010070B58C180578401C2D
S11385506B075B0F01D10378401C2A1106D1027806
S1138560401C03E006780E70401C491C5B1EF9D1C8
S11385702B0705D40023521E0DD40B70491CFAE7B7
S11385800378401CCB1A921C03E01D780D70491C23
S11385905B1C521EF9D5A142D8D3002070BD70B522
S11385A006F078FE0524204616F082FA00252846B7
S11385B006F064FE204616F07BFA0126304606F0EB
S11385C039FE204616F074FA284606F033FE20469B
S11385D016F06EFA304606F051FE204616F068FAA0
S11385E070BDB0B506F056FE0524204616F060FABC
S11385F00125284606F042FE204616F059FA284680
S113860006F018FE204616F053FA002006F012FE7B
S1138610204616F04DFAB0BDF0B581B006F026FE46
S1138620052016F045FA08270026012006F002FE70
S11386300524204616F03CFA204616F039FA06F0D6
S11386400BFE0546204616F033FA002006F0F2FD34
S1138650204616F02DFA76002E437F1E3806E4D10C
S1138660F0B201B0F0BD70B50446002006F0E2FDA2
S113867006F010FE052016F01BFA0826E0B2C00929
S113868006F0FCFD0525284616F012FA012006F036
S1138690D1FD284616F00CFA002006F0CBFD284642
S11386A016F006FA284616F003FA6400761E300621
S11386B0E4D1052016F0FCF9012070BDF0B583B0BB
S11386C0019314460E4607460120384302900325C1
S11386D004E000F08EF86D1E280631D000F067F833
S11386E03846FFF7C0FF00F0A7F80028F1D1304664
S11386F0FFF7B9FF00F0A0F80028EAD100F057F81E
S11387000298FFF7B0FF00F097F80028E1D1019834
S113871002280BD3451E0026FFF77EFF2070FFF7CB
S11387203EFF641C761CF0B28542F5DCFFF774FF53
S11387302070FFF756FF00F05CF8202003B0F0BD76
S1138740102003B0F0BDF0B583B01C460092019137
S11387500290032504E000F04CF86D1E280623D097
S113876000F025F80298FFF77EFF00F065F8002876
S1138770F1D10198FFF777FF00F05EF80028EAD105
S1138780002C0CD00026009F3878FFF76CFF00F017
S113879053F80028DFD1761C7F1CA642F4D300F0E6
S11387A028F8082003B0F0BD102003B0F0BDB0B528
S11387B006F070FD0524204616F07AF901252846B6
S11387C006F038FD204616F073F9284606F056FDEB
S11387D0204616F06DF90025284606F04FFD204688
S11387E016F066F9284606F025FD642016F060F9B7
S11387F0B0BDB0B506F04EFD0524204616F058F97C
S11388000025284606F016FD204616F051F92846A4
S113881006F034FD204616F04BF90125284606F0F3
S113882009FD204616F044F9284606F027FD642089
S113883016F03EF9B0BD0000B0B506F017FD0524F2
S1138840204616F035F9012006F0F4FC204616F017
S11388502FF90B4D06F000FD044606F0E5FC002C54
S113886002D06D1E2804F5D10525284616F020F9FE
S1138870002006F0DFFC284616F01AF92046B0BDA9
S113888033210000034801780B2901D8491C0170E9
S11388907047C0466F2B002070B584B00025039547
S11388A002950195009506F0BFFC0F20C6430E4CBF
S11388B01036F1B2A0206A461023FFF744FF204689
S11388C016F0F6F8204616F0F3F8912EF0D3A02017
S11388D0B0216A461023FFF736FF204616F0E8F869
S11388E00248058004B070BD581B0000622B0020B4
S11388F070B5022902D2EB24E0B270BD891EEB25CB
S11389000022134605E0401C5B1CDDB2A94225464B
S11389100EDB04786C40154604E034466E1C072DCB
S11389203546F0D26608E407F7D09A246640F4E7A7
S1138930E0B270BDF0B591B00C91417810AA1170FD
S113894083781B025918C37804792402E3181B04A2
S113895059180B0ED3700C0C94700D0A55700B91B2
S113896008956918099409190A93C9180278D24319
S11389708918427983791B029A18C379047A2402EC
S1138980E3181B049A188918130A0693C918130CC0
S11389900593C9180792120E04928918827AC37A31
S11389A01B029A18037B0F90447B2402E3181B04D8
S11389B098180918020A02928918020C019289185F
S11389C00D910390000E0E9000200346014606E030
S11389D032409A40D2B211435B1C082B0ED00126C0
S11389E035469D400746024602E07F1C042FEFD027
S11389F010ACE45D2542F8D0521CF6E70E9C0D98AD
S1138A000019C3B20F98827B934205D0427A9142F7
S1138A1002D1002011B0F0BD1021FFF769FF0C99BD
S1138A20CC72019A8A72029A4A72039A0A72049A5E
S1138A30CA71059A8A71069A4A71079A0A710A9A42
S1138A40CA70099A8A70089A4A700B9A0A7011B00F
S1138A50F0BDF0B58DB055220270002747720B7837
S1138A604370CA79059202728A790492C2714A7972
S1138A70039282710A7902924271CA7A089242730D
S1138A808A7A019202734E7AC6720C7A84720CAAA4
S1138A9013704D782D02EB188D78C97809024919A5
S1138AA00904CB18190E01711D0CC57009931B0A1A
S1138AB00B90837038460A91D17007959570069390
S1138AC0537031020919089A1202019BD218120438
S1138AD05118089103990902029A8918059A1202F9
S1138AE0049BD2181204511805913D463A4605E0FC
S1138AF02640AE4032436D1C082D0ED00124214681
S1138B00A9400346064602E05B1C042BF0D00CAFE0
S1138B10FF5C3942F8D0761CF6E70B9B5A72099831
S1138B2006994018079940180A994018059A801820
S1138B30110A4018110C4018110E4018089A801898
S1138B40110A4018110C4018110E40185638987329
S1138B5010211846FFF7CCFE0DB0F0BDF0B58FB074
S1138B600446FF20E070A07060700F20C0430290A4
S1138B700F302070704815F09BFF70490868632817
S1138B8001D8642008606E4F002038806D4E01903B
S1138B90308008E00B99814222D338881030388025
S1138BA080B2A1286DD206F03FFB3978A02003AA39
S1138BB01023FFF783FD30802028EED103AD0BA9ED
S1138BC02846FFF7B7FEE97B8842E6D12878552886
S1138BD0E3D15D48017800290298DBD10846D9E742
S1138BE03888A0284DD8C0B20021019105E006F0D4
S1138BF01BFB3988C8B2A12943D2C1B2A02003AA61
S1138C001023FFF75BFD308039881031398020282C
S1138C1037D103AD07A92846FFF78CFEE97B8842CC
S1138C20E5D128785528E2D14748007800280299F0
S1138C3000D1014607988842D9D240490A68962152
S1138C4051430B9A824208D90818904219D30BA9B0
S1138C500E222046FFF70BFBC9E78918814210D387
S1138C6007A90E222046FFF702FB0BA80A9981816F
S1138C7007980B9008980C9009980D9038880190EB
S1138C80B5E72078617809020818A178E278120221
S1138C90511809040818401C24D100200190388080
S1138CA0A020B02103AA1023FFF708FD308020285C
S1138CB018D103AD0BA92846FFF73CFEE97B884297
S1138CC010D1287855280DD11F480078002800D1EC
S1138CD002900B980299884204D20BA90E222046D6
S1138CE0FFF7C5FA2078617809020818A178E278BC
S1138CF01202511809040818401C0CD10020E0721B
S1138D00A07260722072E071A07160712071E070D5
S1138D10A070607020700198388020786178090212
S1138D200818A178E27812025118090408180749B2
S1138D30086030880FB0F0BD701101005C2B00207A
S1138D40622B0020582B00205B2B0020682B002076
S1138D50F0B581B000910646214800250570002A2F
S1138D602ED01446C036631B71190F200840102200
S1138D70101A834200D303461A480278102A01D0FD
S1138D80042A1AD1C809FE2707405F2F13D80127E8
S1138D90B8436038C0B29E3282420CD3009A521952
S1138DA0C9B2DFB23B46FFF789FC0F490880ED19D1
S1138DB0A542D8D304E0082000E004200A49088032
S1138DC0094801880020042902D0082900D0012084
S1138DD003490870411E8841400001B0F0BDC046FF
S1138DE06E2B00205A2B00206C2B00200A4A0123F2
S1138DF013700A4A10700A4A11600A4A002111606D
S1138E00042801D105218901102801D11D208101E7
S1138E10054801807047C0465B2B00205A2B002078
S1138E205C2B0020682B0020602B0020F0B587B05D
S1138E30994D00262E80994B1B688B4224D1994C66
S1138E402188202925D1029000920196964C002772
S1138E502760964D964E2878062809D806F0E4F93E
S1138E602068401C2060B042F5D38D480421018065
S1138E702F70904C20880107029B31D08848202114
S1138E800180854D019E0BE0012040028449088049
S1138E9006E003A8FFF762FE20808148802101805C
S1138EA07F4800883F2807DD874988420BDC40283B
S1138EB012D0802810D010E004280DD008280AD041
S1138EC0202809D009E001214A02904204D0C902B5
S1138ED0884201D001E002262E80288807B0F0BD28
S1138EE0A128019E00D32780009A012A6A4D1ED131
S1138EF0187B012856D1DF719F715F711F711F7339
S1138F00587B012804D1DF729F725F721F725F73F6
S1138F1003AF38461946FFF79CFDF87320880028F4
S1138F2046D01038C1B2A02003AA102344E0002A7E
S1138F30B6D1614801780029B2D002701878597806
S1138F40090208189978DA781202511809040818E5
S1138F505A490978002901D00F21C943884233D2E4
S1138F60274603AC20461946FFF773FDE0733978B2
S1138F70A02010232246FFF7E6FB029A4849088006
S1138F8008288DD13888103038801078517809023B
S1138F9008189178D278120251180904081848491F
S1138FA008607DE7597B012911D10128A3D0A7E7E7
S1138FB0A02003AA10230146FFF7C5FB3849088007
S1138FC03D48009901706BE70120C0025EE73D480F
S1138FD00078012812D103AC20461946FFF739FD69
S1138FE0E073A020B02110232246FFF7ACFB2C49EC
S1138FF008800828E4D133480770E1E718785978E5
S1139000090208189978DA78120251180904081824
S11390102B490968214A12685118884203D2204812
S113902040210180CCE725490978002901D00F218E
S1139030C94388422DD203AF384619461C46FFF770
S113904008FDF8731B480178A02010233A46FFF767
S11390507AFB134908800828B2D1164908881030D1
S113906008802078617809020818A178E278120251
S11390705118090408181249086008490A6815219A
S11390805143FFF75DF800299AD101200D4908707A
S113909096E70120C00291E7742B00205C2B00208E
S11390A0722B0020582B0020782B00206F2B0020DF
S11390B0818D5B00622B0020642B00205B2B002041
S11390C0682B0020702B0020FF010000F0B585B054
S11390D00646434C0027278004921018414A128800
S11390E0904241D201910397404F00200290386092
S11390F03F4C404D2078052809D806F095F838688B
S1139100401C3860A842F5D33748042101800298F6
S113911020703948018839480278102A01D0042A7D
S113912032D188190346C033049C651A0F240440C5
S11391301020001B854200DB0546DC09603C01264B
S11391403002E7B27F09052F12D3B443E6B29E3250
S1139150B242234C039F0DD301984218D9B2EBB20B
S11391603046FFF7F0FA05E01F482021018011E0A6
S11391701B4C039F1C49088008280BD1E8B21E4AE7
S113918011880818108005E0012080021649088023
S1139190134C039F144800881F2809DD202813D08E
S11391A001210A0290420FD0890288420CD00CE0BF
S11391B0042809D0082808D10F4800880499884257
S11391C001D3022700E001272780208802210143E0
S11391D0022902D1084900220A8005B0F0BDC04628
S11391E0742B0020602B0020722B0020782B002091
S11391F06F2B0020818D5B007C2B00205A2B0020DC
S1139200F0B585B0044600200190042C6FD20BF019
S113921075FB002801D10BF0F1FB0020009000BF8A
S11392200098401C00900BF069FB03900398002801
S113923003D0484900988842F2D30398002856D1B5
S1139240042145480BF03CFB444845490880210172
S1139250444A515C4900404A505A41490A88012114
S1139260090300F055F902900120049020013D49C2
S113927040184078002801D100264BE020013949EC
S113928040184078012802D13548068842E0200180
S113929034494018407802282AD120014018057921
S11392A02901304A515C49002B4A505A2C490A88FA
S11392B00121090300F02CF9064628012A49431824
S11392C02801284940180289280140180021C7684C
S11392D03046B84706462801224BC018C2882801E8
S11392E0C0188178304600F087F8064612E02DE079
S11392F020011C4940184078032804D0200140185C
S11393004078132804D1200116494018868801E0CA
S1139310002004900498002818D020011249431812
S11393202001104940180289200140183146C768BD
S11393300298B847019020010A4BC018C288200146
S1139340C0188178019800F057F80190019805B091
S1139350F0BD000050C300000C0100208813000081
S113936006010020C0F5010000F60100F8B505462D
S11393700E4614460020009001211C4801751C482B
S1139380007888431A490870084680780821084301
S11393901749887000208871084600780121084325
S11393A01349087008460572002717E01048007832
S11393B0802108430E49087000BF0E48007D002834
S11393C0FBD000200B4908750948C0892080A41CE3
S11393D00748C1890098081800907F1CB742E5D35C
S11393E031460098FEF7ACFE80B2F8BD4061004003
S11393F0005004404060004010B50346012908D1E4
S1139400094CA41A9C4202D99C18A0B20BE006484D
S113941009E0022906D1934202DD9C1AA0B202E0BF
S1139420002000E0184610BDFFFF000010B5044600
S11394300121202001F0D0FF0020324908700121D1
S113944031480175002031490875152015F018F8C8
S11394502C488078E17808432A4988700846807847
S113946021780843274988702078802806D1084647
S11394700079E1794900084322490871214880783C
S1139480E17A08431F498870A078002803D1084670
S1139490007908710FE0A078012806D119480079F5
S11394A0602108431749087105E0164800798021B6
S11394B008431449087113488079217908431149F4
S11394C0887108468079617908430E498871207A49
S11394D0C872607A8872084600783821884309493E
S11394E00870084600786178C90008430549087087
S11394F0A07A0873084600780121084301490870DE
S113950010BD000000500440406100404060004035
S1139510F8B504460E461746002E01D100250FE08B
S1139520A64201DC3D460BE00094009C20467843B3
S1139530009031460098FEF703FE0090009885B233
S11395402846F8BD0146042904D28A00024BD218E9
S1139550508800E000207047AC2400200146042914
S113956003D28A00024B985C00E0002070470000A0
S1139570AC240020FFB587B004460898844203DA7F
S11395800A988068002802D12448019042E0089893
S1139590001B82B20292002625460A9880680021A8
S11395A02F463A463346049605910690FEF722FE6E
S11395B005460E46002328463146029AFEF7EAFD88
S11395C005460E46304600210A46494050400143B4
S11395D002D0124801901DE003950A98C068039DCB
S11395E0A84202D30020019014E00A98C1680398AD
S11395F0401A039009990398FEF7A2FD039003987B
S1139600000C0004002802D00448019002E00398F2
S113961080B2019001980BB0F0BD0000FFFF000084
S113962010B5084800788021884306490870012154
S113963005480175002005490875152014F020FF20
S113964010BD0000005004404061004040600040F4
S1139650F8B505460E4614461F4621462846FEF731
S113966085FD80B2F8BD0000FFB587B006460A98B4
S11396704068002801D1029035E00A9801684068EA
S113968008180390002534460021274603980695C0
S11396900491059038462946049B059AFEF7AAFDD5
S11396A004460D460A98406802460023019020466D
S11396B02946FEF76FFD04460D4600232046294641
S11396C0099AFEF767FD04460D46284607492140DE
S11396D0002359405840014303D00448C04302903A
S11396E001E0A0B2029002980BB0F0BD0000FFFFB1
S11396F010B5FE4800688079030014F0A7FE070542
S11397009ED8F5F4F3F2F100F848006840790300BC
S113971014F09CFE0805138A2A8A468A638A11F08B
S113972027F80020F1490968C873F04800684079B7
S1139730401CEE49096848717DE0ED494969EB4AEE
S11397401268D27A885C11F08BF8E8480068407996
S1139750401CE64909684871E44800684079401CA7
S1139760E2490968487166E009F008FC002810D154
S113977011F076F8DD4800684079401CDB4909683F
S11397804871DA4800684079401CD8490968487132
S113979005E011F017F80020D449096848714AE03F
S11397A009F0ECFB002811D1112011F059F8CF4831
S11397B000684079401CCD4909684871CB4800686D
S11397C04079401CC9490968487105E010F0FAFF66
S11397D00020C649096848712DE009F0CFFB002834
S11397E01BD1C2480068C07A401CC0490968C872CD
S11397F0BE480068C07ABE49097888420DDB002063
S1139800BA490968C872B94909684862B748006822
S11398108079401CB5490968887110F0D3FF002095
S1139820B2490968487106E010F0CCFF0020AF4946
S11398300968487100BF00BF32E3AC480068407C4F
S1139840002817D0AA48C068002803D0A848C168D7
S1139850192088470020A54909684862A348006880
S11398608079401CA1490968887100209F490968D2
S113987048711BE09D480068406A282807D29B482D
S11398800068406A401C9949096848620EE000205B
S1139890964909684862954800688079401C934954
S11398A0096888710020914909684871F8E28F4875
S11398B000684079030014F0C9FD080518A42FA41A
S11398C04CA480A410F054FF002088490968C87390
S11398D0864800684079401C84490968487197E0CB
S11398E0D4E2C7E230E25DE194E0814949697F4A0C
S11398F01268D27A885C10F0B3FF7C480068407923
S1139900401C7A4909684871784800684079401CCD
S11399107649096848717BE009F030FB002811D1D1
S1139920012010F09DFF714800684079401C6F4988
S1139930096848716D4800684079401C6B490968A2
S1139940487105E010F03EFF00206849096848713D
S11399505EE009F013FB002828D164490968C97A3C
S113996024225143634A12688918604A1268D27BE0
S1139970885C10F075FF5D480068C07B401C5B4943
S11399800968C87359480068C07B242814D3574811
S113999000684079401C554909684871534800687B
S11399A04079401C51490968487105E010F00AFFEC
S11399B000204E49096848712AE009F0DFFA0028BE
S11399C018D14A480068C07A401C48490968C872DE
S11399D046480068C07A4649097888420ADB002074
S11399E042490968C872414800688079401C3F496F
S11399F00968887110F0E6FE00203C490968487146
S1139A0006E010F0DFFE002038490968487100BF05
S1139A1000BF45E2354800684079030014F016FDA4
S1139A200A0614B92BB948B978B995B910F0A0FE53
S1139A3000202E490968C8732C4800684079401CEE
S1139A402A4909684871ABE029494969274A1268DB
S1139A50D27A885C10F004FF244800684079401CE6
S1139A60224909684871214800684079401C1F490F
S1139A700968487194E009F081FA002811D14A205C
S1139A8010F0EEFE194800684079401C1749096837
S1139A904871164800684079401C144909684871A7
S1139AA005E010F08FFE002010490968487177E046
S1139AB009F064FA002824D1FF2010F0D1FE0B48ED
S1139AC00068C07B401C09490968C87307480068DE
S1139AD0C07B24281BD3054800684079401C0349F7
S1139AE00968487101480068407905E0D007002002
S1139AF0402B0020CC070020401CEA49096848712B
S1139B0005E010F05FFE0020E6490968487147E06F
S1139B1009F034FA002811D1FF2010F0A1FEE14829
S1139B2000684079401CDF4909684871DD480068D5
S1139B304079401CDB490968487105E010F042FE99
S1139B400020D849096848712AE009F017FA00286A
S1139B5018D1D4480068C07A401CD2490968C87238
S1139B60D0480068C07AD049097888420ADB0020CE
S1139B70CC490968C872CB4800688079401CC9493F
S1139B800968887110F01EFE0020C64909684871F2
S1139B9006E010F017FE0020C2490968487100BFB2
S1139BA000BF7DE1BF4800684079030014F04EFC1B
S1139BB00C0715C32CC349C366C382C39FC310F0EB
S1139BC0D7FD0020B7490968C873B64800684079D2
S1139BD0401CB44909684871B4E0B3494969B14AC1
S1139BE01268D27A885C10F03BFEAE480068407977
S1139BF0401CAC4909684871AA4800684079401C77
S1139C00A849096848719DE009F0B8F9002811D104
S1139C10772010F025FEA34800684079401CA14934
S1139C20096848719F4800684079401C9D4909684B
S1139C30487105E010F0C6FD00209A490968487192
S1139C4080E009F09BF9002811D10C2010F008FEE7
S1139C50944800684079401C9249096848719148C9
S1139C6000684079401C8F490968487105E010F08C
S1139C70A9FD00208B490968487163E009F07EF969
S1139C80002810D110F0ECFD864800684079401C93
S1139C90844909684871834800684079401C8149B7
S1139CA00968487105E010F08DFD00207D490968C0
S1139CB0487147E009F062F9002811D1132010F02F
S1139CC0CFFD784800684079401C7649096848719E
S1139CD0744800684079401C72490968487105E07D
S1139CE010F070FD00206F49096848712AE009F0FE
S1139CF045F9002818D16B480068C07A401C6949AE
S1139D000968C87267480068C07A67490978884258
S1139D100ADB002063490968C872624800688079D8
S1139D20401C60490968887110F04CFD00205D49B1
S1139D300968487106E010F045FD0020594909689A
S1139D40487100BF00BFABE056480068407903008B
S1139D5014F07CFB080513872A874787638710F074
S1139D6007FD00204F490968C8734E4800684079D0
S1139D70401C4C49096848717AE04B494969494A91
S1139D801268D27A885C10F06BFD4648006840790E
S1139D90401C444909684871424800684079401CA5
S1139DA040490968487163E009F0E8F8002811D1D6
S1139DB0492010F055FD3B4800684079401C394962
S1139DC009684871374800684079401C354909687A
S1139DD0487105E010F0F6FC00203249096848712A
S1139DE046E009F0CBF8002810D110F039FD2D48D9
S1139DF000684079401C2B4909684871294800686B
S1139E004079401C27490968487105E010F0DAFCE4
S1139E1000202449096848712AE009F0AFF80028B5
S1139E2018D120480068C07A401C1E490968C872CD
S1139E301C480068C07A1C49097888420ADB002063
S1139E4018490968C872174800688079401C154988
S1139E500968887110F0B6FC00201249096848713D
S1139E6006E010F0AFFC00200E490968487100BFFD
S1139E7000BF15E000200B49096888710949096889
S1139E804871062007490968C87009E010F09AFC77
S1139E90002004490968487102490968887100BFB3
S1139EA000BF10BDD0070020402B002010B56A4829
S1139EB000684079030014F0C9FA090610C627C6E1
S1139EC044C6608EC60010F053FC634800684079B5
S1139ED0401C614909684871BCE0604949695E4AAF
S1139EE01268D27A885C10F0BBFC5B480068407949
S1139EF0401C594909684871574800684079401C1A
S1139F00554909684871A5E009F038F8002811D1CD
S1139F107F2010F0A5FC504800684079401C4E4951
S1139F20096848714C4800684079401C4A490968EE
S1139F30487105E010F046FC002047490968487163
S1139F4088E009F01BF8002810D110F089FC424881
S1139F5000684079401C4049096848713E480068DF
S1139F604079401C3C490968487105E010F02AFC1E
S1139F7000203949096848716CE008F0FFFF0028A7
S1139F8022D135480068C07A401C33490968C87238
S1139F9031480068C07A3149097888420FDB0020D3
S1139FA02D490968C8722C4800684079401C2A4928
S1139FB009684871002028490968486208E00020BF
S1139FC025490968487103E000202349096848715C
S1139FD010F0F8FB3EE020480068407C002816D0D2
S1139FE01E48C068002803D01C48C168192088474F
S1139FF000201949096848621749096848711649D7
S113A00009688871052014490968C8701AE0124863
S113A0100068406A282807D20F480068406A401C3C
S113A0200D49096848620DE000200B49096848623F
S113A0300949096848710849096888710520064971
S113A0400968C87006E010F0BDFB002002490968E9
S113A050487100BF00BF10BDD0070020402B002076
S113A06010B50024F7480068807A01287ED1F548AD
S113A0700068C07900287AD0F24800688079002806
S113A08004D0012874D0022873D191E1ED4800680E
S113A090007B24286ED2EB480068C07901287AD16D
S113A0A0002475E0E7480068C07A24214843E64963
S113A0B009684018E3490968097B415CE148006884
S113A0C0C07A24225043E14A12688018DD4A12689B
S113A0D0127B805C814229D0DA480068C07A24214E
S113A0E04843DA4909684018D6490968097B415C44
S113A0F0D4480068C07A24225043D34A1268801896
S113A100D04A1268127B8154CE480068407B2428D0
S113A11005D3CC480068007BCA4909684873C9481C
S113A1200068007BC7490968887308E0C54800686F
S113A130407B242803D20120C24909688871C148A0
S113A1400068007B401CBF4909680873BD4800686B
S113A150007B242808D3BB480068407B242803D212
S113A1600120B84909688871B64805E0D3E1CDE11A
S113A17069E0BAE138E00EE00068007B242804D2EC
S113A180B04800688079012800D103E0601CC4B2A3
S113A190242C87D356E0002413E0AA480068C07A30
S113A1A024214843A94909684018015DA54800686D
S113A1B0C07A24225043A44A126880180155601CB6
S113A1C0C4B2242CE9D300209E4909684873232093
S113A1D09C490968887301209A4909688871242078
S113A1E09849096808732DE00020964909680873A6
S113A1F094480068C07A401C92490968C872914822
S113A2000068C07A92490978884217DB8D48006853
S113A210007C012804D102208A490968887106E07B
S113A220002088490968887186490968C871002036
S113A23084490968C87283490968087400208149FF
S113A2400968487161E17F4800684079030014F0AF
S113A250FDF8080513A62AA651A68EA60120794961
S113A2600968087410F084FA764800684079401C44
S113A27074490968487199E075494969714A1268D5
S113A280D27A885C10F0ECFA6E4800684079401C81
S113A2906C49096848716B4800684079401C6949F9
S113A2A00968487182E008F069FE00281BD16549FD
S113A2B00968497B491CC8B210F0D2FA61480068A9
S113A2C0407B60490968C8735E4800684079401C57
S113A2D05C49096848715B4800684079401C5949E9
S113A2E00968487105E010F06DFA002055490968C5
S113A2F048715BE008F042FE00282BD151490968FF
S113A300C97A24225143504A126889184D4A126866
S113A310D27B885C10F0A4FA4A480068C07B401CD9
S113A32048490968C87347480068C07B45490968BB
S113A330897B88421ADD434800684079401C4149C2
S113A340096848713F4800684079401C3D490968E4
S113A35048710BE010F036FA3A480068407B3949FE
S113A3600968C87300203749096848711EE008F07D
S113A37005FE00280CD1334909688871242031492D
S113A3800968C8732F49096848732E490968887396
S113A39010F018FA00202B490968487106E010F003
S113A3A011FA002027490968487100BF00BFACE0DA
S113A3B0244800684079030014F048F808050F8E1B
S113A3C0268E4C8E688E10F0D3F91E4800684079B2
S113A3D0401C1C490968487185E01D494969194AAE
S113A3E01268D27A885C10F03BFA1648006840790B
S113A3F0401C144909684871124800684079401C9F
S113A4001049096848716EE008F0B8FD002811D1C0
S113A410492010F025FA0B4800684079401C09498E
S113A42009684871074800684079401C0549096873
S113A430487105E010F0C6F9002002490968487126
S113A44051E00000D0070020CC070020C8070020FE
S113A450402B002008F092FD002810D110F000FAE3
S113A4609C4800684079401C9A4909684871994899
S113A47000684079401C97490968487105E010F06C
S113A480A1F900209349096848712CE008F076FD91
S113A49000281AD18F480068C07A401C8D49096889
S113A4A0C8728C480068C07A8B49097888420CDBF2
S113A4B0002088490968C8728649096888718549F5
S113A4C00968487183490968C87110F07BF9002054
S113A4D080490968487106E010F074F900207D494C
S113A4E00968487100BF00BF0FE010F06BF900204D
S113A4F07849096848717749096888717549096814
S113A500087374490968C87200BFE2E00020714909
S113A51009688872DDE06F480068807A0228F4D107
S113A5206C480068007A002879D06A48006840794D
S113A530030013F08BFF0B0711BB25BB41545EBB1B
S113A5407590BB0010F014F9624800684079401C13
S113A550604909684871B7E05F494969087810F0B3
S113A5607FF95C4800684079401C5A490968487181
S113A570584800684079401C564909684871A3E06E
S113A58008F0FCFC002810D110F06AF9514800686A
S113A5904079401C4F49096848714E480068407929
S113A5A0401C4C490968487105E010F00BF9002083
S113A5B048490968487187E008F0E0FC002807D1A1
S113A5C0444800684079401C42490968487103E0E6
S113A5D0002040490968487110F0F4F874E010F064
S113A5E0C7F83C4800684079401C3A4909684871FA
S113A5F06AE0394949690978491CC8B210F030F950
S113A600344800684079401C32490968487131482F
S113A61000684079401C2F490968487154E054E0AF
S113A62008F0ACFC00280FD110F074F8294909682F
S113A6308870012010F0E8F8264800684079401C32
S113A64024490968487105E010F0BCF8002021494C
S113A6500968487138E01F480068807811280CD1D7
S113A66000201C4909680872AA201A4909688870E0
S113A670002018490968487011E0164800684078BD
S113A680401C14490968487012480068407803283F
S113A69005D308F013FD00200E490968487010F036
S113A6A091F800200B49096848710DE010F08AF810
S113A6B00020084909684871064909684870AA20B9
S113A6C004490968887000BF03E000200149096853
S113A6D0887210BDD0070020402B002010B5024620
S113A6E09000074BC018405C002802D00320C043F0
S113A6F010BD01209300024C1B1958540020F7E7A9
S113A700E826002070B5002508E06D1C1B48854232
S113A71002D20AF09FF901E0002503E00AF0EEF806
S113A7200028F2D100BF022100200AF0F5F803212D
S113A73000200AF0F1F8052100200AF0EDF80721C5
S113A74000200AF0E9F8002408E00020A1000C4AE7
S113A7505054A10089184880601CC4B2042CF4D35E
S113A76001200849087000204870052088700020E6
S113A770C87005480549088070BD000050C300003A
S113A780AC240020080100208813000006010020EA
S113A790F8B58D480078030013F058FE060405163A
S113A7A03D5EFDFC0EE10AF029F900208649C870DF
S113A7B0487008468078002802D10320087002E01F
S113A7C0022081490870FDE07F488078002804D089
S113A7D07D488078401E7C4988700AF08FF80028F4
S113A7E00BD10AF00BF900207749C870084680782D
S113A7F000280FD1032008700CE07348C078401C77
S113A8007149C8700846C078052803D3052008702C
S113A8100AF020F9D6E00AF071F800280ED10421DC
S113A8206A480AF04DF800206749C87048706848C3
S113A830684908800420644908700CE06248C078C4
S113A840401C6149C8700846C078052803D3052018
S113A85008700AF0FFF8B5E05B49497809015E4ADF
S113A860515C4900594A505A5A490A88012109033E
S113A870FEF74EFE009001255348407800015649EA
S113A88040184078002801D100243CE04E4840782C
S113A8900001514940184078012802D14D480488EC
S113A8A031E04948407800014B494018407802287B
S113A8B012D1454949780901474A89180879FEF7B0
S113A8C041FE0446404949780901434A89180879F8
S113A8D0FEF744FE054616E03B48407800013E4939
S113A8E040184078032806D03748407800014018C3
S113A8F04078132806D1344840780001364940187E
S113A900848800E00025002D2FD02F4840780001D6
S113A910324943182C48407800012F4940180289D5
S113A92029484078000140182146C7680098B84774
S113A9300646254840780001274BC018C2882248A3
S113A94040780001C01881783046FEF755FD064670
S113A9501D484078800022494018468001201A4949
S113A960497889001E4A50540AE000201649497863
S113A97089001B4A89184880134949788900505432
S113A98011484078401C1049487008464078042813
S113A99009D301E013E007E00AF030F800200A4987
S113A9A04870032008700DE009F0A8FF002803D1C7
S113A9B001200549087001E00AF04CF802E0FFF7B5
S113A9C0A1FE00BF00BFF8BD080100200C0100205B
S113A9D08813000006010020C0F5010000F6010004
S113A9E0AC24002010B509F053FF002405E000203A
S113A9F0A100074A5054601CC4B2042CF7D30020B1
S113AA00044908700520887003480449088010BD73
S113AA10AC24002008010020881300000601002057
S113AA2070B50446002000F0AFF8002000F0DAF81A
S113AA30002000F09BF8002000F0C4F8002000F093
S113AA4087F8002000F0AEF800BF012000F08EF877
S113AA50012000F0B7F8002521E0002000F086F87E
S113AA60002000F0AFF880202040002806D001200C
S113AA7000F08AF8012000F0B5F805E0002000F0AD
S113AA8083F8002000F0AEF800BF012000F06EF85B
S113AA90012000F097F86006040E681CC5B2082D6A
S113AAA0DBDB012000F054F8012000F07BF870BDDE
S113AAB070B504460D46012000F066F8012000F050
S113AAC091F8002000F052F8002000F07BF80020FC
S113AAD000F03EF8002000F065F800BF012000F00F
S113AAE045F8012000F06EF8002628E0002000F070
S113AAF03DF8002000F066F880202040002803D0B4
S113AB00012000F041F802E0002000F03DF8802030
S113AB102840002803D0012000F064F802E000205F
S113AB2000F060F800BF012000F020F8012000F0E0
S113AB3049F86006040E6806050E701CC6B2082E9D
S113AB40D4DB012000F004F8012000F02BF870BDE4
S113AB5010B50446002C04D0812103200AF008F823
S113AB6003E0802103200AF003F810BD10B5044669
S113AB70002C04D08121042009F0FAFF03E0802195
S113AB80042009F0F5FF10BD10B50446002C04D0D4
S113AB908121022009F0ECFF03E08021022009F06A
S113ABA0E7FF10BD10B50446002C04D081210448F1
S113ABB009F0DEFF03E08021014809F0D9FF10BD50
S113ABC00107000010B50446002C05D081210720A0
S113ABD0000209F0CDFF04E080210720000209F003
S113ABE0C7FF10BD10B50446002C04D081210448D1
S113ABF009F0BEFF03E08021014809F0B9FF10BD50
S113AC000207000010B5F920FFF70AFF8820FFF7BC
S113AC1007FF9020FFF704FF9820FFF701FF0821AA
S113AC200846FFF745FFE820FFF7FAFE1221084621
S113AC30FFF73EFFA020FFF7F3FE70210846FFF761
S113AC4037FFA820FFF7ECFE70210846FFF730FF1E
S113AC50B020FFF7E5FE70210846FFF729FFB82072
S113AC60FFF7DEFE00210846FFF722FFC020FFF7B2
S113AC70D7FE00210846FFF71BFFC820FFF7D0FED0
S113AC8000210846FFF714FFD020FFF7C9FE2F214B
S113AC900846FFF70DFFD820FFF7C2FE2F21084614
S113ACA0FFF706FFE020FFF7BBFE2F210846FFF762
S113ACB0FFFE4020FFF7B4FE00210846FFF7F8FE30
S113ACC00A20FFF7ADFE002405E000210846FFF747
S113ACD0EFFE601CC4B25A2CF7DB00240AE000200B
S113ACE00B4908550B4908550B4908550B4908559C
S113ACF0601CC4B25A2CF2DB8120FFF791FE0020C5
S113AD00074908708870C8700871487010BD000049
S113AD10EC21002046220020A0220020FA2200205C
S113AD20D000002010B58020FFF77AFE10BD00008F
S113AD30002004490870012003490870002048706D
S113AD4070470000D5000020D000002010B548480E
S113AD50007800287AD046488078030013F076FB08
S113AD600604434A535A687E414800794149085CC5
S113AD703F490979404A515C884209D13C480079ED
S113AD803E49085C3A4909793D4A515C88421BD0E6
S113AD90374800793749085C35490979364A5054AF
S113ADA0334800793549085C31490979344A5054AB
S113ADB02F48C078002803D004202D49887011E062
S113ADC001202B4988700DE000202949C8700846ED
S113ADD00079401C0871084600795A2802DB0020DB
S113ADE00871087041E04020FFF71AFE0220204954
S113ADF088703AE01E4A11791079FFF759FE032052
S113AE001B49887031E00A20FFF70AFE0420184924
S113AE1088702AE0164A1279194B995C144A1279FF
S113AE20154B985CFFF744FE0520114988701CE01F
S113AE300F480079401C0E490871084600795A28C9
S113AE4005DB002008710870C87003E00EE00120E3
S113AE500749C87000200649887006E000200449AC
S113AE6008708870C870087100BF00BF10BD000072
S113AE70D0000020EC21002046220020A022002047
S113AE80FA22002010B510F0AFF8012811D10E48B5
S113AE9000780A2806D1FF22A5320021012011F0F2
S113AEA08DFD0FE04B22D2000021012011F086FD20
S113AEB008E00020054988804880002211460120CE
S113AEC011F07CFD10BD0000200100201C000020BA
S113AED00020034908724870887048607047000079
S113AEE0D00C002058221152704710B5044601219D
S113AEF0022000F071FA0021022000F06DFA10BD6A
S113AF00014600205322525C10231A40002A08D024
S113AF105322525C0C231A409210032A18D10320A6
S113AF2016E05422525A0123DB031A40002A0ED0A1
S113AF305322525C0C231A409210032A05D0532248
S113AF40525C9207920F032A01D1022000E00120F3
S113AF5070470246002058239B5A0B40002B01D017
S113AF60012000E000207047014600226020405A82
S113AF70FF231B0218400005020F1001014BC018EB
S113AF80704700000055044010B5002A0AD056232B
S113AF901B5A0C0223435624235256231B5A8B4319
S113AFA0235209E056231B5A0C02A343562423526E
S113AFB056231B5A0B43235210BD0000F8B5044618
S113AFC00D46012700263448844203D10121022082
S113AFD000F002FA2878401EA0702088FF21013179
S113AFE0084320802088400840002080A878401E24
S113AFF0C1B25A20015568790007000CE9790902A9
S113B0000843A97908435C210853288981B2402068
S113B0100153A868C000C10C42200153A88981B221
S113B02044200153E868C000C10C46200153288A1B
S113B03081B2482001532869C000C10C4A20015341
S113B040A88A81B24C2001536869C000C10C4E200B
S113B05001535020005B2979090208435021085309
S113B0605020005B297988435021085300E0761C66
S113B0705020005B4007400F2979884202D00748DE
S113B0808642F4D15020005B4007400F2979884262
S113B09000D000273846F8BD00540440FFFF0000EC
S113B0A030B5034600201C898C4209DD082A05D2EC
S113B0B018244C431D682C19A05C02E0002000E019
S113B0C0002030BD10B5024613898B4205DD1823DC
S113B0D04B431468E318987C00E0002010BD01463F
S113B0E0FF22C889C007C00F00280AD00120C881E8
S113B0F000E0521EC889C007C00F002801D0002AF2
S113B100F7D1C889C007C00F00280FD10220C88119
S113B1100420C881487A400840004872487A38239D
S113B1209843487200204872012070470020FCE7D1
S113B1300246507A012318435072507A0B78DB0090
S113B14018435072087A012808D1888850814868C9
S113B150000C0123DB031843908108E0087A0028DF
S113B16005D15081486880001A4B18409081487A74
S113B170012804D1507A40231843507206E0487ADB
S113B180002803D1507A402398435072087800284D
S113B19011D1C87A1072087B1070487B5070887B7C
S113B1A09070CB7BD370087C10714B7C5371887C7E
S113B1B09071CB7CD371887A002803D00120C0021F
S113B1C0D08101E00820D081FF200130D08101200E
S113B1D070470000FC1F0000002904D0427A80233D
S113B1E01A43427203E0427A80239A4342727047C0
S113B1F030B5024600200F4B5024A45A0D022C43B4
S113B2005025AC525024A45A8C43AC5200E05B1E2F
S113B2105024A45A6407640F8C4201D0002BF6D149
S113B2205024A45A6407640F002C01D0002000E0CD
S113B230012030BDFFFF0000827A80231A40802A5B
S113B24000D081727047000070B5044600250023C9
S113B250002D02D00126602006530420C88188896D
S113B2600126F6033040002808D001201072888996
S113B270C004C0084E893043506006E000201072BC
S113B28088890F4E304080105060087AD0720023B5
S113B29004E0CE5C10460C30C6545B1CD07A984255
S113B2A0F7DCC88904263040002804D1C889F60296
S113B2B03040002801D0002070BDD07AFCE70000A7
S113B2C0FC1F0000027C80231A40802A00D00174F5
S113B2D0704710B50246FF23D089C007C00F00286D
S113B2E00AD00120D08100E05B1ED089C007C00FC6
S113B2F0002801D0002BF7D1D089C007C00F002847
S113B30001D0002010BD507A012420435072507A9D
S113B3103824A0435072C87A1072487A00280FD19A
S113B320087B1070487B5070887B9070CC7BD47005
S113B330087C10714C7C5471887C9071CC7CD471E5
S113B340FF200130D0814000D081107ADAE700007C
S113B350F8B504460D460020002C00D100BF002A99
S113B36000D100BF012C01D141263043012A01D173
S113B37012263043022C01D1C0263043022A01D1C7
S113B38030263043134E307076788027BE43114FF9
S113B3907E70012C08D1FF2100BF0E4EB3781E46EB
S113B3A00E4033468B42F8D10A4E76784027BE438E
S113B3B0084F7E70012A0BD10026009603E000BFDF
S113B3C0009E761C0096FF276937009EBE42F6D980
S113B3D0F8BD000000040240002905D0054A127897
S113B3E00243044B1A7004E0024A12788243014B70
S113B3F01A70704720040240002905D0054A927E45
S113B4000243044B9A7604E0024A927E8243014B43
S113B4109A7670470008024001200649087000BF70
S113B42004480078802108400028F9D0012002490E
S113B43008707047000C0240A401002070B5034658
S113B44014460020002B01D1C0B202E0054680352D
S113B450E8B2012902D1051DE8B206E0022903D1B0
S113B46005460835E8B200E0C0B2012C02D1851CC3
S113B470E8B200E0C0B2084DA870AD7801263543AB
S113B480054EB570002201E000BF521C7D252D0140
S113B490AA42F9D970BD0000000C024070B5002426
S113B4A02448007920210840002801D0224D3FE0A3
S113B4B000F046F80546214800788021084000281D
S113B4C036D01E4880780840002801D01A4D02E08A
S113B4D000F036F80546194880780007840F022CDE
S113B4E001DBAD0804E0012C01D16D0800E000BFD0
S113B4F0124880788007C00F002801D02D0101E098
S113B5000C2045430D4800784007840F002C02D1DD
S113B510601CC4B207E0032C03D1601C4006040E77
S113B52001E06006040E21462846FCF709FE0546A4
S113B530284670BD0004024000127A00000C02404C
S113B54000B5C0229178F82211401C4A12781143A8
S113B550EA2923D00ADC0A46E03A130012F076FF07
S113B5600A181C20242A2A2A2A161A2AED291FD04E
S113B57004DCEB2916D0EC291CD117E0F02903D008
S113B580F82917D10E4817E00E4815E00E4813E0CD
S113B5900E4811E00E480FE00E480DE00E480BE097
S113B5A00E4809E00E4807E00E4805E00E4803E0A7
S113B5B00E4801E00D4800BF00BF00BD201C024042
S113B5C00090D003006CDC020048E80100366E01F4
S113B5D00024F400001BB70000127A00808D5B0089
S113B5E000093D00C0C62D0080841E0040420F00AB
S113B5F010B50446204600F05FFD002010BD000099
S113B60010B590211348FCF74BFE1248124908600C
S113B61012484860062008810020887206220F49DB
S113B6200D4800F04BFA00210B48FFF705FE80217E
S113B6300B48FCF735FE0A480A4948600A4B0422C5
S113B6400A49084800F0CBFB55210648FFF73AFEAB
S113B65010BD0000480800202808002030F2010036
S113B660D808002034080020F1B50000C0F1010022
S113B6700C4A127812060B4B5B781B041A43094BD5
S113B6809B781B021A43074BDB781A431046420887
S113B6904240D20083085A401146034A5140034AAB
S113B6A0116070471B0700200102000020070020E2
S113B6B0F8B504460F46A07A4006400E002874D11F
S113B6C00025ACE01820684321680818407C012854
S113B6D03CD1012118206843226810180174002607
S113B6E00CE018206843216808180830815D182090
S113B6F06843226810188155701CC6B2082EF0D316
S113B7000021182068432268101801741820684327
S113B7102268101841741820684322681018416187
S113B720182068432268101881742C2068436168CB
S113B7300818406A002809D018236B432268D018DF
S113B7402C236B436268D218516A884718206843D7
S113B750216808184069FF21C94388425DD8182030
S113B7606843216808184069C11918206843226891
S113B77010184161182068432168081841692C2079
S113B7806843626810188069814246D31820684370
S113B79021680818807C55283FD05521182068431B
S113B7A0226810188174002624E03CE018206843C5
S113B7B021680818805D2C21694362685118103192
S113B7C0895D08401821694322685118885518205A
S113B7D0684321680818805D2C2169436268511808
S113B7E00831895D08431821694322685118885536
S113B7F0701CC6B2082ED9D32C206843616808187F
S113B800806A002809D018236B432268D0182C239F
S113B8106B436268D218916A8847681C85B2208994
S113B820A84200DD4EE7F8BD10B50446002013F031
S113B83071F9022841D121480078002802D1012061
S113B8401E4908701D48007801281FD11B48407804
S113B850401C1A49487021465A20FCF771FC1749CC
S113B8604978884229D800201449487008468078CD
S113B870401C8870084680780A2803D3002088700A
S113B88002200870002013F075F916E00B480078C8
S113B890022812D109484078401C084948702146C2
S113B8A07D20C000FCF74CFC04494978884204D848
S113B8B000200249487013F05DF910BD78000020A3
S113B8C000B587B0002168460171042141710C481C
S113B8D00290411003910B49049105910A48069086
S113B8E0FFF78EFE01A813F0A9F900F02FFB00F07A
S113B8F00FF80021054809F0A7F907B000BD0000C2
S113B900FFFF1F00FFFFFF1F45BB000002050000F3
S113B91010B5FF20023065494860002008720120FC
S113B920087000204872012088726148FFF7D7FB35
S113B9305E495F48FFF7FCFB01215D48FFF74CFCC3
S113B9405C485A49486000200872012008700020B1
S113B95048720120887256481030FFF7C0FB5349E3
S113B96053481030FFF7E4FB012151481030FFF732
S113B97033FC5048401E4D494860002008720120A5
S113B9800870002048720120887249485030FFF73F
S113B990A6FB464946485030FFF7CAFB01214448FC
S113B9A05030FFF719FC4348C13840494860002033
S113B9B008720120087000204872012088723C48F7
S113B9C04030FFF78CFB394939484030FFF7B0FB72
S113B9D0012137484030FFF7FFFBFF201230334985
S113B9E0486000200872012008700020487201207D
S113B9F088722F486030FFF772FB2C492C48603066
S113BA00FFF796FB01212A486030FFF7E5FBFF2092
S113BA102130264948600020087201200870002067
S113BA204872012088722248A030FFF758FB1F4952
S113BA301F48A030FFF77CFB01211D48A030FFF711
S113BA40CBFB3F20400119494860002008720120C7
S113BA500870002048720120887215482030FFF7D2
S113BA603EFB124912482030FFF762FB01211048C7
S113BA702030FFF7B1FB10480C49486000200872E1
S113BA800120087000204872012088720848303074
S113BA90FFF725FB054906483030FFF749FB012134
S113BAA003483030FFF798FB10BD0000E425002068
S113BAB01055044002040000DF070000F0B50B46F7
S113BAC0144643600481002136E0002216E02C2550
S113BAD04D4346687519AD5C18274F430668F6193F
S113BAE0B5542C254D4346687519AD5C18274F4352
S113BAF00668F6190836B554551CEAB2082AE6D386
S113BB00002518274F430668F619357418274F4344
S113BB100668F619757418274F430668F619B57444
S113BB2018274F430668F619F57418274F4306681B
S113BB30F61975614D1CA9B205898D42C5DC002535
S113BB408572F0BD70B50446606800F01FFE0546BE
S113BB50E27A23460C332946094800F0DFFD0949FF
S113BB606068884203D0491C6068884206D1E17A43
S113BB70A28890B222460C3202F070FD70BD000023
S113BB8028080020DF070000F8B5054600262C46EB
S113BB90002C07D000BF03E0FF20A055701CC6B2E4
S113BBA0082EF9D304F08CFCC00008210840074695
S113BBB02068884338432060F8BDF8B50546002660
S113BBC02C46002C07D000BF03E0FF20A055701CBA
S113BBD0C6B2082EF9D304F0EBFC07122088000A41
S113BBE000023843208004F0E3FC0002FF21090234
S113BBF008400746208888433843208004F0CEFD5F
S113BC0007126088000A00023843608004F0C6FD11
S113BC100002FF2109020840074660888843384330
S113BC206080F8BDFEB5054600260020019001F0B5
S113BC301FFD0A210090FCF783FA074604F074FC08
S113BC400A210090FCF792FA80B201902C46002C55
S113BC5007D000BF03E0FF20A055701CC6B2082E19
S113BC60F9D30721090620688843019909120906B6
S113BC70072212061140084320606068000A00028F
S113BC800199C9B208436060FF21090260688843D2
S113BC90390C0902FF2212021140084360601102AC
S113BCA060688843390A090412021140084360603D
S113BCB060680002000A3906090E0906084360603C
S113BCC004F0F2FBC007C00FC007009020684000DA
S113BCD0400800990843206003F096FE0007000F17
S113BCE0009020680009000100990843206003F0D7
S113BCF085FE022806D101210907206888434018DF
S113BD00206004E00121090720688843206004F0D2
S113BD1091FB0001F02108400090206888430099BD
S113BD200843206004F05AFCFF2806DDFF210904C3
S113BD3020688843401820600BE004F04FFC0004A6
S113BD40FF210904084000902068884300990843B3
S113BD502060FEBDFEB505460026002001900027A8
S113BD6004F00EFA64210090FCF700FA80B201900E
S113BD70002001F08FFC87B22C46002C07D000BFB6
S113BD8003E0FF20A055701CC6B2082EF9D320682A
S113BD90000A00020199C9B208432060FF21090486
S113BDA02068884339120904FF2212041140084311
S113BDB0206020680002000A3906090E09060843BB
S113BDC0206003F027FE28300002FF21090208400A
S113BDD0009020688843009908432060FEBDFFB5A9
S113BDE081B004460F4600250026002000902760FD
S113BDF0039820810498E0600020207400BF9DE037
S113BE001C206843216808586A01616888501C2016
S113BE1068432168081880686A0161688918486065
S113BE201C2068432168081840686A016168891801
S113BE3088601C20684321680818C0686A0161682A
S113BE408918C8601C20684321680818007C6A01AE
S113BE506168891808741C20684321680818407CAC
S113BE606A016168891848741C20684321680818AD
S113BE70807C6A016168891888831C206843216872
S113BE800818C07C6A0161688918887400206A01F6
S113BE9061688918C8741C206843216808184068C0
S113BEA0002813D01C20684321680818C07C00288F
S113BEB005D1401E6A0161688918C8831AE0002010
S113BEC0C0436A0161688918C88313E01C20684371
S113BED021680818C07C002805D000206A01616828
S113BEE08918C88306E000206A0161688918C8833C
S113BEF001200090002607E000216A016068801894
S113BF0014308155701CC6B2690160684018808B7A
S113BF10B042F1DC1C2068432168081840690028FD
S113BF200AD06B016268D218104614301C236B438C
S113BF302268D21851698847681CC5B22089A84272
S113BF4000DD5DE7009805B0F0BD000000B58BB0E2
S113BF5056480790002108A801706846017608A891
S113BF604170002052498872082108A8C17000203D
S113BF7004E0002209A90A54411CC8B208A9C978DE
S113BF808142F6DC4B48FFF7AAF806A94948FFF7B7
S113BF90CFF84648401C0790002108A80170684665
S113BFA0017608A84170002041498872082108A838
S113BFB0C170002004E0002209A90A54411CC8B23F
S113BFC008A9C9788142F6DC3A484030FFF787F87F
S113BFD006A938484030FFF7ABF845200001079028
S113BFE0002108A801706846017608A84170002065
S113BFF02F498872082108A8C170002004E000229B
S113C00009A90A54411CC8B208A9C9788142F6DCBE
S113C01028485030FFF763F806A926485030FFF748
S113C02087F8112040010790002108A80170684694
S113C030017608A8417000201D498872082108A8CB
S113C040C170002004E0002209A90A54411CC8B2AE
S113C05008A9C9788142F6DC16482030FFF73FF87A
S113C06006A914482030FFF763F8FD20C0000290B1
S113C0700021684601730171417381730821C17302
S113C080002004E0002204A90A54411CC8B26946F5
S113C090C97B8142F6DC07481030FFF720F801A97C
S113C0A004481030FFF744F80BB000BDEE06000062
S113C0B0E42500208055044030B585B004460025B1
S113C0C020680190A1796846C172617941720021AA
S113C0D00172017000BF05E020460830415D03A8ED
S113C0E041556D1C6846C07AA842F5D81121490112
S113C0F00198401A1BD023210901401A11D011497B
S113C1004018002802D0012817D104E069460E48DF
S113C110FFF7DFF812E069460B484030FFF7D9F823
S113C1200CE0694608485030FFF7D3F806E069464A
S113C13005482030FFF7CDF800E000BF00BF05B090
S113C14030BD000062FDFFFF80550440F0B585B0AE
S113C15004460F4600250026207C4006400E552844
S113C1607ED100BF76E1690160684018807C0028B8
S113C17077D169016068401840686A01616889186C
S113C1808968884209D26901606840184068C0190A
S113C1906A016168891848605AE169016068401859
S113C1A0C068AF49884208D8690160684018C0680F
S113C1B0401C6A0161688918C86069016068401898
S113C1C0C07C002821D1002607E000216A016068B4
S113C1D0801814308155701CC6B26901606840181B
S113C1E0808BB042F1DC1C20684321680818406948
S113C1F000280AD06B016268D218104614301C2340
S113C2006B432268D21851698847690160684058B5
S113C2100090690160684018017C68460171002142
S113C2204171690160684018017F68468171690144
S113C23060684018417C6846C171002608E06901C5
S113C240606840181430815D02A88155701CC6B224
S113C250690160684018808BB042F0DCE06801E05E
S113C260FCE01DE0002806D06846E16888476A01C2
S113C27061688918C874690160684018C07C002826
S113C28004D16A01616889184860E1E06901606865
S113C29040184068C01B6A01616889184860D7E08B
S113C2A069016068401880680028EED06901606800
S113C2B04018C08B0028E8D0690160684018C08B22
S113C2C06A0161688918C968884207D16901606890
S113C2D04018C08B6249C94388427DD169016068B6
S113C2E0401840686A01616889188968884209D2DF
S113C2F06901606840184068C0196A01616889185A
S113C3004860A5E000206A016168891848606901F5
S113C31060684018C0685249884208D8690160685A
S113C3204018C068401C6A0161688918C86000260A
S113C33007E000216A016068801814308155701C80
S113C340C6B2690160684018808BB042F1DC1C20E1
S113C350684321680818406900280AD06B016268A4
S113C360D218104614301C236B432268D21851692A
S113C3708847690160684058009069016068401806
S113C380017C6846017100214171690160684018AF
S113C390017F68468171690160684018417C684684
S113C3A0C171002608E06901606840181430815D9D
S113C3B002A88155701CC6B2690160684018808B60
S113C3C0B042F0DCE068002808D06846E16888479D
S113C3D06A016168891800E015E0C8746901606841
S113C3E04018C07C002804D16A016168891848603B
S113C3F02EE06901606840184068C01B6A016168EA
S113C4008918486024E01C206843216808184068A3
S113C41000280FD00020C0436A0161688918C883CE
S113C4201C2068432168081840686A0161688918FB
S113C430886008E000206A0161688918C8836A017D
S113C44061688918886000206A0161688918C86079
S113C450681CC5B22089A84200DD84E605B0F0BDA1
S113C4600000FFFF7CB500BF19212C480078FBF7C2
S113C47067FE04462A4860432A4A811800220120A4
S113C4800BF0A2FD20460A2250436430001981B209
S113C490002201200DF064FB01200A2262431219DC
S113C4A0D1B20A22624312190090D0B201231A4673
S113C4B008F0D2FEBA220721002006F0F7FB012083
S113C4C0009001900B20604382B20B20604381B244
S113C4D0002301200CF07CFE6F20604381B2012018
S113C4E00DF0E4FD104860430246032101200AF0E8
S113C4F06DFC002505E0012128460AF0A1FB681C1B
S113C500C5B20F2DF7DB21460B2251436431C8B26B
S113C5100EF030F80EF018F87CBD00007300002017
S113C520672B0000A0860100FCB101000020054932
S113C53008700549087005490870054908700549DF
S113C54008707047740000207500002073000020FC
S113C5507200002071000020F0B589B000BF00BF58
S113C56000BF00BF00BF00BF00BF00BF00BF00BFCF
S113C57003215C480078FBF7F9FD5B4948430290CE
S113C58003210120029A0AF021FC05215548007874
S113C590FBF7D6FD0446E1B201200AF0DFF90321DE
S113C5A050480078FBF7E2FD0B214843643080B229
S113C5B00690E1B201231846069A09F027F9494981
S113C5C009788A0088180621FBF7D0FDFF21F53190
S113C5D0484380B207900798FBF7C8FDC7B23946B5
S113C5E0012009F0F7FD03213E480078FBF7BEFD6A
S113C5F00B214843643080B208900022012008993E
S113C6000DF0AEFA032137480078FBF7AFFD374948
S113C61048433749401803900022012003990BF046
S113C620D3FC03212F480078FBF7A0FD0B214843DE
S113C63080B2049003212B480078FBF797FD0B216F
S113C640484386B20120F1B20090049AD0B201238B
S113C6501A4608F001FEBA220721002006F026FB44
S113C660032120480078FBF781FD0B21484385B264
S113C6700120009000232A46294601900CF0A8FDD1
S113C680032118480078FBF771FD6F21484380B2FD
S113C6900590012005990DF009FD164800783C2805
S113C6A005DA14480078401C1249087002E03C2066
S113C6B0104908700F4800781D2805DC09480078E7
S113C6C0401C084908700BE006480078002802D195
S113C6D00449087004E003480078401E01490870CA
S113C6E009B0F0BD74000020FCB10100672B00000C
S113C6F0A086010075000020002000BF06E0002194
S113C700044A1154044A1154411CC8B25A28F6DB95
S113C71070470000EC210020A0220020FFB581B06A
S113C72004460F463D462089A8422DDD1820684363
S113C73021680818007C002826D1002609E0049806
S113C740815D182068432268101808308155701CD8
S113C750C6B2082EF3D301211820684322681018AA
S113C76041742C20684361680818006A00280BD0C3
S113C77018236B432268D218104608302C236B43CD
S113C7806268D218116A884705B0F0BD01460620D8
S113C790104BCA1A99420FD008DCCA1FFA3A002A71
S113C7A012D0102A0AD01F2A10D10BE0C02A07D0B9
S113C7B0C12A0BD100200BE0012009E0022007E090
S113C7C0032005E0042003E0052001E0062000BF6B
S113C7D000BF70474103000010B504467D21C90025
S113C7E061430846322103F06DFC10BD0148006826
S113C7F070470000500000200148006870470000A6
S113C8004C00002010B505490988652251430846AB
S113C8106421FBF7ABFC80B210BD00005A0000207D
S113C82001480078704700005F000020014800784C
S113C830704700005800002010B50EF0D5FB012809
S113C8402CD100F063F8012000F066F803F09EFCA0
S113C850044600F043F803F045FE044600F04AF8AD
S113C86003F0CEFF012805D100F03EF8012000F0CE
S113C87047F805E0002000F037F8002000F040F809
S113C88000201349086013480068134988421ED2E7
S113C89010480068801C0F49086018E000200D490A
S113C8A008600B4800680C49884204D208480068B4
S113C8B0801C07490860002000F028F8012000F0DF
S113C8C02BF8002000F00AF8002000F013F810BD47
S113C8D0500000204C000020FFFFFF7F014908802A
S113C8E0704700005A00002001490870704700009A
S113C8F05F00002001490880704700005C000020B0
S113C9000149087070470000600000200149087068
S113C910704700005800002001490870704700006B
S113C9205E0000200021014A117170470060004040
S113C930002201494A757047006000400022014905
S113C9404A767047006000400021014A1172704726
S113C950006000400021014A1173704700600040EC
S113C9600021014A11747047006000400021014A0F
S113C97011757047006000400021014A117670472C
S113C98000600040002201494A7370470060004083
S113C990002201494A7470470060004010B51C4CE5
S113C9A01C49206888421ED106221B49201DFBF722
S113C9B082FC002817D10D22184920460A30FBF7C3
S113C9C07AFC00280FD10622154920461730FBF7C0
S113C9D072FC002807D10622124920461D30FBF7BD
S113C9E06AFC00280DD000F079FE0A480E49086060
S113C9F0074812F0F0F90C4A2421054812F016FAFF
S113CA0004E0242221460848FBF731FC10BD000055
S113CA10000250007AA7A55A3107002037070020EA
S113CA202B07002025070020B82A002000200849F1
S113CA300870084908700120074908700020074958
S113CA4008700748074908600020074908707047C4
S113CA501307002012070020150700201A070020E2
S113CA6025060000440700202407002070B5054671
S113CA7000BF9120684304460A212046FBF760FB6F
S113CA800446641D204670BD70B5A8B00546002458
S113CA900026A0216846FBF703FC00F09FFC1E491A
S113CAA00A6814216943505000211B48026814206D
S113CAB0684310184160184802681420684310182D
S113CAC0816015484068002824D000BF17E0600644
S113CAD0060E282E00D316E00F4801681420604388
S113CAE00858B1006A4650500B480168142060434E
S113CAF008184168701C80001150601CC4B20648BC
S113CB00007AA042E3DC00BF620003486946436840
S113CB100220984728B070BD082B002030B5A9B07A
S113CB2000240025A02101A8FBF7BAFB00BF25E0E3
S113CB306006050E00F052FC1F490A681421614387
S113CB40505000211C4802681420604310184160B2
S113CB50194802681420604310188160282D0BD2F4
S113CB6015480168142060430858A90001AA5050D0
S113CB700021681C80001150601CC4B20E48007A69
S113CB80A042D5DC0C484068002813D00A48007A3B
S113CB904000282806D30848282201A94368022017
S113CBA0984707E00448007A4200034801A9436813
S113CBB00220984729B030BD082B002010B50EF094
S113CBC013FA01287ED1FFF717FE5549884216D281
S113CBD00F2054494871887108468078002801D193
S113CBE0052048704F488078052802D100204D491F
S113CBF0487000204B4908724872087035E0FA20EA
S113CC004849487188714849088803F095FB4648AB
S113CC10807800280CD14349087008464079C870D0
S113CC2008468079087100208870487048721CE0BA
S113CC3001203C4908700846407A022805D10120A9
S113CC4048720020C87008710FE03648407A002806
S113CC500BD1022033494872084640788870084650
S113CC604079C8700846807908712E4880782D492B
S113CC704978884213DD00202A49C87008460079A3
S113CC80401C0871084600798979884222DB00201B
S113CC902449087108468078401E88701AE02148AB
S113CCA0807820494978884214DA00201D490871A7
S113CCB00846C078401CC8700846C0784979884244
S113CCC008DB00E01EE000201649C87008468078A2
S113CCD0401C887014488078002803D10120114931
S113CCE008721BE010480088732803DB02200D49FA
S113CCF0087213E00C48008870280FDC00200949F2
S113CD0008720BE000200749087008464079C87093
S113CD1008468079087100200872487210BD00002E
S113CD20B80B0000580900207C00002000200449B2
S113CD3088704870C87008710872487270470000A3
S113CD405809002000200649088088700549887029
S113CD504870FA20C8700871002008724872704741
S113CD607C0000205809002070B503F03FFA044607
S113CD7003F04EFA05460EF037F901282ED10521AD
S113CD801A48FEF79FF9552804D1002018498870E5
S113CD90088027E0012D04D10020154988700880FF
S113CDA020E00120124988701248844202DB201AD4
S113CDB084B200E000240A212046FBF7D7F90529B4
S113CDC001DB601D84B20C48844200DD04460A2164
S113CDD02046FBF7CBF90649088003E0002004490C
S113CDE088700880FFF7EAFE70BD00002808002064
S113CDF07C000020AA0A0000C60700001CB5002021
S113CE000090019000F0EAFA0B49086000200B49F9
S113CE10096808600A48006800280CD007490968B6
S113CE2008680A21FBF78CF9009001226946052065
S113CE30034B1B6898471CBDE0070020D407002063
S113CE40DC07002000200849488008490880084978
S113CE500880084908700849887208490880488091
S113CE6001200871704700003400002024000020D5
S113CE7026000020280000200C0800202C000020A0
S113CE80F8B503F095F9074603F0A4F90090FFF70D
S113CE90CDFC012860D10521C548FEF713F95528BA
S113CEA002D00098012807D10020C2490870C24965
S113CEB00880C249887256E0BE480078002810D124
S113CEC00120BC4908703D462846E917890F091816
S113CED089030D0CBA48854200DD0546B648058035
S113CEE041E0B648807A4000B4490F520846867A39
S113CEF00EE07000B1490D5A701E4000085A7100CE
S113CF00AE4A5052701E400011460D52701EC6B2F9
S113CF10002E08DD7000A949095A701E4000A74A76
S113CF20105A8142E5DBA548807A401CA3498872E7
S113CF300846807A052816DB002088720846C588D2
S113CF402846E917890F09188D109D48854200DD90
S113CF5005469948058006E00020964908709649E0
S113CF600880964988729448058896480088A842A3
S113CF7057DA94480088281A84B292480079012824
S113CF8027D190484088A0420BDA8E4840880A3066
S113CF908C49488008464088A04204DD0846448005
S113CFA001E088484480874844882046E117890F77
S113CFB009188C100A2C00DA0A2482480088001907
S113CFC08049088008460088A84201DD084605809B
S113CFD0CDE07C484088142805DD7A484088143820
S113CFE07849488002E000207649488075484488A2
S113CFF02046E117890F09188C100A2C03DA012046
S113D00070490871B3E06F480088A04205DD6D489F
S113D0100088001B6B490880A9E00020694908804A
S113D020A5E068480088A84259DD66480088401B8E
S113D03084B264480079012827D1624840881428C2
S113D04005DD6048408814385E49488002E00020CD
S113D0505C4948805B4844882046E117890F0918D9
S113D0608C100A2C03DA0220564908717FE05548D7
S113D07000880019534908800846008850498842AE
S113D08075DD08464F49088071E04E484088A0424B
S113D0900BDA4C4840880A304A49488008464088A0
S113D0A0A04204DD0846448001E0464844804548E7
S113D0B044882046E117890F09188C100A2C00DADD
S113D0C00A24404800882919884202DA3D4805802C
S113D0D04DE03C480088001B3A49088047E0394845
S113D0E044882046E117890F09188C100A2C3EDD6C
S113D0F034484088142805DD3248408814383149C2
S113D100488002E000202F4948802E484488204669
S113D110E117890F09188C102A480079012813D1C6
S113D1200A2C03DA02202749087120E025480088E8
S113D130001924490880084600882149884216DDE0
S113D14008462049088012E00A2C03DA01201D4910
S113D15008710CE01B480088A04205DD19480088CE
S113D160001B1849088002E0002016490880164870
S113D1700088502804DC134800881349088016E00E
S113D1801048008810490988884204DD0D48008849
S113D1900D4908800BE00B4800880B490988081AE0
S113D1A084B2502C03DB0748008807490880F8BD87
S113D1B02808002028000020240000200C0800205B
S113D1C0E02E00002C0000202600002010B50446AC
S113D1D064204443A1212046FAF7B2FF04462046C6
S113D1E010BD00007CB5002400200190009000F0E8
S113D1F03FFA05460A21FAF7A3FF044601226946CD
S113D200042000F06DFC0098401C002814D17D20FF
S113D210C0002018114908600846006801900122E6
S113D22001A9032000F09AFC012000900122694624
S113D230042000F093FC0FE0009801280CD17D201D
S113D2400001201805490860084600680190012281
S113D25001A9032000F082FC7CBD0000280100200D
S113D26010B501200F49087000200F4909680860B3
S113D2700D49096848600C490968886000F07EF926
S113D280FFF7BCFDFFF74AFC08480068002807D0F8
S113D29001220548016808310020044B1B689847A7
S113D2A010BD0000AD070020A8070020A40700203F
S113D2B010B5184800681849884229D117480068F1
S113D2C0002804D01548006880471549087015489F
S113D2D00068002804D01348006880471249087089
S113D2E012480068002804D010480068804710499C
S113D2F0088010480068002805D00E480068804760
S113D3000D49088002E00D480B49088000F078F8C8
S113D31010BD0000B807002078563412940700208E
S113D320AC07002098070020AE0700209C070020CF
S113D330B0070020A0070020B2070020102700003B
S113D34010B50023174C2360174C2370174C23701F
S113D350174C2370174C2380174C2380174C2370D1
S113D360174C13682360174C53682360164C93685A
S113D3702360164CD3682360154C1369236000287E
S113D3800CD0144B1860134C0B682468A360002362
S113D390104C246823600F4C246863600E4B014CCE
S113D3A0236010BDB8070020B4070020AC0700209C
S113D3B0AE070020B0070020B2070020AD07002010
S113D3C094070020980700209C070020A007002055
S113D3D0A4070020A80700207856341205480068E6
S113D3E00549884203D105480068806870470020D9
S113D3F0C043FBE7B807002078563412A807002082
S113D40070B50024002500263048007801285CD13E
S113D4102F480078002858D12E480078012854D18C
S113D4202D4805882D490988694308462C49FAF78F
S113D43087FE85B2E1200001854207D8192169439E
S113D44008460921FAF77CFE044600E0244C2548EE
S113D45000680068001923490968086021480068C9
S113D4600068204909684968884207D31D48006854
S113D47000681C4909684968461A0AE019480068A6
S113D48040680021C943081A164909680968401808
S113D490461C1548864218D3344601462046FAF7FE
S113D4A04FFE04460F48006841680F48604308185F
S113D4B00C490968486001200C4908700948006853
S113D4C08068001907490968886070BDAC070020AE
S113D4D0AD070020AE070020B0070020B2070020EF
S113D4E010270000A8070020A0860100B407002030
S113D4F000220C4B1A600C4B0A681A600B4B4A68EA
S113D5001A600B4B8A681A600A4BCA681A600A4B85
S113D5100A691A60002801D0084A1060084A014BC1
S113D5201A607047B807002094070020980700206D
S113D5309C070020A0070020A4070020A8070020C3
S113D5407856341210B50A48006800280ED00948ED
S113D550007801280AD100200649087001220648F3
S113D560016808310020024B1B68984710BD000079
S113D570A4070020B4070020A80700201CB5002041
S113D580009001900024FFF729FF04460E4800682C
S113D590046000200C49096848600B4909688860E8
S113D5A00A48006800280DD0074800680068009009
S113D5B00548006840680190022269460120034B37
S113D5C01B6898471CBD0000BC070020C007002052
S113D5D0F8B505460C4616460027002D17D00E4810
S113D5E00560FFF7FBFE07462068B84203D90A48E6
S113D5F00068076003E00849206809680860064974
S113D6006068096848600449A0680968C8600348FC
S113D610066000F005F8F8BDBC070020C007002034
S113D62070B500240025FFF7D9FE04460F480068B2
S113D6300068A04200D903E00C4800680068251A7D
S113D6400A48006840684019084909688860074822
S113D6500068806805490968C968884205D9034893
S113D6600068C06801490968886070BDBC07002073
S113D6700148006880687047BC070020002801D07A
S113D680024A1060024A116070470000BC07002083
S113D690C0070020014610480268142048431018AF
S113D6A082680D480368142048431818C0688242F1
S113D6B00BD909480268142048431018C268064868
S113D6C00368142048431818826003480268142031
S113D6D04843101880687047082B0020002005E09C
S113D6E019490A5C19490A54411CC8B20628F7DBD7
S113D6F0002006E016490A5C1449891D0A54411C9D
S113D700C8B20D28F6DB002006E012490A5C0F4976
S113D71013310A54411CC8B20628F6DB002006E087
S113D7200D490A5C094919310A54411CC8B206283A
S113D730F6DB002005E0002204491F310A54411C95
S113D740C8B20128F7DB704731070020BC2A00204B
S113D750370700202B0700202507002010B50020E4
S113D76005490860486008724872887202F0AEFE8B
S113D7700149C87210BD00006409002070B500247E
S113D780002502F0A3FE6549C87202F085FD044637
S113D79002F08CFD0546FFF749F8012874D10121F8
S113D7A05F48FDF78FFC552807D100205B490872BC
S113D7B04872086048608872AFE0FF2C01D0FF2DEA
S113D7C063D1FF2C2AD1FF2D28D0002053490872A1
S113D7D00120487253480860FF20143068434860B1
S113D7E048686621FAF7ACFC4C4948600846406832
S113D7F04C49884202D9084648494860474840682D
S113D800AA2803D345484068FA2803D9012043498C
S113D810887282E00020414988727EE0FF2C2AD081
S113D820FF2D28D101203D490872002048723D484F
S113D8304860FF2014306043086008686621FAF7E6
S113D8407FFC36490860084600683649884202D998
S113D85008463249086031480068AA2803D32F4893
S113D8600068E62803D901202C49887255E000207D
S113D8702A49887251E02B482849086048600020F2
S113D88088720872487248E040E001202349087217
S113D8904872FF2014306043086008686621FAF774
S113D8A04FFC1E490860084600681E49884202D998
S113D8B008461A490860FF20143068431749486035
S113D8C048686621FAF73CFC1449486008464068F9
S113D8D01449884202D90846104948600F48006834
S113D8E0AA280BD30D480068E62807D80B484068DF
S113D8F0AA2803D309484068FA2803D90120074914
S113D90088720AE000200549887206E00020034975
S113D9100872487208604860887270BD640900200B
S113D92028080020DE030000FFB583B006460D463C
S113D930174600240020029000BF14207843801969
S113D9400190002E57D00198002854D02B4806602F
S113D9502A49069848600846077200BF45E0FFF769
S113D9603DFD0290200129580298814204D82001EB
S113D9702858401C002806D1204902980A6814211E
S113D9806143505006E0200129581C4802681420C5
S113D99060431150200140194068401C002807D101
S113D9A0002116480268142060431018416008E002
S113D9B0200140194168114802681420604310187E
S113D9C041602001401981680C48026814206043BA
S113D9D01018C16020014019017B08480268142016
S113D9E0604310180161601CC4B20448007AA0426C
S113D9F0B5DC00F005F807B0F0BD0000082B0020EE
S113DA0070B5002400250026FFF7E8FC054600BF9A
S113DA104EE02A480168142060430858A84239D8C7
S113DA20264801681420604308582E1A23480168C8
S113DA3014206043081840688119204802681420A3
S113DA406043101881601D48016814206043081861
S113DA5081681A480268142060431018C068814223
S113DA6024D9164801681420604308180069002866
S113DA7003D02046FFF708F818E010480168142086
S113DA8060430818C1680D480268142060431018E8
S113DA9081600BE00948016814206043081840685D
S113DAA006490A681421614351188860601CC4B295
S113DAB00248007AA042ACDC70BD0000082B0020B4
S113DAC010B500BF14244C432318002805D0002BA4
S113DAD003D0024C20606260217210BD082B00202C
S113DAE0F8B505460E4614462B0010F0AFFC0504AD
S113DAF0121920272E001748FBF730F81649087032
S113DB001448FAF7E5FB07466421FAF719FB30607D
S113DB101CE0A004020C31461020FBF719F915E0B3
S113DB20A004020C31463020FBF712F90EE0A004E9
S113DB30020C31465020FBF70BF907E0A004020C5D
S113DB4031467020FBF704F900E000BF00BF00205D
S113DB50F8BD0000CE230020D900002070B5054692
S113DB600E4614462B0010F071FC05041C232A31C8
S113DB7038003068002802D1FAF78EFE10E06422E3
S113DB803168514308461649FAF7ACFB00201549A1
S113DB900870012264211248FBF748F91149087002
S113DBA01CE0A004020C31461020FBF78FFA15E0AC
S113DBB0A004020C31463020FBF788FA0EE0A004E2
S113DBC0020C31465020FBF781FA07E0A004020C56
S113DBD031467020FBF77AFA00E000BF00BF70BD49
S113DBE0C0230020D800002000B5AFB050211BA8EE
S113DBF0FAF756FB00201A90142115A8FAF750FBE7
S113DC0000201290139014901190402101A8FAF76B
S113DC1047FB00203F49086001221BA9FFF760FF72
S113DC201B98401C002801D11A9001E01B981A90FF
S113DC3039481590394816903948179000201890A3
S113DC403848199015AA1AA93748FFF779FB022218
S113DC501CA90120FFF744FF1C98401C002801D197
S113DC60129001E01C9812901C98401C002801D1CD
S113DC70139001E01D9813902C48149012A92C487D
S113DC80199AFFF7A5FC08221EA90220FFF728FF16
S113DC901E98401C002801D1019001E01E980190BB
S113DCA01F98029023480390012069460874801E3F
S113DCB0059021490791012101A80177881E099047
S113DCC01D490B91012109A80173881E0D901A4961
S113DCD00F9101210DA80173042201A91748199B72
S113DCE0FFF722FE01221BA90320FFF7F9FE1449C6
S113DCF01B9808601B98401C002806D1FF20F530B3
S113DD00086001220320FFF729FF0E48014908603B
S113DD102FB000BDDC0000202DC8000021C8000089
S113DD2005C800005DDB00005423002076841E003B
S113DD30602300200F2700009F860100702300202D
S113DD4028010020A33AA55A00B585B014216846DD
S113DD50FAF7A6FA00200F4908600F4800900F4810
S113DD6001900F480290002003900E4804906946E9
S113DD700D48FFF7BDFB0D480499FFF77FFC042114
S113DD800B48049AFFF79CFE0A480249086005B054
S113DD9000BD0000DC0000202DC8000021C80000E8
S113DDA005C800005DDB0000542300206023002030
S113DDB070230020A33AA55A00200B4908800B4980
S113DDC008800B49088001200A49087000200A498C
S113DDD008730A4908804880012008710020064918
S113DDE048800880704700003C0000203E0000206E
S113DDF040000020420000201808002044000020B9
S113DE00FEB502F00FFA009002F016FA0190FEF748
S113DE100DFD01286BD10521D448FDF753F9552890
S113DE2007D10020D2490870D2490880D24988809D
S113DE3067E00198012807D10020CD490870CD4939
S113DE400880CD4988805CE0C9480078002808D162
S113DE500120C7490870009D0A206843C54908800D
S113DE604FE0009881B2C448007B4200C248801D44
S113DE708152801F067B11E07100BF48801D455A06
S113DE80701E4100BC48801D415A72008152701EB0
S113DE904100B948801D4552701EC6B2002E0ADDED
S113DEA07100B548801D415A701E4200B248801D61
S113DEB0805A8142E0DBB048007B401CAE490873C5
S113DEC00846007B032807DB002008730846058901
S113DED00A206843A74908800020A7490880488091
S113DEE0A448008888800120A149087009E0002026
S113DEF09F4908709F4908809F490880488008739B
S113DF0088809C4805889D480088A84256D29B4832
S113DF100088281A84B299480079012826D19748A4
S113DF204088A0420BDA95484088801C9349488079
S113DF3008464088A04204DD0846448001E08F483A
S113DF4044808E48448803212046FAF70FF984B2AE
S113DF50022C00DA022489480088001987490880C5
S113DF6008460088A84200D90D80CDE08348408847
S113DF70062805DD81484088801F8049488002E0EA
S113DF8000207E4948807D48448803212046FAF7D2
S113DF90EDF884B2022C03DA012078490871B3E069
S113DFA076480088A04205DD74480088001B734948
S113DFB00880A9E0002071490880A5E06F48008826
S113DFC0A84259D96D480088401B84B26B48007937
S113DFD0012827D169484088062805DD674840881C
S113DFE0801F6649488002E00020644948806348F5
S113DFF0448803212046FAF7B9F884B2022C03DAE4
S113E00002205E4908717FE05C48008800195B4982
S113E0100880084600885A49884275DD08465749F1
S113E020088071E055484088A0420BDA5348408884
S113E030801C5249488008464088A04204DD0846B6
S113E040448001E04D4844804C48448803212046E4
S113E050FAF78CF884B2022C00DA022447480088CC
S113E0602919884202D245490D804DE04348008871
S113E070001B4249088047E0404844880321204669
S113E080FAF774F884B2022C3EDD3C484088062836
S113E09005DD3A484088801F3849488002E0002066
S113E0A0364948803548448803212046FAF75EF80B
S113E0B084B232480079012813D1022C03DA0220F9
S113E0C02E49087120E02D48008800192B4908804A
S113E0D0084600882A49884216DD084627490880F0
S113E0E012E0022C03DA0120244908710CE02348D1
S113E0F00088A04205DD21480088001B1F490880D4
S113E10002E000201D4908801C4800881D49098838
S113E110884203DA194800880F2804DA174800886F
S113E120184908800AE01548008816490988081A21
S113E1300F2803DB1148008812490880114807881A
S113E1400B48007800280DD06C20474364213846E2
S113E150F9F7F6FF07460A48874200D907460A49F5
S113E1600F8002E0002008490880FEBD2808002036
S113E170420000203C000020180800204400002039
S113E180C6070000400000203E0000200020074990
S113E19008800749088007490880488001200871E1
S113E1A00020054948800880704700003E00002098
S113E1B040000020440000201808002000200249EC
S113E1C00870024908707047880000208900002008
S113E1D010B5FEF72BFB012813D103210C48FCF7E3
S113E1E071FF552805D100200A4908700A490870B2
S113E1F00CE002F065F80749087001200649087030
S113E20004E00020034908700349087010BD0000B1
S113E210280800208800002089000020F0B5A9B05B
S113E22004460E460025002700202890A0216846B9
S113E230FAF736F8FFF7D2F826490A681421614341
S113E240505024480168142060430818C068B04244
S113E2500CD220480168142060430818C1681D4886
S113E2600268142060431018416005E019480168F1
S113E270142060430818466016484068002826D0D9
S113E280002517E06806070E282F00D316E0114872
S113E2900168142068430858B9006A4650500D4874
S113E2A001681420684308184168781C80001150E4
S113E2B0681CC5B20748007AA842E3DC00BF6A00C4
S113E2C0044869464368022098470120289028980A
S113E2D029B0F0BD082B002010B500F0EDFD00F0D2
S113E2E0D7F80FF0C1F800F00DFB00F001F810BDF5
S113E2F070B541480078912800D070BD00F0BEF898
S113E300012876D13D4800883D4908800846807838
S113E310F021884320303A49887008468078000903
S113E32000013549097A0907090F084334498870FF
S113E3303148807A401E3049887208460089401C62
S113E340088108460089C988884216DA08202C49C1
S113E350887200240EE0284841882848001D415C4A
S113E3602748C01C015524484088401C2249488045
S113E370601CC4B2072CEEDB2DE01F4800891E4947
S113E380C98888421CD11C4800791B498978401AE5
S113E390C5B2681C1A49887200240EE016484188E8
S113E3A01648001D415C1648C01C0155124840889F
S113E3B0401C11494880601CC4B2AC42EEDB0AE048
S113E3C000F006FD00200C4908700C49088809215A
S113E3D000F0B8F991E7012000F0BCFC084A917AFA
S113E3E01088921C00F070F905490888002100F09B
S113E3F0C1F800BF81E700006C2800200828002035
S113E400982700201B49097E002932D01949897EAA
S113E4100C225143174A515A174A118000200CE02C
S113E4201449897E0C225143124A8918891C0A5CBA
S113E4301149891C0A54411CC8B20828F0DB0D4953
S113E440897E0C2251430B4A8918897A0A4A9172AF
S113E4500121D1720749097E491E064A11761146E7
S113E460897E491C91761146897E022901DB0021AF
S113E47091767047642700208C2700200349487B4D
S113E480012802D10021014A517370477C280020E1
S113E49010B533484068002861D13148007B03003F
S113E4A00FF0D4FF07590512212E3D4A59002D487B
S113E4B00078002807D000202A4908702A490888D3
S113E4C0012100F03FF947E026480078002809D0F0
S113E4D000202449087025494A8808880123091D19
S113E4E000F040F938E01F480078002807D00020E9
S113E4F01C4908701C490888022100F023F92BE00C
S113E50018480078002809D00020164908701749D7
S113E5104A8808880923091D00F024F91CE01148E1
S113E5200078002807D000200E4908700E4908889A
S113E530092100F007F90FE00A480078002809D003
S113E54000200849087009494A8808880323091DDE
S113E55000F008F900E000BF00BF00F039FC10BD76
S113E5607C2800206C28002008280020A4270020F4
S113E5707047000070B504460D4634480088A04238
S113E58063D1002D61D13248007822284ED004DCBA
S113E59020283DD0212856D141E0902802D091284E
S113E5A051D115E02A48C08801280AD10020284901
S113E5B0087000F00DFC27490888002100F0C2F81B
S113E5C005E0032000F0C6FBA020214908703BE0D1
S113E5D01F4800891E49C98888420AD100201C4965
S113E5E0087000F0F5FB1B490888002100F0AAF828
S113E5F00DE01748807A002806D000F0E9FB1449A2
S113E600087B00F089FB02E0032000F0A3FB1BE081
S113E610062000F09FFB11200D49087014E006202D
S113E62000F098FB11200A4908700DE00020084909
S113E630087000F0CDFB08494A8808880923091DA1
S113E64000F090F800E000BF00BF70BD80270020FC
S113E6506C28002008280020A427002070B5034659
S113E660184C247E022C00DB70BD164C647E0C25F5
S113E6706C43144D2B5300200AE0155C114C647E4E
S113E6800C2674430F4EA419A41C2554441CE0B258
S113E6908842F2D30B4C647E0C267443094EA419B1
S113E6A0A1723446247E641C35462C762C46647E46
S113E6B0641C6C762C46647E022C01DB00246C7690
S113E6C000BFD1E764270020F0B585B007460D46AA
S113E6D016461A480780002406E031781748801C43
S113E6E00155761C601CC4B2AC42F6DB2C4605E036
S113E6F0AA211248801C0155601CC4B2082CF7DB07
S113E7000E480088019008216846C17200214172B8
S113E71001720170002406E00848801C015D03A812
S113E7200155601CC4B2082CF6DB69460448FCF7AA
S113E730D0FD01200149887205B0F0BD802700207A
S113E7409055044070B504460D46294620460EF007
S113E750B7FD70BD70B504460D46294620460EF03F
S113E760BDFD70BDF8B504460D4616461F463B4632
S113E7703246294620460EF0B2FDF8BDF8B50746EC
S113E7800E4615465C480078002804D00921384616
S113E790FFF7D8FFF8BD002D01D0602D04DD09215D
S113E7A03846FFF7CFFFF5E754480780458000243B
S113E7B006E031785148001D0155761C601CC4B236
S113E7C0AC42F6DB00204C49487008468580FF20A7
S113E7D088727F2008730846808808282EDA012072
S113E7E0C880084680884880012008814348008802
S113E7F04349088008468078F0218843404988705E
S113E80008468078000900013B4909790907090F86
S113E81008433B49887038480079401C88720024BA
S113E82007E03648001D015D3548C01C0155601CD9
S113E830C4B231488088A042F3DC4AE00721681C56
S113E840F9F794FC002907D0072128460830F9F786
S113E8508DFC2949C88005E00721681CF9F786FC6E
S113E8602549C8800620244948800120088123487E
S113E87000882349088008468078F02188431030B6
S113E8801F49887008468078000900011A49898860
S113E8900905090F08431A49887008464088FF2172
S113E8A009028843144989880902FF22120211408F
S113E8B008431349488008208872002407E00F4861
S113E8C0001D015D0E48001D0155601CC4B2062CDC
S113E8D0F5DB012000F03EFA094A917A1088921C77
S113E8E0FFF7F2FE902004490870054908880021CA
S113E8F0FFF740FE00BF4DE76C28002008280020E9
S113E9009827002010B5FFF77DFD1448C07A002831
S113E91022D0124880780009002806D0012807D0A8
S113E92002280AD0032810D10CE000F09DF90FE072
S113E93000F09EF800F05AFA0AE000F011F800F036
S113E94055FA05E000F000F902E0FFF711FE00BF00
S113E95000BF00200149C87210BD00008C270020B0
S113E96010B540480078112800D010BD3E480088FA
S113E9703F214901884200D0F7E73B4880780007EF
S113E980000F3849097A0907090F88420CD0002082
S113E9903449087000F01CFA34494A880888042372
S113E9A0091DFFF7DFFEE0E72E480089401C2D49D2
S113E9B008810846807A401E887208460089C98802
S113E9C088421BDA2848807A082800D0CDE7002442
S113E9D00EE02548C01C015D224842882348001DE2
S113E9E0815420484088401C1E494880601CC4B2A1
S113E9F0072CEEDB062000F0ADF930E019488088E2
S113EA0018494988401A1849897A884203DA16480D
S113EA10807A082800D0A8E700240EE01248C01C21
S113EA20015D104842881148001D8154601CC4B225
S113EA300C484088401C0B4948800A4840880949D2
S113EA4089888842EADB00200649087000F0C0F992
S113EA5006494A8808880023091DFFF783FE00BF82
S113EA6083E700006C2800208C270020A4270020C6
S113EA7070B53248007880210840802800D170BDEC
S113EA802F4800883F214901884200D0F7E72C48ED
S113EA90807A082800D0F2E72948807805072D0FEE
S113EAA02D0227484088000A0543082D00DAE6E7CE
S113EAB000202249487006204880084685800120AD
S113EAC00881082088720020C8728988481C0721A0
S113EAD0F9F74CFB002909D0184989880846083001
S113EAE00721F9F743FB1549C88007E013498988D2
S113EAF0481C0721F9F73AFB1049C88010480088E0
S113EB001049088008464580002407E00C48001D91
S113EB10015D0C48001D0155601CC4B2062CF5DBD8
S113EB20042000F017F9102004490870054A5188A0
S113EB301088FFF70FFE00BFA1E700006C2800203B
S113EB408C270020A427002010B544480078A02872
S113EB5008D042480078912804D040480078A12881
S113EB6000D010BD3E4800883F21490188420AD0A8
S113EB703C4908880921FFF7E5FD00F029F9002048
S113EB8036490870EDE73648807A08280AD03549B6
S113EB9008880921FFF7D6FD00F01AF900202F4953
S113EBA00870DEE72E4880780007000F002804D0A4
S113EBB0012825D0022843D12EE028484078002897
S113EBC000D048E02648C078002803D1012023491A
S113EBD0487003E02248C078204988721F480078B2
S113EBE0912803D01E4800791C49087391201B49C1
S113EBF0087000F0EDF81949087B00F08DF82AE060
S113EC0016484078002800D025E0A1201349087058
S113EC10032000F09FF81EE010484078002800D040
S113EC2019E00E480078A02809D10E490888082167
S113EC30FFF788FD00F0CCF80020084908700AE0CE
S113EC40084908880521FFF77DFD00F0C1F8002080
S113EC500249087000BF00BF00BF82E76C28002093
S113EC608C2700200828002010B52848007880212F
S113EC700840802800D110BD24480078002806D020
S113EC80234800883F214901884200D0F3E7204807
S113EC90807A1F4989780907090F884203DD1C48D7
S113ECA0807A082800D0E6E7194880780007000F2A
S113ECB0002805D0164880780007000F072800DDDB
S113ECC0D9E7134800881349088011488078000761
S113ECD0000F4880002407E00D48C01C015D0D486A
S113ECE0001D0155601CC4B20A484088A042F3DCF0
S113ECF000200649087000F06BF806494A88088825
S113ED000023091DFFF72EFD00BFB4E76C28002087
S113ED108C270020A42700207F2805DC7D21C90042
S113ED2041430A4A91600DE0F12808DBF92806DC2A
S113ED300107090F64225143044A916002E0044927
S113ED40024A91600221014A517370477C280020D5
S113ED5018F0010000B503000FF078FB0729050B3C
S113ED6011171D2329000121144A117314495160FC
S113ED7022E00221114A1173114951601CE0032160
S113ED800E4A11730F49516016E004210B4A1173A6
S113ED900D49516010E00521084A117300215160AA
S113EDA00AE00621054A11730849516004E0002174
S113EDB0024A1173516000BF00BF00BD7C280020CF
S113EDC0A8610000F824010028230000F049020093
S113EDD000200149087370477C28002002490988F3
S113EDE00918014A118070477C28002010B52F486B
S113EDF00078102818D12E48408860280ADD2D4854
S113EE00807800090001801C2A4988702220274943
S113EE10087025E02748807800090001254988709A
S113EE202020224908701BE020480078112816D1C0
S113EE301E48807A002800D010BD1C484078002865
S113EE4000D0F9E70820194988721A488078000927
S113EE5000011849887020201449087000E0EBE78D
S113EE60FD20C0001349088008468078F0218843BB
S113EE703030104988700846C0780020C8700846B1
S113EE80007914200871032088720220FFF762FFC2
S113EE90084A917A1088921CFFF716FC05490888E5
S113EEA00021FFF767FB00BFC6E700006C280020C5
S113EEB0A427002098270020244A118852888A42D7
S113EEC042D0224A52888A4204DA204A52888A1A54
S113EED090B207E01D4A52880023DB439A1A521C61
S113EEE0521890B2194A5180127B002A10D0174A46
S113EEF05268002A0CD0154A5268824205D9134A36
S113EF005268121A114B5A6002E000220F4B5A60E9
S113EF100E4A527B022A17D10C4A9268002A0CD05E
S113EF200A4A9268824205D9084A9268121A074B23
S113EF309A6002E00022054B9A60044A9268002A13
S113EF4002D10122014B5A73704700007C28002033
S113EF50FEB50027002002900190009000250026B5
S113EF600024FDF763FC012879D10021A748FCF7B0
S113EF70A9F8552808D1A6480178A648F9F790F9C8
S113EF800020A349087040E101F0AEF9074601F002
S113EF90BFF9029001F0B2F9019001F0C3F90090B9
S113EFA001F098F99C490870F020384000110A28B3
S113EFB005DBF02038400011C01C054303E0F020BD
S113EFC03840001105432D023807000F0A2804DBDE
S113EFD03807000FC01C054302E03807000F054343
S113EFE02D02F0210298084000110A2805DB02983E
S113EFF008400011C01C054304E0F02102980840B9
S113F000001105432D0202980007000F0A2805DBB2
S113F01002980007000FC01C054303E00298000794
S113F020000F0543F0210198084000110A2805DB70
S113F030019808400011C01C064304E0F021019827
S113F040084000110643360201980007000F0A2801
S113F05006DB01980007000FC01C064304E0CCE067
S113F06001980007000F06433602F021009808407B
S113F07000110A2805DB009808400011C01C064353
S113F08004E0F0210098084000110643360200987D
S113F0900007000F0A2805DB00980007000FC01CBA
S113F0A0064303E000980007000F06435A4800781F
S113F0B0002811D100240AE00020A100554A505034
S113F0C0A100564A5050A100554A5050641C482C87
S113F0D0F2D3002053490870524800784E49097809
S113F0E0884218DA002D16D04E4802784B4928463B
S113F0F000F0D8F800280ED14A480078800047492B
S113F1000D5048480078401C46490870084601786C
S113F110424800F0D8F8434800783F4909788842CB
S113F12018DA002E16D03F4802783C49304600F0E9
S113F130B9F800280ED13B480078800037490E50BA
S113F14038480078401C374908700846017833482D
S113F15000F0B9F8334800782F49097888420EDD69
S113F160002407E00020A1002C4A5050A1002C4AA2
S113F1705050641C482CF5D300202A4908702948B3
S113F18000782549097888423FD100240FE0A00087
S113F19022490858A100224A50500020A1001F4AC9
S113F1A050501B4801781E4800F08DF8641C1D481F
S113F1B000788442EBD31848007815490870002081
S113F1C018490870002413E0A00012490858A1004F
S113F1D0134A515888420AD0A00011460858A10089
S113F1E00C4A50500A480178104600F06CF8641C30
S113F1F0074800788442E7D307E0054801780548CA
S113F200F9F74EF8002002490870FEBD28080020D6
S113F21082000020B00B002080000020900A002013
S113F220700900208100002010B505F0E7FD10BD35
S113F23000BF704710B504468020204301460320D8
S113F240400205F095FC10BD10B5102103204002CA
S113F25005F08EFC10BD000010B50224024805F034
S113F260D7FC0446204610BD0106000010B500215D
S113F270014805F07DFC10BD0106000010B50446F0
S113F280802020430146024805F072FC10BD0000B6
S113F2900106000010B51021014805F069FC10BDFD
S113F2A00106000030B503460C460021002000BFD3
S113F2B006E08D0065599D4200D101204D1CE9B244
S113F2C09142F6DB30BDF8B505460E4600240EE04B
S113F2D0601CC7B207E0BA005119A200501900F02F
S113F2E00AF8781CC7B2B742F5DB601CC4B2701EC2
S113F2F0A042EDDCF8BD10B503680C68A34203D945
S113F3000A6803680B60026010BD70B505460024EE
S113F310FFF71EFE70BD00002E480078401C2D49EA
S113F32008702D480078401C2B4908702B48007841
S113F330401C2A4908702A480068401C2849086073
S113F34008460068FF219131884202D900202449EF
S113F350086020480078C82802D900201D49087098
S113F3601D480078842802D900201B4908701B48D6
S113F3700078502802D90020184908701948184903
S113F3800968405C18490870184812490978405CBB
S113F39017490870174810490978405C16490870E5
S113F3A016480E490978405C154908701548094902
S113F3B00978405C14490870144806490978405C8F
S113F3C013490870134803490978405C12490870CE
S113F3D07047000053070020540700205507002001
S113F3E05807002053F901004C070020E3FA0100FC
S113F3F04D070020ABFB01004E070020F7FC010085
S113F400500700202FFC01004F07002047FD01009A
S113F410510700200FFE01005207002010B58200A2
S113F420054BD218525C012A04D100228300024CFD
S113F4301B195A5410BD0000E826002010B50446DC
S113F440204600F049FA204600F002F810BD000002
S113F45010B50446B248007800287DD1B148008830
S113F460B149884278DAB148007800284FD0B048D2
S113F4700078002803D0AB480088AE490880AE4825
S113F4800078002818D1A7480188AA4800881930B4
S113F490814206D30120A8490870A2480088A549E2
S113F4A00880A0480088A349098888421CDA9D483E
S113F4B00088A049088017E09E4801889948008880
S113F4C01930814206D300209B4908709548008872
S113F4D0984908809348008896490988884203DD42
S113F4E0904800889349088093480078002857D1B1
S113F4F092480078042803D08D480078002807D06B
S113F50088480088822803DA05208C490870A1E025
S113F5108A480078032803D085480078002809D059
S113F52080480088FF211931884203DA0420834986
S113F53008708FE081480078022803D07C48007866
S113F54000280AD077480088FF21AF31884204DAC6
S113F55003207A4908707DE0E0E0784800780128CB
S113F56003D073480078002808D06E480088744996
S113F570884203DA0220714908706BE06F48007812
S113F580002803D06A480078002863D065480088C2
S113F5903721090188425DDA01206849087059E081
S113F5A065480078012855D164480078012803D0C3
S113F5B05F480078002809D05A480088372109019B
S113F5C0884203DB00205D49087043E05B48007813
S113F5D0022803D056480078002808D051480088F3
S113F5E05749884203DB01205449087032E05348EC
S113F5F00078032803D04E480078002809D04948F1
S113F6000088FF21AF31884203DB02204B49087098
S113F61020E04A480078042803D0454800780028B0
S113F62009D040480088FF211931884203DB0320B8
S113F630424908700EE041480078052803D03C4850
S113F6400078002806D037480088822802DB04208E
S113F6503A490870FDF7D0F83349643988425DD3DC
S113F6603848006800193749086031480078002894
S113F67008D000202E490870324908602F480078CD
S113F6803149087000F082FD00281FD12D48006820
S113F6902E49884239D300202A4908602A48007834
S113F6A026490978884205DA27480078401C26490B
S113F6B008702AE02448007820490978884224DD2B
S113F6C021480078401E204908701EE01D4800684B
S113F6D01F49884219D300201A4908601A48007843
S113F6E016490978884205DA17480078401C1649FB
S113F6F008700AE01448007810490978884204DD4B
S113F70011480078401E104908700F4800780B49D2
S113F7100978884202D100200A49086010BD00001F
S113F7200B000020020000201C0C0000120000202E
S113F73008000020040000200A0000200600002029
S113F740760200001800002007000020C05D0000C1
S113F750407E050000200B4908700B490870012009
S113F7600A4908700A49087000200A4908700A49C1
S113F77008700A4908800A4908800A4908800A4929
S113F78008707047060000200700002008000020D1
S113F790090000200A0000200B0000200C000020BB
S113F7A00E000020100000201200002000200B4951
S113F7B008700B49087001200A4908700A4908704A
S113F7C000200A4908700A4908700A4908800A4951
S113F7D008800A4908800A4908707047060000201A
S113F7E00700002008000020090000200A00002073
S113F7F00B0000200C0000200E0000201000002050
S113F80012000020F1B500272D480078002804D00C
S113F8100320F9F797FE2B4908802B480088192804
S113F82047D300202849088028480078142829D282
S113F8300320F9F787FE0746002407E06000244907
S113F840085AB84200DD05E0601CC4B21F480078C5
S113F8508442F3DB00BF1D48057808E0681E4000C1
S113F8601B49085A69001A4A5052681EC5B2A5427B
S113F870F4DC600016490F5214480078401C134908
S113F880087016E00026052405E060001049085AB7
S113F8908619601CC4B20F2CF7D30A213046F8F73E
S113F8A04FFC0849088000200849087001200949D4
S113F8B00870054801880098081803490880F8BDB5
S113F8C00900002002000020160000200000002093
S113F8D0E4070020120000203A4909881E2928DA8A
S113F8E00021394A1180394A118039490988394A35
S113F8F0914207DC38490978002914D03449098831
S113F900914210DD0121354A11700021344A1170F1
S113F910344A1170304A11700121334A11700021A8
S113F920324A11704CE02A4909880918284A118082
S113F93046E024490988274A643291422BDB00219E
S113F940234A1180214A11801F490988AF221201DC
S113F950914207DC20490978002916D01A49098800
S113F960914212DD02211D4A117000211C4A1170BE
S113F97005211C4A11700021174A117001211A4AED
S113F98011700021194A11701AE00F4909880918E9
S113F9900D4A118014E000210D4A11800A4A118099
S113F9A00A4909880B4A914205DD00210B4A11706E
S113F9B0094A117004E0054909880918034A1180AD
S113F9C07047000002000020100000200C000020FE
S113F9D00E000020B80B0000090000200B000020DE
S113F9E00600002007000020080000200A00002074
S113F9F00148007870470000580900200148007A47
S113FA0070470000580900200148807870470000C2
S113FA105809002001480088704700007C0000203D
S113FA20F8B50023002500950024002200BF94E0CF
S113FA3001259D40ACB20D8825400095009DA5424E
S113FA406FD11A468D79012D0DD1464D032636020C
S113FA50AD192D5C012696403543424E03273F02E3
S113FA60F61935540CE03F4D03263602AD192D5CD2
S113FA7001269640B5433B4E03273F02F619355401
S113FA80CD78002D4ED1374D60352D5CCE78002ECB
S113FA9001D1012600E000269640B543314E603680
S113FAA035548D78002D2ED12E4D19267601AD19A1
S113FAB02D5C8E78002E01D1012600E000269640B0
S113FAC0B543284E19277F01F61935540D79002DB9
S113FAD00ED1244D50352D5C0E79002E01D1012616
S113FAE000E000269640B5431E4E5036355423E0C0
S113FAF01C4D50352D5C0E7996403543EEB2194DB0
S113FB0050352E5418E0174D19267601AD192D5C89
S113FB108E7896403543134E19277F01F6193554D4
S113FB200AE018E00F4D60352D5CCE7896403543E1
S113FB30EEB20C4D60352E544D79012D0AD1094D8C
S113FB4030352D5C012696403543EEB2054D3035F7
S113FB502E5400E000BF5D1CABB2082B00DA67E74F
S113FB60F8BD000000000440FFB5074615461E46D8
S113FB7000243846019900F01FF8002802D0012023
S113FB8004B0F0BD00240CE00A2060430949085C7D
S113FB90B04204D12946204600F05EF807E0601C1C
S113FBA084B20A2060430349085C0028ECD100BFFA
S113FBB00020E5E7B00100200246002A03D14029D5
S113FBC001DD01207047032A03D1022901DD012050
S113FBD0F8E7042A03D1202901DD0120F2E7052AF0
S113FBE003D1202901DD0120ECE70C2A03D11029DF
S113FBF001DD0120E6E70D2A05D1012903DD4029B5
S113FC0001DA0120DEE70E2A03D1202901D10120E7
S113FC10D8E70020D6E7000010B5064A03231B02EC
S113FC20D218125C8A43034B032424021B191A546E
S113FC3010BD00000000044010B5064A03231B0257
S113FC40D218125C0A43034B032424021B191A54CE
S113FC5010BD00000000044070B502460020B1E071
S113FC600A2353435A4C1B195B1C440004191B19E7
S113FC709B788B427DD10A235343554C1B195B1C43
S113FC80440004191B195B78082B33D10A2353430E
S113FC904F4C1B195B1C440004191B574D4C4E4D13
S113FCA06419E35C012423430A245443484D641932
S113FCB0641C450045196457464D474EAD192B55F4
S113FCC00A235343424C1B195B1C440004191B5761
S113FCD0404C35466419E35C022423430A2454430C
S113FCE03B4D6419641C450045196457394DAD19E1
S113FCF02B5564E00A235343354C1B195B1C440009
S113FD0004191B195B78092B34D10A235343304C53
S113FD101B195B1C440004191B572E4C2E4D6419EF
S113FD20E35C402423430A245443294D6419641C8E
S113FD30450045196457274D274EAD192B550A2305
S113FD405343234C1B195B1C440004191B57214CBF
S113FD5035466419E35C8024A3430A2454431C4DB0
S113FD606419641C4500451964571A4DAD192B5587
S113FD7025E025E00A235343154C1B195B1C440062
S113FD8004191B57134C144D6419E35C0A2454439F
S113FD900F4D6419641C45004519641965780124E4
S113FDA0AC402343DCB20A235343094D5B195B1C6B
S113FDB0450045195B57074D074EAD19EC5404E057
S113FDC0431CD8B2032800DA4AE700BF70BD000024
S113FDD0B00100200000044075080000F8B50024BC
S113FDE0FCF724FD012861D100F030FB0446BA225F
S113FDF00721002002F05AFF012C21D100F0A4FBBE
S113FE0000280ED000F056FB054600F047FB0646DE
S113FE1001200346024629460090304605F01CFAAC
S113FE2050E000F047FB054600F038FB0646012091
S113FE300023024629460090304605F00DFA41E0C1
S113FE40022C21D100F080FB00280ED000F032FB00
S113FE50054600F023FB06460120034602462946D8
S113FE600090304605F0F8F92CE000F023FB05463D
S113FE7000F014FB0646002001231A462946009090
S113FE80304605F0E9F91DE000F05EFB054600F0A0
S113FE9011FB064600F002FB0746012003462A46F2
S113FEA031460090384605F0D7F90BE000200346B0
S113FEB002460146009005F0CFF9002207211046C2
S113FEC002F0F4FEF8BD0000F0B585B000247348DC
S113FED00078012824D1FCF7A9FC012812D1FCF7F1
S113FEE0C1FA00BF0BE0182C02D1601CC4B204E0BC
S113FEF0BA222146002002F0D9FE601CC4B2242C90
S113FF00F1DBC8E0FCF7F8FB002406E00022214600
S113FF10104602F0CBFE601CC4B2242CF6DBBAE01F
S113FF20FCF784FC01287DD1FCF766FC5C4988421F
S113FF307FD35C480088032805DA5A480088401CAF
S113FF405849088011E000205649088000F0ACFAB6
S113FF50064600F0C7FA07460A21F8F7F1F8054605
S113FF6032462946012009F0FBFD00F02DFC06462F
S113FF7000F0D2FB0A210390F8F7E2F8054600F0FE
S113FF8093FA07463246294608F01EF8FFF726FF83
S113FF9000F050FA05462946012006F0DFFC00F087
S113FFA09BFA0646FF21F531F8F7E0F8C5B2294679
S113FFB0012006F00FF9FFF71BFD0546FFF72AFDA8
S113FFC00646FFF721FD07462B46324639460120F7
S113FFD005F01CFC00F0E0F80546294601200AF073
S113FFE065F800F0B3FB054600F0BAFA064600F0E7
S113FFF06DFA074600F0B0FB039000F0B7FA3B46F9
S21401000000960195029001460120039A09F0E0F856
S21401001000F076FB054600F06DFB064600F076FB29
S214010020074601E008E004E02A46314606F0CEFE27
S21401003031E0FCF791FA2EE0FCF75EFB002223216B
S214010040104602F033FE00222221104602F02EFE58
S21401005000220721104602F029FE00220821104640
S21401006002F024FE00220921104602F01FFE0022A3
S2140100700A21104602F01AFE00221321104602F051
S21401008015FE00221121104602F010FE0022122158
S214010090104602F00BFE05B0F0BD00000301002083
S2140100A0B80B000076000020014908607047000088
S2140100B08007002002480068401C0149086070471C
S2140100C07C070020F3B581B0064600200E49086083
S2140100D000F01EF8044600F01BF805462F1B3046BC
S2140100E0029903F087FD00900AE000F011F805463A
S2140100F02F1B06480068002802D004480068804785
S21401010000988742F1D3FEBD7C07002080070020BF
S21401011001480068704700007C0700200B490978F9
S214010120012901D101200FE008490978022901D1EE
S214010130022009E005490978032901D1042003E0DA
S2140101400121024A117001207047000015070020A6
S21401015010B5094B1B8899B20A12C8B2D343313382
S214010160064C2370C3432333637013465633A37080
S21401017003467133E37010BD440700201B070020BF
S21401018001480088704700002400002001480088CC
S214010190704700003C0000200148007870470000CE
S2140101A08800002001480078704700008900002080
S2140101B010B5002205210648FAF772FF0402012253
S2140101C005210348FAF76CFF201880B210BD000025
S2140101D02808002010B5062205210348FAF760FF1B
S2140101E0C006C00F10BD00002808002010B504226C
S2140101F005210648FAF754FF040205221146034872
S214010200FAF74EFF201880B210BD00002808002023
S21401021010B5062205210248FAF742FFC01110BDAB
S2140102202808002010B5022205210248FAF738FFF7
S21401023010BD00002808002010B50622052103483D
S214010240FAF72EFF8006C00F10BD00002808002018
S21401025010B5042202210348FAF722FFC007C00F97
S21401026010BD00002808002010B505220221034811
S214010270FAF716FFC007C00F10BD000028080020BF
S21401028010B5002204210348FAF70AFF4006400F82
S21401029010BD00002808002010B5002201210248E8
S2140102A0FAF7FEFE10BD00002808002010B5012256
S2140102B011460248FAF7F4FE10BD00002808002097
S2140102C010B5022203210248FAF7EAFE10BD00002B
S2140102D02808002010B5032200210248FAF7E0FEA4
S2140102E010BD00002808002010B500221146024863
S2140102F0FAF7D6FE10BD00002808002010B504222B
S21401030000210248FAF7CCFE10BD000028080020A4
S21401031010B5012200210248FAF7C2FE10BD000006
S2140103202808002010B5052200210248FAF7B8FE79
S21401033010BD000028080020322815DA3C498978CB
S214010340012903DD01213A4A517070E03849897864
S214010350002905DD2F286ADC0021354A517066E048
S2140103600021334A517062E03E2817DA322815DB45
S2140103702F498978022903DD02212D4A517056E062
S2140103802B498978012905DD3B2850DC0121284AC3
S21401039051704CE00121264A517048E0502817DA86
S2140103A03E2815DB22498978032903DD0321204AEB
S2140103B051703CE01E498978022905DD4D2836DC5E
S2140103C002211B4A517032E00221194A51702EE077
S2140103D0622817DA502815DB15498978042903DDC8
S2140103E00421134A517022E011498978032905DD59
S2140103F05F281CDC03210E4A517018E003210C4AC9
S214010400517014E073280FDA62280DDB08498978E9
S214010410042905DD70280ADC0421054A517006E02E
S2140104200421034A517002E00521014A51707047C8
S2140104305809002001480078704700000700002096
S2140104400148007870470000F0000020014800785D
S21401045070470000EF000020F8B5002600240025B4
S214010460FDF706F907460A21F7F76AFE0546094829
S2140104700068854200D303E006480068461B344600
S2140104807D200001844200D30446034804600068CE
S214010490F8BD000028010020240100200148007852
S2140104A070470000FB0000200148007970470000FB
S2140104B0E80000200148407870470000FB0000205B
S2140104C00148807970470000E80000200148407923
S2140104D070470000E80000200148008870470000CF
S2140104E02600002010B50024FFF7DEFF00280AD101
S2140104F00A4800880A49884202DB084607490880FC
S2140105000648048808E005480088FCF75FFE84B2C8
S2140105100448844200DB0446204610BD3E0000200D
S214010520C6070000CE040000002005490988054AD8
S214010530914202DB1146024A118001490888704740
S2140105403E000020C6070000014800787047000002
S2140105504D07002001480078704700004F07002033
S2140105600148007A704700006409002070B5002435
S2140105700E48C07A01280ED10C490868FCF776FAB5
S2140105800546323564212846F7F7DAFD84B2632C36
S2140105900ADD632408E005480088401D84B20A216C
S2140105A02046F7F7E3FD84B2204670BD64090020BB
S2140105B070B5002407490868FCF758FA05460A2171
S2140105C0F7F7BEFD84B20448844200DD04462046A7
S2140105D070BD000064090020DE03000010B5002491
S2140105E000F016F8012801D103240CE000F010F801
S2140105F0022802D1FF24373405E00A210348008887
S214010600F7F7B4FD84B2204610BD000002000020BA
S21401061001480078704700000B00002010B5002448
S214010620044804F0F5FA002801D0012400E0002473
S214010630204610BD0307000010B50024054804F04D
S214010640E7FA002802D00120044601E00020044613
S21401065010BD00000507000010B50024054804F091
S214010660D7FA002802D00120044601E00020044603
S21401067010BD00000707000010B50024062004F096
S214010680C7FA002801D0012400E00024204610BD4E
S21401069010B50024054804F0BBFA002802D001205A
S2140106A0044601E00020044610BD000006070000D5
S2140106B010B50024044804F0ABFA002801D0012448
S2140106C000E00024204610BD0305000010B50024FC
S2140106D0044804F09DFA002801D0012400E000241B
S2140106E0204610BD040500000148807A70470000CE
S2140106F0640900200148807870470000D00C002073
S2140107000148406870470000D00C0020014840783E
S21401071070470000D00C002070B50024FFF7C4FE1F
S214010720002803D1FCF7A4FF04460DE0FFF7BCFE4A
S214010730012806D1FCF79CFF0546FCF747FD044659
S21401074002E0FCF795FF0446204670BD0148407A5A
S214010750704700006409002070B500240E48C07A76
S21401076001280ED10C494868FCF780F90546323558
S21401077064212846F7F7E4FC84B2632C0ADD63247F
S21401078008E005488088401D84B20A212046F7F714
S214010790EDFC84B2204670BD6409002070B50024CB
S2140107A007494868FCF762F905460A21F7F7C8FCCD
S2140107B084B20448844200DD0446204670BD000031
S2140107C064090020DE03000070B50024FFF76CFE0C
S2140107D0002803D1FCF75EFF04460FE0FFF764FE36
S2140107E0012807D10020FCF755FF0546FCF7EEFC73
S2140107F0044603E00020FCF74DFF0446204670BD8A
S21401080001480078704700004200002070B5054698
S2140108100024032D00D170BD002D01D0012D1BD168
S21401082081210320800204F0A3F98021134804F0FB
S2140108309FF932211248FFF745FC002409E0A20087
S214010840104BD2189178A200985A04F091F9601CC6
S214010850C4B23B2CF3DB0FE0022D0DD1002409E0DE
S214010860A200094BD2189178A200985A04F080F998
S214010870601CC4B23B2CF3DB00BFCCE702060000D1
S214010880A0860100E8EF0100D4F00100F8B50021D0
S21401089000240023002200BF0AE001258D40ABB2F0
S2140108A005881D402C469C4200D10A464D1CA9B223
S2140108B01029F2DB0588FF2D1FDC284D6D7E06888A
S2140108C0B543264E757635462D7E0688B543234EAE
S2140108D0357635466D7E8678F607F60F96403543B3
S2140108E01E4E757635462D7E867802273E40760862
S2140108F096403543194E357622E0184DED7E068832
S214010900B543164EF5763546AD7E0688B543134E8D
S214010910B5768578ED07ED0F1646083EB5400F4EC5
S214010920F67E35430D4EF5768578022635406D0800
S2140109301646083EB540094EB67E3543074EB57697
S2140109400025009505E000BF6D462D786D1CEEB2C2
S21401095000966D462D78012DF5D9F8BD206B044023
S214010960C107C90F002905D00021394A117100229B
S21401097038490A7102210140002905D00021344A74
S2140109801172002233490A7204210140002905D060
S21401099000212F4A117300222E490A7308210140B3
S2140109A0002905D000212A4A1174002229490A7417
S2140109B010210140002905D00021254A1175002289
S2140109C024490A7520210140002905D00021204A2A
S2140109D0117600221F490A7640210140002904D0E1
S2140109E000221B494A711B494A7180210140002996
S2140109F004D0002216494A7216494A72FF21013173
S214010A000140002904D0002211494A7311494A7352
S214010A10012149020140002904D000220C494A74F0
S214010A200C494A74012189020140002904D00022A0
S214010A3007494A7507494A750121C902014000293B
S214010A4004D0002202494A7602494A7670470000DD
S214010A500060004000610040C107C90F002905D0B1
S214010A6001223C490A7100213B4A117102210140D1
S214010A70002905D0012237490A720021364A11722F
S214010A8004210140002905D0012232490A730021C0
S214010A90314A117308210140002905D001222D4950
S214010AA00A7400212C4A117410210140002905D036
S214010AB0012228490A750021274A11752021014083
S214010AC0002905D0012223490A760021224A1176FF
S214010AD040210140002905D001221E494A71002209
S214010AE01D494A7180210140002905D0012219497A
S214010AF04A72002218494A72FF2101310140002939
S214010B0005D0012213494A73002213494A73012171
S214010B1049020140002905D001220E494A740022EB
S214010B200D494A74012189020140002905D001229C
S214010B3008494A75002208494A750121C90201403F
S214010B40002905D0012203494A76002202494A7645
S214010B5070470000006100400060004010B50C487E
S214010B600078002803D00B4A5068916888470848E7
S214010B704078002803D0084A50689168884704489E
S214010B808078002803D0054A50689168884710BDD0
S214010B9000600040000300208004002000060020C2
S214010BA010B508480079002803D0074A1069516932
S214010BB0884704484079002803D0044A5068916861
S214010BC0884710BD00600040000300208C04002010
S214010BD010B50848007A002803D0074AD069116A80
S214010BE088470448407A002803D0044A5068916830
S214010BF0884710BD006000400003002098040020D4
S214010C0010B50848007B002803D0074A906AD16ACD
S214010C1088470448407B002803D0044A50689168FE
S214010C20884710BD0060004000030020A404002097
S214010C3010B50848007C002803D0074A506B916B1A
S214010C4088470448407C002803D0044A50689168CD
S214010C50884710BD0060004000030020B00400205B
S214010C6010B50848007D002803D0074A106C516C67
S214010C7088470448407D002803D0044A506891689C
S214010C80884710BD0060004000030020BC0400201F
S214010C9010B50848007E002803D0074AD06C116DB5
S214010CA088470448407E002803D0044A506891686B
S214010CB0884710BD0060004000030020C8040020E3
S214010CC010B50848407F002803D0074A506891684D
S214010CD088470448007F002803D0044A906DD16DF0
S214010CE0884710BD00600040D404002000030020A7
S214010CF010B508484078002803D0074A5068916824
S214010D00884704480078002803D0044A506E916E44
S214010D10884710BD20600040E0040020000300204A
S214010D2010B509480079002803D0084A106F516FA2
S214010D3088470548001D4078002803D0044A5068BB
S214010D409168884710BD0000206000400003002025
S214010D50EC04002010B5034AD06F783291688847BA
S214010D6010BD00000003002010B5024A50689168CB
S214010D70884710BD8403002010B50948007C002870
S214010D8003D0084A50689168884705481030407873
S214010D90002803D0044A50689168884710BD0000B7
S214010DA020600040900300201005002010B5024A84
S214010DB050689168884710BD9C03002010B5024A10
S214010DC050689168884710BDA803002010B50948EF
S214010DD0007F002803D0084A506891688847054874
S214010DE01C304078002803D0044A50689168884730
S214010DF010BD000020600040B40300203405002030
S214010E0010B50C480078002803D00B4A506891684A
S214010E10884708484078002803D0084A50689168F7
S214010E20884704488078002803D0054A50689168AE
S214010E30884710BD40600040C003002040050020E8
S214010E40C006002010B50D480079002803D00C4AD2
S214010E505068916888470948001D4078002803D0EB
S214010E60084A5068916888470448001D8078002821
S214010E7003D0054A50689168884710BD406000401D
S214010E80CC0300204C050020CC06002010B50D48F0
S214010E90007A002803D00C4A5068916888470948B0
S214010EA008304078002803D0084A5068916888477F
S214010EB0044808308078002803D0054A50689168B5
S214010EC0884710BD40600040D80300205805002028
S214010ED0D806002010B50D48007B002803D00C4A28
S214010EE050689168884709480C304078002803D03C
S214010EF0084A50689168884704480C308078002872
S214010F0003D0054A50689168884710BD406000408C
S214010F10E403002064050020E406002010B50D4817
S214010F20007C002803D00C4A50689168884709481D
S214010F3010304078002803D0084A506891688847E6
S214010F40044810308078002803D0054A506891681C
S214010F50884710BD40600040F00300207005002067
S214010F60F006002010B5024A50689168884710BD07
S214010F70FC03002010B50948007E002803D0084A6B
S214010F80506891688847054818304078002803D093
S214010F90044A50689168884710BD000040600040D0
S214010FA0080400208805002010B50948007F0028A5
S214010FB003D0084A50689168884705481C30407835
S214010FC0002803D0044A50689168884710BD000085
S214010FD040600040140400209405002010B5084825
S214010FE00078002803D0074A50689168884704486B
S214010FF04078002803D0044A50689168884710BD9D
S2140110006060004020040020A005002010B50948BB
S2140110100079002803D0084A506891688847054837
S214011020001D4078002803D0044A5068916888471C
S21401103010BD0000606000402C040020AC050020BC
S21401104010B50948007A002803D0084A506891680C
S2140110508847054808304078002803D0044A50687D
S2140110609168884710BD0000606000403804002089
S214011070B805002010B5024A50689168884710BD2F
S2140110804404002010B5024A50689168884710BD94
S2140110905004002010B50948007D002803D0084AF6
S2140110A0506891688847054814304078002803D076
S2140110B0044A50689168884710BD0000606000408F
S2140110C05C040020DC05002010B50948007E0028DD
S2140110D003D0084A50689168884705481830407818
S2140110E0002803D0044A50689168884710BD000064
S2140110F06060004068040020E805002010B509483B
S214011100007F002803D0084A506891688847054840
S2140111101C304078002803D0044A506891688847FC
S21401112010BD00006060004074040020F40500203B
S21401113010B5FE4800688079002806D001286ED0D8
S21401114002286DD003286CD104E2F8480068407983
S21401115003000DF07BF90A0614BC2BBC47BC67BC28
S2140111609BBC09F005FB0020F0490968C873EF48ED
S21401117000684079401CED4909684871AEE0EC49C9
S2140111800969EA4A1268D27A885C09F069FBE7487D
S21401119000684079401CE54909684871E3480068E1
S2140111A04079401CE1490968487197E001F0E6FE84
S2140111B0002810D109F054FBDC4800684079401C37
S2140111C0DA4909684871D94800684079401CD7490E
S2140111D00968487105E009F0F5FA0020D349096865
S2140111E048717BE001F0CAFE002811D1012009F008
S2140111F037FBCE4800684079401CCC4909684871E5
S214011200CA4800684079401CC8490968487105E029
S21401121009F0D8FA0020C549096848715EE05FE028
S214011220FEE0A3E101F0AAFE002828D1BF49096823
S214011230C97A24225143BF4A12688918BB4A1268E8
S214011240D27B885C09F00CFBB8480068C07B401C68
S214011250B6490968C873B5480068C07B242814D30A
S214011260B24800684079401CB04909684871AF48E7
S21401127000684079401CAD490968487105E009F0ED
S214011280A1FA0020A9490968487127E001F076FE15
S214011290002815D1A5480068C07A401CA3490968F2
S2140112A0C872A2480068C07AA1490978884207DB5B
S2140112B000209E490968C87201209C490968887106
S2140112C009F080FA002099490968487106E009F09A
S2140112D079FA002095490968487100BF00BF4FE1BF
S2140112E092480068407903000DF0B0F808051391A4
S2140112F02A914791709109F03BFA00208B490968C1
S214011300C8738A4800684079401C88490968487152
S21401131084E087490969854A1268D27A885C09F0AF
S2140113209FFA824800684079401C804909684871E4
S2140113307E4800684079401C7C49096848716DE028
S21401134001F01CFE002811D1262009F089FA774801
S21401135000684079401C75490968487173480068FF
S2140113604079401C71490968487105E009F02AFA7C
S21401137000206E490968487150E001F0FFFD002821
S2140113801DD1012009F06CFA68480068C07B401C3A
S21401139066490968C87365480068C07B242814D369
S2140113A0624800684079401C6049096848715F4896
S2140113B000684079401C5D490968487105E009F0FC
S2140113C001FA002059490968487127E001F0D6FD65
S2140113D0002815D155480068C07A401C5349096851
S2140113E0C87252480068C07A51490978884207DBBA
S2140113F000204E490968C87202204C490968887164
S21401140009F0E0F9002049490968487106E009F049
S214011410D9F9002045490968487100BF00BFAFE00F
S21401142042480068407903000DF010F80805138B58
S2140114302A8B478B638B09F09BF900203B4909688F
S214011440C8733A4800684079401C384909684871B1
S2140114507EE037490969354A1268D27A885C09F014
S214011460FFF9324800684079401C304909684871E4
S2140114702E4800684079401C2C490968487167E08D
S21401148001F07CFD002811D1252009F0E9F9274853
S21401149000684079401C254909684871234800685E
S2140114A04079401C21490968487105E009F08AF92C
S2140114B000201E49096848714AE001F05FFD0028D6
S2140114C010D109F0CDF9194800684079401C174938
S2140114D009684871154800684079401C1349096835
S2140114E0487105E009F06EF9002010490968487155
S2140114F02EE001F043FD002815D10C480068C07AA3
S214011500401C0A490968C87208480068C07A084938
S2140115100978884207DB002004490968C87203205D
S21401152002490968887109F04DF905E0D0070020E5
S214011530402B0020CC070020002012490968487182
S21401154006E009F03FF900200E490968487100BF1E
S21401155000BF15E000200B49096888710949096830
S2140115604871062007490968C87009E009F02AF998
S214011570002004490968487102490968887100BF5A
S21401158000BF10BDD007002010B56A48006840793A
S21401159003000CF05BFF090610C627C644C6608E22
S2140115A0C60009F0E5F8634800684079401C6149C7
S2140115B009684871BCE0604909695E4A1268D27AD6
S2140115C0885C09F04DF95B4800684079401C594930
S2140115D009684871574800684079401C55490968B0
S2140115E04871A5E001F0CAFC002811D14F2009F08E
S2140115F037F9504800684079401C4E4909684871DF
S2140116004C4800684079401C4A490968487105E021
S21401161009F0D8F8002047490968487188E001F0C8
S214011620ADFC002810D109F01BF94248006840794A
S214011630401C4049096848713E4800684079401C92
S2140116403C490968487105E009F0BCF800203949B1
S214011650096848716CE001F091FC002822D13548F8
S2140116600068C07A401C33490968C872314800686E
S214011670C07A3149097888420FDB00202D49096874
S214011680C8722C4800684079401C2A49096848718C
S214011690002028490968486208E0002025490968B1
S2140116A0487103E0002023490968487109F08AF867
S2140116B03EE020480068407C002816D01E48C068DE
S2140116C0002803D01C48C168192088470020194902
S2140116D00968486217490968487116490968887196
S2140116E0052014490968C8701AE012480068406A63
S2140116F0282807D20F480068406A401C0D4909682F
S21401170048620DE000200B490968486209490968EA
S2140117104871084909688871052006490968C87032
S21401172006E009F04FF8002002490968487100BF39
S21401173000BF10BDD0070020402B002010B50024AC
S214011740F7480068807A01287ED1F5480068C0799C
S21401175000287AD0F24800688079002804D0012851
S21401176074D0022873D191E1ED480068007B2428EB
S2140117706ED2EB480068C07901287AD1002475E062
S214011780E7480068C07A24214843E64909684018BA
S214011790E3490968097B415CE1480068C07A242274
S2140117A05043E14A12688018DD4A1268127B805C59
S2140117B0814229D0DA480068C07A24214843DA49B0
S2140117C009684018D6490968097B415CD448006815
S2140117D0C07A24225043D34A12688018D04A12682D
S2140117E0127B8154CE480068407B242805D3CC4820
S2140117F00068007BCA4909684873C9480068007BCD
S214011800C7490968887308E0C5480068407B2428F2
S21401181003D20120C24909688871C1480068007B6B
S214011820401CBF4909680873BD480068007B24282E
S21401183008D3BB480068407B242803D20120B8495E
S21401184009688871B64805E0D3E1CDE169E0BAE1FF
S21401185038E00EE00068007B242804D2B048006817
S2140118608079012800D103E0601CC4B2242C87D300
S21401187056E0002413E0AA480068C07A24214843B1
S214011880A94909684018015DA5480068C07A242264
S2140118905043A44A126880180155601CC4B2242C17
S2140118A0E9D300209E490968487323209C490968AA
S2140118B0887301209A490968887124209849096823
S2140118C008732DE00020964909680873944800685B
S2140118D0C07A401C92490968C87291480068C07A6B
S2140118E092490978884217DB8D480068007C0128F8
S2140118F004D102208A490968887106E000208849D7
S2140119000968887186490968C87100208449096890
S214011910C8728349096808740020814909684871BA
S21401192061E17F480068407903000CF08FFD0805EF
S21401193013A62AA651A68EA601207949096808741D
S21401194008F016FF764800684079401C744909681B
S214011950487199E075490969714A1268D27A885CBA
S21401196008F07EFF6E4800684079401C6C490968A3
S21401197048716B4800684079401C6949096848719C
S21401198082E001F0FBFA00281BD165490968497B12
S214011990491CC8B208F064FF61480068407B604992
S2140119A00968C8735E4800684079401C5C4909684C
S2140119B048715B4800684079401C5949096848717C
S2140119C005E008F0FFFE00205549096848715BE014
S2140119D001F0D4FA00282BD151490968C97A24228A
S2140119E05143504A126889184D4A1268D27B885C66
S2140119F008F036FF4A480068C07B401C4849096821
S214011A00C87347480068C07B45490968897B884296
S214011A101ADD434800684079401C4149096848710D
S214011A203F4800684079401C3D49096848710BE011
S214011A3008F0C8FE3A480068407B39490968C8730F
S214011A4000203749096848711EE001F097FA00281E
S214011A500CD1334909688871242031490968C87353
S214011A602F49096848732E490968887308F0AAFE49
S214011A7000202B490968487106E008F0A3FE002003
S214011A8027490968487100BF00BFACE024480068D8
S214011A90407903000CF0DAFC08050F8E268E4C8E7A
S214011AA0688E08F065FE1E4800684079401C1C4997
S214011AB00968487185E01D490969194A1268D27A90
S214011AC0885C08F0CDFE164800684079401C144931
S214011AD009684871124800684079401C1049096835
S214011AE048716EE001F04AFA002811D1252008F06D
S214011AF0B7FE0B4800684079401C094909684871DF
S214011B00074800684079401C05490968487105E0A6
S214011B1008F058FE002002490968487151E00000AB
S214011B20D0070020CC070020C8070020402B00204B
S214011B3001F024FA002810D108F092FE64480068EB
S214011B404079401C624909684871614800684079DB
S214011B50401C5F490968487105E008F033FE002023
S214011B605B49096848712CE001F008FA00281AD18F
S214011B7057480068C07A401C55490968C8725448DD
S214011B800068C07A5349097888420CDB0020504926
S214011B900968C8724E49096888714D4909684871D3
S214011BA04B490968C87108F00DFE002048490968CC
S214011BB0487106E008F006FE0020454909684871AC
S214011BC000BF00BF0FE008F0FDFD00204049096896
S214011BD048713F49096888713D49096808733C495D
S214011BE00968C87200BF71E0002039490968887227
S214011BF06CE037480068807A022867D1344800686C
S214011C00007A00285ED0324800684079002804D067
S214011C1001280CD0032846D11BE008F0A9FD2C486A
S214011C2000684079401C2A490968487149E000204B
S214011C3008F016FE264800684079401C24490968C9
S214011C404871234800684079401C21490968487159
S214011C5037E008F057FD002812D11D48006840788B
S214011C60401C1B49096848701948006840780328D9
S214011C7012D301F023FA00201549096848700BE0D9
S214011C800020134909680872AA201149096888705A
S214011C9000200F490968487008F094FD00200C499F
S214011CA0096848710DE008F08DFD002008490968B3
S214011CB04871074909684870AA200549096888706B
S214011CC000BF03E0002002490968887210BD0000C9
S214011CD0D0070020402B0020F8B504460D4600260C
S214011CE00C2060431D49085C002801D00120F8BD86
S214011CF00C2060431949401885600C206043401849
S214011D008068002801D10120F1E701210C20604301
S214011D10124A115400222046E317DB0E1B185B11F2
S214011D205B01E31A9B000E4FDB19E717FF0E3F1905
S214011D307F11DA550CF0BCFB00222046E317DB0EC0
S214011D401B185B115B01E31A9F00064BFB18E71794
S214011D50FF0E3F197F11DA553046C8E70003002011
S214011D60006000400061004000BFFEE709480088AF
S214011D70401C08490880084600880749884208DD53
S214011D8006480078002804D0084602490880012049
S214011D9088707047E4000020DC050000EF0000209A
S214011DA010B515488078012824D1144800780128F8
S214011DB00CD113480078012808D1002011498870F9
S214011DC0084602F0F7FC00200D4908700B48007821
S214011DD002280CD10C480078012808D100200949B6
S214011DE08870084602F0E6FC0020074908700020CB
S214011DF00249087010BD0000E4000020EF0000203A
S214011E00F1000020FB000020F200002070470000D7
S214011E1010B500F03DFE012803D1002001490880DD
S214011E20887010BDE4000020F0B505460E46174642
S214011E3000243A463146284600F038FE00BF42E00C
S214011E4000202101394A126850522101374A12688E
S214011E508918488000212001344A12688018818040
S214011E602001324A12688018C18020012F4A126868
S214011E708018017220012D4A1268801841722001D3
S214011E802A4A1268801881722001284A126880182E
S214011E90C17200202101254A1268891808730021A1
S214011EA02001224A126880184173002021011F4A2E
S214011EB0126889188873002120011C4A126880184C
S214011EC0C173601CC4B21A484078A042B8DC6420D2
S214011ED01849096808807D20C000164909684880AD
S214011EE015481449096888807D2000011149096850
S214011EF0C88010490968088110480E490968488158
S214011F000F480C490968888140000A490968C88158
S214011F103220084909680882FF20F530054909681A
S214011F204882044909688882F0BD000090070020B5
S214011F30840700208C0700204C04000010270000B6
S214011F403075000038B5002404E000201349085518
S214011F50601C84B2282CF8D30121684641700170B8
S214011F606A460F490D48FFF75FFF7D21C900322001
S214011F7000F08CF90B490C4800F0A6F909486430CA
S214011F8000F038F90748C83000F044F9074800F077
S214011F9057F9074800F06AF938BD0000DC23002035
S214011FA058F5010028230000B80B00005424000057
S214011FB01027000010B521480078002803D1012021
S214011FC01E49087038E01D480078012810D11C48C9
S214011FD00078012808D100201A498870084602F0C6
S214011FE0E9FB00201649087002201449087023E016
S214011FF012480078022810D113480078012808D129
S214012000002010498870084602F0D4FB00200E49D3
S21401201008700320094908700EE008480078032874
S21401202003D104200549087006E004480078042816
S21401203002D100200149087010BD0000EF00002009
S214012040F1000020FB000020F2000020F8B500247B
S214012050002500263648007800281ED1354800782D
S214012060002803D101203349087016E03148007872
S214012070012803D102202F4908700EE02D48007870
S214012080022803D103202B49087006E0294800786E
S214012090032802D100202749087025480078012826
S2140120A00ED101241725002623480123324629464E
S2140120B00090204601F0E2FD01202049087036E03C
S2140120C01B48007802280FD101243B2500261A4818
S2140120D0401C0123324629460090204601F0CEFDE1
S2140120E001201749087022E01148007803280DD115
S2140120F0FEF7DAF9002803D101201249087102E03F
S2140121000020104908710CF073F910E008480078B7
S21401211004280CD1FEF7DAF9002803D10120094979
S214012120487102E00020074948710CF061F9F8BDDA
S214012130EF000020F0000020FB000020F10000204E
S214012140F2000020E800002010B5044623000CF041
S2140121507DF90942060E1617181940414500FAF78F
S2140121604BFB2049884201D3FFF770FF37E0FAF7AF
S21401217043FB1C49884201D3FFF71CFF2FE02EE0EA
S2140121802DE02CE0FAF738FB1649884220D301F0FF
S2140121903FFD1548007803280ED114480078002822
S2140121A00AD1FEF78DF9002803D101201049887164
S2140121B002E000200E4988710B480078012805D1FD
S2140121C00A480078002801D1FAF7A8FC09F0D8FFE0
S2140121D005E004E003E0FFF7C9FD00E000BF00BF33
S2140121E010BD0000B80B0000F0000020EF0000203A
S2140121F0E800002001460020054A126852898A42FA
S21401220001DC012002E0024A1268118170470000D9
S2140122108C07002001460020084A126812898A426B
S21401222001DB012009E0054A126892898A4201DC35
S214012230012002E0014A1268518170478C07002094
S21401224001460020084A126852898A4201DB0120B1
S21401225009E0054A1268D2898A4201DC012002E0BF
S214012260014A1268918170478C07002001460020C0
S214012270054A126892898A4201DB012002E0024A7D
S2140122801268D181704700008C07002002460020AA
S2140122900C4B1B681B8A934201DD012010E08A4229
S2140122A001DB01200CE0074B1B689B888B4201DC9D
S2140122B0012005E0034B1B681A80024B1B685980FE
S2140122C0704700008C070020024600200C4B1B685C
S2140122D01B8A934201DD012010E08A4201DB0120C6
S2140122E00CE0074B1B685B88934201DB012005E08D
S2140122F0034B1B689A80024B1B68D980704700000D
S2140123008C07002070B5044600250C206043FE496A
S214012310096840184068002807D00C216143FA4A32
S214012320126889184868804705460C206043F649BC
S2140123300968085C002873D10C206043F2490968DB
S21401234040188068002874D02001F04909684018B8
S214012350C07A02280AD1032D08D10C206043EA4A2C
S2140123601268801881680120884762E02001E749E9
S21401237009684018C07A02280AD1042D08D10C2019
S2140123806043E14A1268801881680220884750E05D
S2140123902001DE4909684018C07A02280AD1052DB5
S2140123A008D10C206043D84A12688018816803203F
S2140123B088473EE02001D54909684018C07A0228BE
S2140123C00AD1062D08D10C206043CF4A1268801826
S2140123D08168042088472CE02001CC490968401810
S2140123E0C07A02280AD1072D08D10C206043C64ABC
S2140123F0126880188168052088471AE02001C349C1
S21401240009684018C07A02280BD1082D09D10C2082
S2140124106043BD4A1268801881680620884708E034
S2140124200DE00C206043B84A1268801881680020CD
S21401243088472001B54909684018C5720CE30C208D
S2140124406043B1490968085C012873D10C206043D8
S214012450AD49096840188068002874D02001AB494E
S21401246009684018C07A03280AD1022D08D10C2029
S2140124706043A54A1268801881680120884762E097
S2140124802001A24909684018C07A04280AD1022D01
S21401249008D10C2060439C4A12688018816802208B
S2140124A0884750E02001994909684018C07A0528F4
S2140124B00AD1022D08D10C206043934A1268801875
S2140124C08168032088473EE020019049096840184A
S2140124D0C07A06280AD1022D08D10C2060438A4A08
S2140124E0126880188168042088472CE020018749FB
S2140124F009684018C07A07280AD1022D08D10C2095
S2140125006043814A126880188168052088471AE06E
S21401251020017E4909684018C07A08280BD1022D8F
S21401252009D10C206043784A126880188168062019
S214012530884708E00DE00C206043734A1268801853
S2140125408168002088472001704909684018C572D3
S21401255082E20C2060436C490968085C0228F7D1C6
S214012560002D7DD1200169490968085A6849096822
S214012570098A884275DA200164490968085A0A30CE
S21401258081B22001614A1268115220015F4909682F
S214012590085A5F490968098A884231DB20015B498C
S2140125A00968401840885A4909680988884227DB23
S2140125B020015649096840184088554909684988E4
S2140125C088421DDC00202101504A12688918488083
S2140125D020014E4909684018807A0028B8D10C209D
S2140125E0604349490968401880680028B0D00C202B
S2140125F06043454A126880188168012088472BE2AB
S214012600200142490968085A41490968098A8842ED
S2140126109EDB20013D490968401840883C4909680D
S2140126208988884294DB2001384909684018408827
S21401263037490968C98888428ADC00202101334A63
S2140126401268891848802001304909684018807A44
S2140126500028D4D10C2060432B490968401801E0BA
S21401266063E00BE080680028C9D00C206043264A4E
S21401267012688018816802208847EDE10020210158
S214012680224A1268891848802101204A126889184E
S214012690C872002120011D4A12688018C1802001DD
S2140126A01A4A1268801841722001184A1268801866
S2140126B08172184801782001144A12688018017244
S2140126C000202101114A12688918888021010F4AC9
S2140126D012688918087321010C4A12688918487310
S2140126E021010A4A12688918887300212001074AC5
S2140126F012688018C1730C206043034909684018AA
S21401270080680028B9D007E08807002090070020DD
S2140127108C070020840700200C206043CF4A1268F3
S214012720801881680020884796E1012DA5D12001F7
S214012730CB4909684018C07AA84225D0002120015B
S214012740C74A12688018418000202101C44A1268D5
S2140127508918C8802001C24909684018C572C14855
S21401276000782101BE4A12688918487200202101AA
S214012770BB4A126889188880BA4801782001B84A8D
S21401278012688018017267E12001B549096840188E
S214012790007AB4490978884220D0B24800782101ED
S2140127A0AF4A1268891808722001AD4909684018B5
S2140127B0407AAC490978884209D02001A8490968BD
S2140127C0401880882101A64A12688918C88000210D
S2140127D02001A34A12688018818012E02001A049D6
S2140127E0096840188088A04988420AD220019C497D
S2140127F00968401880880A302101994A12688918A8
S2140128008880200196490968401840889649884280
S2140128100AD2200192490968401840880A302101ED
S2140128208F4A12688918488020018D490968401826
S214012830407A8C490978884205D001202101884ACE
S21401284012688918887220018549096840184088ED
S214012850864909680988884204DB00212001804AEC
S2140128601268115220017E4909684018807A0028B2
S2140128707ED10C2060437949096840188068002899
S21401288077D0200176490968401840887749096859
S2140128900989884214DB2001714909684018007BC8
S2140128A000280DD10C2060436C4A1268801881689C
S2140128B00320884701202101694A12688918087394
S2140128C020016749096840184088684909684989AC
S2140128D0884214DB2001624909684018407B0028C1
S2140128E00DD10C2060435D4A12688018816804206F
S2140128F08847012021015A4A126889184873200125
S21401290057490968401840885849096889898842A2
S21401291014DB2001524909684018807B00280DD13C
S2140129200C2060434D4A126880188168052088474C
S214012930012021014A4A12688918887320014849F2
S21401294009684018408849490968C989884210DBE6
S2140129502001434909684018C07B00287CD10C201F
S21401296060433E4A1268801881680620884701E065
S21401297007E03BE001202101394A12688918C87333
S2140129806AE02001364909684018407A01282ED1AC
S2140129903448007802282AD12001314909684018B4
S2140129A0C08832490968498A884255DB20012C498A
S2140129B00968401880882D490968898A88424BDB56
S2140129C00C2060432549096840188068002843D0D8
S2140129D00C206043214A12688018816807208847C6
S2140129E0002021011E4A12688918487234E020012D
S2140129F01B4909684018407A02282DD119480078E9
S214012A00012829D12001164909684018C0881749AC
S214012A100968898A88421FDB200111490968401824
S214012A20808812490968498A884215DB0C20604370
S214012A300A4909684018806800280DD00C206043B8
S214012A40064A1268801881680820884700202101FC
S214012A50034A12688918487270BD00008807002072
S214012A609007002084070020F0FF00008C0700205C
S214012A7010B5002400BF04E02046FFF743FC601CAD
S214012A80C4B202484078A042F6DC10BD840700209C
S214012A9010B50024044802F0BBF8002800D000E07E
S214012AA00124204610BD00000304000010B5074BAA
S214012AB014781C7054785C70054B1960054B1860CF
S214012AC003461833044C236010BD00008407002021
S214012AD0880700208C0700209007002010B50446C8
S214012AE0012C09D1BA220C21002000F0DFF80121C7
S214012AF0022004F0A5F808E000220C21104600F0A0
S214012B00D5F80021022004F09BF810BD10B5002472
S214012B1004210848F8F7D6FA552801D1012407E020
S214012B20042000F0E7FF002801D0002400E0012483
S214012B30204610BD2808002010B50446012C09D1F6
S214012B40BA221C21002000F0B1F80121062004F071
S214012B5077F808E000221C21104600F0A7F80021B3
S214012B60062004F06DF810BD10B50024062000F014
S214012B70C1FF002801D0012400E00024204610BD3A
S214012B8010B50446012C09D1BA221721002000F005
S214012B908DF80121042004F053F808E000221721E3
S214012BA0104600F083F80021042004F049F810BD17
S214012BB000200449097A002901D0012000E0002004
S214012BC070470000D00C002010B50446022C1CD122
S214012BD000220D21104600F069F8FDF7B5FC00282B
S214012BE009D0BA220B21002000F060F801210D2047
S214012BF004F026F847E000220B21104600F056F8B4
S214012C0000210D2004F01CF83DE0032C1CD100220D
S214012C100B21104600F04AF8FDF796FC002809D073
S214012C20BA220D21002000F041F801210D2004F008
S214012C3007F828E000220D21104600F037F80021A1
S214012C400D2003F0FDFF1EE0012C0ED1BA220D214E
S214012C50002000F02BF800220B21104600F026F889
S214012C6001210D2003F0ECFF0DE000220D2110469E
S214012C7000F01CF800220B21104600F017F8002186
S214012C800D2003F0DDFF10BD10B50024FCF7B6FEE5
S214012C90022801D1022406E0FCF7B0FE012801D18A
S214012CA0032400E00124204610BD000010B5064BA9
S214012CB01B78834207DD242905D224234343034C92
S214012CC024681B195A5410BD402B0020C807002049
S214012CD010B574480068407903000BF0B7FB0B078A
S214012CE011D325D35A6D77D38DA8D30007F040FDB5
S214012CF06C4800684079401C6A4909684871CFE011
S214012D0069494969087807F0ABFD6648006840796B
S214012D10401C644909684871624800684079401C53
S214012D20604909684871BBE000F028F9002811D114
S214012D307F2007F095FD5B4800684079401C5949A3
S214012D4009684871574800684079401C5549096828
S214012D5048711DE0534800684078401C5149096895
S214012D60487050480068407803280BD300204D492E
S214012D7009684870AA204B490968887003204949A8
S214012D800968C87007F01EFD0020464909684871A9
S214012D9086E000F0F3F8002807D142480068407941
S214012DA0401C40490968487103E000203D49096814
S214012DB0487107F007FD73E007F0DAFC3948006850
S214012DC04079401C37490968487169E036494969C4
S214012DD00978491CC8B207F043FD324800684079BB
S214012DE0401C3049096848712E4800684079401CEB
S214012DF02C490968487153E000F0C0F800280FD14B
S214012E0007F088FC274909688870012007F0FCFC58
S214012E10244800684079401C22490968487105E049
S214012E2007F0D0FC00201F490968487138E01D48AA
S214012E300068807818280CD102201A4909680870A1
S214012E400020184909684870042016490968C870A6
S214012E5011E0144800684078401C1249096848701F
S214012E60104800684078032805D300F027F90020B1
S214012E700C490968487007F0A5FC00200949096853
S214012E8048710DE007F09EFC00200649096848716C
S214012E90044909684870AA2002490968887000BF79
S214012EA000BF10BDD0070020402B002010B53148D0
S214012EB000684079002804D001280CD0032848D1A6
S214012EC01DE007F055FC2B4800684079401C294955
S214012ED0096848714BE028490969087807F0C0FC81
S214012EE0244800684079401C2249096848712148F5
S214012EF000684079401C1F490968487137E000F0B6
S214012F003DF800280CD101201A49096808700020F4
S214012F10184909684870042016490968C87011E004
S214012F20144800684078401C1249096848701148E6
S214012F3000684078032805D300F0C0F800200D494A
S214012F400968487007F03EFC00200A490968487184
S214012F500DE007F037FC002006490968487105496D
S214012F6009684870AA2003490968887000BF00BF35
S214012F7010BD0000D0070020402B002010B507F040
S214012F80C1FB04461F4800680078002838D01D4859
S214012F900068C078042833D3002C09D100211948D1
S214012FA00068C07A8200174800681430815027E014
S214012FB014480068C07A81001248006814304058EE
S214012FC01149884211D20F480068C07A81000D4825
S214012FD0006814304058401C0A490968C97A8A00BA
S214012FE008490968143188500AE000F067F80021A2
S214012FF004480068C07A8200024800681430815094
S214013000204610BDD0070020B80B000000B587B0E1
S214013010012069460871084802900848039008484C
S2140130200490084805900848069001A9074800F052
S2140130300FF807B000BD000075330100FD4D01001B
S214013040D9E50100B9F50100B8F501003C240020DE
S214013050F8B506460F46002400253946304600F0EE
S214013060EFF900BF14E000250EE0002124206043A4
S2140130700B4A12688018415524206043094A126899
S21401308080184155681CC5B2242DEED3601CC4B20D
S21401309005480078A042E6DC00F010F8F8BD000014
S2140130A0C8070020CC070020402B00200120024941
S2140130B00968087170470000D007002010B500F0BD
S2140130C073F9002003490968087002490968C87045
S2140130D010BD0000D007002007480068C078062809
S2140130E008D105480068C079002803D101200249AB
S2140130F00968C87170470000D007002010B5554810
S2140131000068C07803000BF0A1F908671D1A1714B0
S214013110110E056650484068002803D04E484168A5
S2140131200020884793E000F0E5F890E000F0C6F84C
S2140131308DE000F0D1F88AE0FFF7B8FE87E0FFF7F0
S214013140C7FD84E044484068002803D042484168EF
S214013150012088473F480068407C00281AD03E4836
S214013160C068002803D03C48C168C82088470020B2
S214013170384909684862374800680078002804D052
S214013180042034490968C87024E0022031490968DE
S214013190C8701FE02F480068406A401C2D49096826
S2140131A048622C480068406A7D21C900884211D3D4
S2140131B000202849096848622648006800780028E7
S2140131C004D0042023490968C87003E0022021497D
S2140131D00968C8703BE000BF1F484068002803D05C
S2140131E01D484168002088471A480068407C00282E
S2140131F013D01948C068002803D01748C168C820F2
S2140132008847002013490968486212480068C07858
S214013210401C10490968C87018E00E480068406AEA
S214013220401C0C49096848620A480068406A7D21CA
S214013230C90088420AD30020064909684862054841
S2140132400068C078401C03490968C87000BF00BF09
S21401325010BD0000D0070020402B002010B51548F7
S2140132600068C078072824D00120124909684874EC
S21401327008E011488068002802D00F498868804716
S214013280FFF73CFF0B480068C0780628F1D10948D3
S2140132900068007A0028ECD106480068C07900284A
S2140132A0E7D104480068807A0028E2D1014909681C
S2140132B0487410BDD0070020402B002010B50548EB
S2140132C000680078012802D1FDF732FF01E0F6F729
S2140132D00FFA10BDD007002010B505480068007829
S2140132E0012802D1FEF750F901E0F6F7DFFD10BD27
S2140132F0D007002010B51D480068807A002829D123
S2140133001A480068007A002803D002201749096885
S214013310887216480068C079002803D00120134936
S21401332009688872114800680079012812D10020C6
S2140133300E49096808710D490968887207200B490A
S2140133400968C8700A484068002803D008484168E0
S21401335000208847054800680078012802D1FEF75A
S214013360EDF901E0F6F77CFE10BD0000D007002065
S214013370402B002010B504462146084801F064FCA5
S21401338007480078002805D1002C03D032210548D3
S214013390FCF798FE0248047010BD0000010300000F
S2140133A00401002050C30000002024490968487029
S2140133B0AA202249096888700020204909684862C5
S2140133C01E49096808711D49096848711B49096841
S2140133D088711A490968C871184909680872174935
S2140133E00968887215490968C8721449096808731A
S2140133F024201249096848731049096888730F49DF
S2140134000968C87300200D49096808740B490968E2
S21401341048740A490968887408490968C8740749DC
S2140134200968486100210548006881610348006811
S214013430C16102480068016270470000D0070020A1
S21401344010B50A780D4B1860034628330C4C2360E0
S21401345024235343044628341B190A4C23600A4C80
S2140134604B6863608B68A360CB68E3604B696361FC
S2140134700B6923610B78237010BD0000D007002074
S214013480C8070020CC070020402B00200748006812
S214013490C078062808D105480068007A002803D1BC
S2140134A0012002490968087270470000D007002011
S2140134B010B50446012C09D1BA2220210020FFF7BD
S2140134C0F5FB0121084603F0BBFB08E000222021A2
S2140134D01046FFF7EBFB0021012003F0B1FB10BD06
S2140134E010B50024032000F005FB002801D00124BC
S2140134F000E00024204610BD10B50446032C0ED172
S214013500BA2215210020FFF7D1FB00221421104614
S214013510FFF7CCFB01210E2003F092FB39E0022CD1
S2140135201CD1FDF711F8002809D0BA221421002079
S214013530FFF7BCFB01210E2003F082FB08E000220E
S21401354014211046FFF7B2FB00210E2003F078FB92
S214013550002215211046FFF7A9FB1AE0012C0ED117
S214013560BA2214210020FFF7A1FB01210E2003F04F
S21401357067FB002215211046FFF798FB09E00022A1
S21401358015211046FFF792FB002214211046FFF783
S2140135908DFB10BD10B50024F9F72EF909498842B4
S2140135A00DD3FDF735F8002807D1FCF743FF0128B6
S2140135B001DD032404E0022402E0022400E00124E9
S2140135C0204610BDB80B000010B50446012C09D1E9
S2140135D0BA221D210020FFF769FB0121002003F01C
S2140135E02FFB08E000221D211046FFF75FFB00219C
S2140135F0084603F025FB10BD10B50024022000F09C
S21401360079FA002810D00124104800780A2805DA33
S2140136100E480078401C0D49087015E00A200B4939
S2140136200870002048700FE00024084840780A28F7
S21401363005DA06484078401C0449487004E00A2030
S2140136400249487000200870204610BD2001002065
S21401365010B50446012C09D1BA221E210020FFF71D
S21401366025FB0121092003F0EBFA08E000221E21C8
S2140136701046FFF71BFB0021092003F0E1FA10BDFD
